:100000000C9430170C9469170C9469170C946917A9
:100010000C941E3E0C941E3E0C941E3E0C941E3EF0
:100020000C9469170C9469170C9469170C94691750
:100030000C9469170C940D270C9469170C9469178C
:100040000C9469170C9423250C941DC30C94691708
:100050000C943B820C9431820C9469170C946917B0
:100060000C9469170C9469170C9469170C94691710
:100070000C9469170C9469170C9469170C94691700
:100080000C9469170C9469170C9469174E414E49EA
:100090004E495459494E46CDCCCC3D0AD7233C1746
:1000A000B7D13877CC2B329595E6241FB14F0A0093
:1000B0000020410000C84200401C4620BCBE4CCA83
:1000C0001B0E5AAEC59D7400407A10F35A00A07200
:1000D0004E18090010A5D4E80000E8764817000083
:1000E000E40B54020000CA9A3B000000E1F5050051
:1000F0000080969800000040420F000000A086019A
:10010000000000102700000000E803000000006469
:1001100000000000000A00000000000100000000D4
:10012000002C76D888DC674F0823DFC1DFAE59E1A9
:10013000B1B796E5E3E453C63AE651997696E8E618
:10014000C28426EB898C9B62ED407C6FFCEFBC9CEB
:100150009F40F2BAA56FA5F490055A2AF75C936BFD
:100160006CF9676DC11BFCE0E40D47FEF520E6B5B8
:1001700000D0ED902E0300943577050080841E0892
:100180000000204E0A000000C80C333333330F98B0
:100190006E12831141EF8D2114893BE65516CFFE77
:1001A000E6DB18D1844B381BF77C1D901DA4BBE403
:1001B00024203284725E228100C9F124ECA1E53D45
:1001C000275045544700504C41005072696E7420CE
:1001D00041626F72746564004D3235005061757311
:1001E000696E672E2E2E004D323400454550524F19
:1001F0004D2056657273696F6E204572726F720082
:10020000454550524F4D20496E64657820457272C5
:100210006F7200454550524F4D2043524320457266
:10022000726F72003F0049676E6F726500526573AE
:10023000657400496E697469616C697A6520454529
:1002400050524F4D0000FE0003FF8007C7C007015A
:10025000E00000E00000F00000700400700E00708C
:100260001F00703F80F00E00E00F01E007C7C003E1
:10027000FF8000FE0000FE0003FF8007C7C00F01E3
:10028000E00E00E03F80F01F00700E007004007070
:100290000000700000F00000E00701E007C7C003A5
:1002A000FF8000FE000E000E000E000E000E000E7D
:1002B000000E000E007FC03F801F000E00040004EF
:1002C000000E001F003F807FC00E000E000E000ECB
:1002D000000E000E000E000E00FFFFFF7F80FFC02B
:1002E000FFC0FFC07F807F80FFC0FFC0FFC03F0016
:1002F0001E000C0050726F6265205A204F666673B4
:1003000065740020082046616374002008204D6158
:1003100078002008204D696E004F6666004F6E0021
:100320004175746F74656D700045207374657073EA
:100330002F6D6D005A2053746570732F6D6D0059C9
:100340002053746570732F6D6D0058205374657061
:10035000732F6D6D00416476616E63656420536533
:100360007474696E67730054656D7065726174753D
:1003700072650053746570732F6D6D00436F6E6608
:10038000696775726174696F6E003F004E657874BD
:1003900020436F726E657200446F6E65004E657823
:1003A0007400486F6D696E672058595A0053746F16
:1003B00072652053657474696E6773004C6F616475
:1003C0002053657474696E677300426564205472CB
:1003D000616D6D696E670050726F6265205A204FC3
:1003E0006666736574004661646520486569676880
:1003F00074004F6666004F6E00426564204C65765F
:10040000656C696E67004C6576656C2042656400BA
:100410004732394E00473239004175746F20486FBA
:100420006D65004D6F74696F6E00526573746F7205
:10043000652044656661756C7473004C6F6164205F
:1004400053657474696E67730053746F72652053DB
:10045000657474696E67730050726F6265205A200C
:100460004F666673657400416476616E63656420EF
:1004700053657474696E6773004D61696E003F0067
:100480004261636B0053746F70004D3232004174EF
:1004900074616368204D65646961004D32310050BC
:1004A00072696E742066726F6D204D6564696100BB
:1004B00052656C65617365204D6564696100436FC9
:1004C0006E66696775726174696F6E0054656D70F0
:1004D00065726174757265004D6F74696F6E00525C
:1004E0006573756D65205072696E740054756E6524
:1004F0000053746F70205072696E74005061757390
:1005000065205072696E7400496E666F2053637285
:1005100065656E000A4D3234004D3233202573007C
:100520003F005374617274205072696E74004361AD
:100530006E63656C005072696E740043616E6E6F1D
:100540007420656E746572207375626469723A20F6
:100550000002202E2E000152656672657368004D00
:1005600061696E002100486F74656E6420746F6F5E
:1005700020636F6C64004261636B0050726F63654F
:100580006564004D6F74696F6E0044697361626CDD
:1005900065205374657070657273004D3834004285
:1005A0006564204C6576656C696E67004175746F93
:1005B00020486F6D6500473238004D61696E00C696
:1005C00001C101436F6F6C646F776E005072656894
:1005D00065617420240046616E2053706565640077
:1005E0004E6F7A7A6C65004D61696E0050726F6271
:1005F00065205A204F666673657400466C6F7700FD
:1006000046616E205370656564004E6F7A7A6C6542
:10061000005370656564004D61696E00486F6D69D7
:100620006E67204661696C6564006F70656E00548A
:100630005249474745524544003A20007A5F6D6968
:100640006E00795F6D696E00785F6D696E0052654E
:10065000706F7274696E6720656E6473746F70205A
:100660007374617475730A0020746F6F206C6F6E01
:100670006720657874727573696F6E207072657625
:10068000656E7465640A0020636F6C64206578741D
:10069000727573696F6E2070726576656E746564CD
:1006A0000A00486F6D652025732573257320466900
:1006B000727374005761726E696E673A20486F6D8D
:1006C000696E672042756D702044697669736F7238
:1006D000203C20310A000202040000E0C0000000BB
:1006E000C000000000000068430000634300007A7F
:1006F000430000A0400000A04000000040FFFDFCBF
:10070000FAF8F6F4F2F0EEECEAE9E7E5E3E1E0DE30
:10071000DCDAD9D7D5D4D2D0CFCDCBCAC8C7C5C3E0
:10072000C2C0BFBDBCBAB9B7B6B4B3B2B0AFADAC5E
:10073000AAA9A8A6A5A4A2A1A09E9D9C9A999897B3
:1007400095949392908F8E8D8B8A898887868483E7
:100750008281807F7E7D7B7A7978777675747372FB
:1007600071706F6E6D6C6B6A6968676665646362F1
:1007700061605F5E5D5C5B5A5958585756555453DB
:10078000525150504F4E4D4C4B4A4A4948474646AD
:10079000454443424241403F3E3E3D3C3B3B3A396B
:1007A000383837363535343332323130302F2E2E1B
:1007B0002D2C2B2B2A2929282727262525242323BE
:1007C00022212120201F1E1E1D1C1C1B1B1A191953
:1007D0001818171616151514131312121111100FDD
:1007E0000F0E0E0D0D0C0C0B0A0A0909080807075D
:1007F00006060505040403030202010000000000D0
:100800000100000001000080005555550000004027
:100810000033333300AAAA2A0049922400000020A2
:1008200000C7711C0099991900D14517005555153D
:10083000003BB113002449120011111100000010F7
:10084000000F0F0F00E3380E0043790D00CCCC0CE5
:1008500000C3300C00E8A20B0064210B00AAAA0A16
:1008600000703D0A009DD80900427B0900922409CE
:1008700000DCD30800888808001042080000000847
:1008800000F0C107008787070075500700711C073B
:10089000003EEB0600A1BC060069900600666606F5
:1008A00000703E06006118060017F4050074D105BB
:1008B000005BB00500B29005006272050055550559
:1008C0000078390500B81E0500050505004EEC044A
:1008D0000087D40400A1BD040090A704004992043D
:1008E00000C17D0400EE690400C7560400444404BE
:1008F000005C3204000821040041100400000004E0
:10090000003FF00300F8E0030026D20300C3C30356
:1009100000CCB503003AA803000A9B0300388E03FD
:1009200000C08103009F750300D0690300505E037F
:10093000001D53030034480300913D03003333038B
:100940000016290300381F030097150300300C031D
:1009500000030303000BFA020049F10200BAE802A7
:10096000005CE002002DD802002DD0020059C80220
:1009700000B0C0020031B90200DAB10200AAAA0236
:1009800000A0A30200BC9C0200FA9502005C8F024A
:1009900000DF88020082820200457C020027760286
:1009A0000027700200436A02007C640200D05E02ED
:1009B000003F590200C853020053746F77205A2D2C
:1009C00050726F6265004465706C6F79205A2D50CB
:1009D000726F626500000061430000614300007AAD
:1009E000430000E0C0000000C00000000053657438
:1009F00074696E67732053746F72656400290A000E
:100A00002062797465733B206372632000536574C0
:100A100074696E67732053746F7265642028004593
:100A20004550524F4D206461746173697A65206549
:100A300072726F722E0A00290A002062797465733F
:100A40003B2063726320002073746F7265642073AF
:100A5000657474696E677320726574726965766512
:100A600064202800202863616C63756C6174656480
:100A700029210A0020213D2000454550524F4D209C
:100A8000435243206D69736D61746368202D202883
:100A900073746F7265642920002053697A653A2067
:100AA00000496E6465783A2000204D61726C696E71
:100AB0003D563836290A00454550524F4D2076653F
:100AC0007273696F6E206D69736D6174636820283D
:100AD000454550524F4D3D0048617264636F6465F7
:100AE000642044656661756C742053657474696E26
:100AF0006773204C6F616465640A000000FA43006C
:100B000000FA430000A0400000C8410000A04200DD
:100B100000A0420000C8430080C043F4010000F47C
:100B2000010000640000008813000020286D6D297A
:100B300000203B204C6576656C696E6720002020A4
:100B40004D3432302053004175746F20426564206B
:100B50004C6576656C696E67002046002048002071
:100B6000204D3134352053004D6174657269616CDC
:100B70002068656174757020706172616D6574655F
:100B8000727300204A002020473239205720490044
:100B900020204D3134392043203B20556E69747339
:100BA00020696E2043656C736975730A0054656D26
:100BB000706572617475726520556E69747300207A
:100BC00020473231203B004C696E65617220556EC2
:100BD0006974730024F4D43050C38E20C2A240172D
:100BE000828B7011127A910D816CD90AA861E1088B
:100BF000C7586607615143061E4B5D05C145A704F2
:100C00001A411104093D9803713931034036DB0262
:100C100065339102D4305402802E1D02632CEE0104
:100C2000752AC501B028A001102781018F25640114
:100C30002B244B01E0223401AC211F018D200D013A
:100C4000801FFC00841EED00971DDF00B81CD20041
:100C5000E61BC600201BBC00641AB200B219A80033
:100C60000A19A0006A189900D117910040178B004B
:100C7000B516840031167E00B31579003A1573005D
:100C8000C7146F0058146A00EE13660088136300DF
:100C900025135E00C7125B006C125700151254003A
:100CA000C111510070114F0021114B00D6104900A5
:100CB0008D1047004610440002104200C00F400053
:100CC000800F3E00420F3C00060F3B00CB0E380069
:100CD000930E37005C0E3500270E3400F30D320002
:100CE000C10D3100900D3000600D2E00320D2D0031
:100CF000050D2C00D90C2B00AE0C2900850C290009
:100D00005C0C2700350C27000E0C2600E80B240095
:100D1000C40B2400A00B23007D0B23005A0B2100E1
:100D2000390B2100180B2000F80A1F00D90A1E00F9
:100D3000BB0A1E009D0A1D00800A1D00630A1C00DC
:100D4000470A1B002C0A1B00110A1A00F7091A0097
:100D5000DD091900C4091900AB091900920917002F
:100D60007B091800630917004C09160036091600A4
:100D7000200916000A091500F5081500E0081400FE
:100D8000CC081400B8081400A4081400900813003C
:100D90007D0812006B081300580812004608120064
:100DA0003408110023081100120811000108110075
:100DB000F0071000E0071000D0071000C007100077
:100DC000B0070F00A107100091070E0083070F0066
:100DD00074070F0065070E0057070E0049070E0045
:100DE0003B070D002E070E0020070D0013070D0016
:100DF00006070D00F9060C00ED060D00E0060C00DC
:100E0000D4060C00C8060C00BC060C00B0060C0092
:100E1000A4060B0099060C008D060B0082060B0041
:100E200077060B006C060B0061060A0057060B00E4
:100E30004C060A0042060A0038060A002E060A007E
:100E400024060A001A060A001006090007060A000E
:100E5000FD050900F4050900EB050900E20509009C
:100E6000D9050900D0050900C7050900BE0509001C
:100E7000B5050800AD050800A50509009C0508009A
:100E8000940508008C050800840508007C0508000E
:100E9000740508006C050700650508005D0507007E
:100EA000560508004E0507004705070040050800E5
:100EB00038050700310507002A050700230507004C
:100EC0001C050600160507000F05070008050600AB
:100ED00002050700FB040600F5040700EE04060007
:100EE000E8040600E2040700DB040600D50406005F
:100EF000CF040600C9040600C3040600BD040600B2
:100F0000B7040600B1040500AC040600A604060000
:100F1000A00405009B04060095040500900406004B
:100F20008A04050085040500800406007A04050093
:100F300075040500700405006B04050066040500D7
:100F4000610405005C040500570405005204050017
:100F50004D04050048040500430405003E04040058
:100F60003A04050035040500300404002C04050093
:100F700027040400230405001E0404001A040400CE
:100F800016040500110404000D0404000904050002
:100F90000404040000040400FC030400F80304003B
:100FA000F4030400F0030400EC030400E80304006D
:100FB000E4030400E0030400DC030400D80304009D
:100FC000D4030400D0030400CC030400C8030300CE
:100FD000C503030024F404D9201BC40C5C0E980440
:100FE000C4095F0265077101F405F900FB04B30051
:100FF00048048700C10369005803550003034500F6
:10100000BE023A008402310053022A002902250060
:1010100004022000E4011C00C8011900AF01170000
:101020009801140084011300710110006101100087
:1010300051010E0043010D0036010B002B010B0086
:1010400020010B00150109000C0109000301080033
:10105000FB000800F3000800EB000700E4000600B6
:10106000DE000600D8000600D2000600CC00050015
:10107000C7000500C2000500BD000400B90004005F
:10108000B5000400B1000400AD000400A900040094
:10109000A5000300A20003009F0004009B000300C2
:1010A00098000300950002009300030090000300E5
:1010B0008D0002008B000300880002008600020001
:1010C00084000300810002007F0002007D00020016
:1010D0007B00020079000200770001007600020028
:1010E0007400020072000100710002006F00020033
:1010F0006D0001006C0002006A000100690002003E
:101100006700010066000100650001006400020044
:101110006200010061000100600001005F00020048
:101120005D0001005C0001005B0001005A0001004D
:10113000590001005800010057000100560001004D
:10114000550001005400010053000000530001004D
:101150005200010051000100500001004F00010049
:101160004E0000004E0001004D0001004C00010047
:101170004B0000004B0001004A0001004900010043
:101180004800000048000100470001004600000040
:101190004600010045000000450001004400010038
:1011A0004300000043000100420000004200010033
:1011B0004100000041000100400001003F0000002C
:1011C0003F0001003E0000003E0001003D00000025
:1011D0003D0001003C0000003C0000003C0001001C
:1011E0003B0000003B0001003A0000003A00010013
:1011F000390000003900010038000000380000000C
:101200003800010037000000370001003600000000
:1012100036000000360001003500000035000000F7
:1012200035000100340000003400000034000100EB
:1012300033000000330000003300010032000000E2
:1012400032000000320001003100000031000000D7
:1012500031000100300000003000000030000100CB
:101260002F0000002F0000002F0000002F000100C1
:101270002E0000002E0000002E0001002D000000B6
:101280002D0000002D0000002D0001002C000000AA
:101290002C0000002C0000002C0001002B0000009E
:1012A0002B0000002B0000002B0001002A00000092
:1012B0002A0000002A0000002A0001002900000086
:1012C0002900000029000000290000002900010079
:1012D000280000002800000028000000280000006E
:1012E0002800010027000000270000002700000060
:1012F0002700000027000100260000002600000053
:101300002600000026000000260001002500000045
:101310002500000025000000250000002500000039
:10132000250001002400000024000000240000002B
:10133000240000002400010023000000230000001E
:101340002300000023000000230000002300000011
:101350002300010022000000220000002200000003
:1013600022000000220000002200010021000000F5
:1013700021000000210000002100000021000000E9
:1013800021000000210001002000000020000000DA
:1013900020000000200000002000000020000000CD
:1013A00020000000200001001F0000001F000000BE
:1013B0001F0000001F0000001F0000001F000000B1
:1013C0001F0001001E0000001E0000001E000000A3
:1013D0001E0000003930000033250000871900008E
:1013E000B00F0000DB080000BD0400007402000024
:1013F0003F01000020436F756E7420583A0045315C
:101400000045002C2073797374656D2073746F70C0
:1014100070656421204865617465725F49443A20B3
:101420000048656174696E67204661696C65640097
:1014300048656174696E67206661696C6564004522
:1014400072723A204D415854454D50004D41585408
:10145000454D502074726967676572656400457216
:10146000723A204D494E54454D50004D494E544519
:101470004D502074726967676572656400202F00A3
:1014800020403A007C3C3E5E2B3D3F2F5B5D3B2C79
:101490002A225C00434F4D4D554E49434154494F1C
:1014A0004E0044525952554E004552524F5253002D
:1014B000494E464F004543484F0053544F50504506
:1014C000442E20005072696E7465722073746F70C0
:1014D0007065642064756520746F206572726F7228
:1014E000732E2046697820746865206572726F7269
:1014F00020616E6420757365204D39393920746F11
:1015000020726573746172742E202854656D706545
:101510007261747572652069732072657365742ECB
:101520002053657420697420616674657220726549
:101530007374617274696E67290A004E6F20436884
:1015400065636B73756D2077697468206C696E656F
:10155000206E756D6265722C204C617374204C692D
:101560006E653A20004E6F20436865636B73756D3E
:101570002077697468206C696E65206E756D626590
:10158000722C204C617374204C696E653A200063A4
:101590006865636B73756D206D69736D61746368E5
:1015A0002C204C617374204C696E653A20004C69A4
:1015B0006E65204E756D626572206973206E6F7462
:1015C000204C617374204C696E65204E756D6265A8
:1015D000722B312C204C617374204C696E653A205B
:1015E000004D3131300053657269616C2073746154
:1015F000747573206D69736D617463680A00534478
:101600002072656164206572726F720A0021212068
:101610004B494C4C2063617573656420627920747A
:101620006F6F206D75636820696E6163746976659C
:101630002074696D65202D2063757272656E74204B
:10164000636F6D6D616E643A20004D656469612061
:10165000496E73657274656400627573793A2070BF
:10166000617573656420666F7220696E7075740AA7
:1016700000627573793A2070617573656420666FD6
:101680007220757365720A00627573793A20707200
:101690006F63657373696E670A00506C656173658B
:1016A000205265736574005052494E54455220488B
:1016B000414C5445440025533A202553004B494C96
:1016C0004C45442E20005072696E7465722068612A
:1016D0006C7465642E206B696C6C28292063616CC6
:1016E0006C6564210A006563686F3A004572726F29
:1016F000723A004F4646004F4E0042696C696E6573
:101700006172204C6576656C696E6720477269640A
:101710003A0A0050726F62696E6720506F696E748A
:101720000025532025692F2569002E0A002F00501F
:10173000726F62696E67206D65736820706F696E85
:10174000742000202844525952554E2900473239FE
:10175000204175746F20426564204C6576656C6924
:101760006E67003F20284C2C522C462C4229206FBB
:101770007574206F6620626F756E64732E0A003F69
:101780002856296572626F7365206C6576656C20DA
:10179000696D706C61757369626C652028302D34D9
:1017A000292E0A00426164205A2076616C75650A10
:1017B000004E6F2062696C696E65617220677269A4
:1017C000640A004732384C300020204D323031203E
:1017D00058004D617820416363656C65726174697E
:1017E0006F6E2028756E6974732F73322900202064
:1017F0004D3230332058004D617820666565647243
:10180000617465732028756E6974732F73290020C5
:10181000520020204D323034205000416363656C0B
:1018200065726174696F6E2028756E6974732F73A9
:1018300032292028503C7072696E742D6163636593
:101840006C3E20523C726574726163742D616363F7
:10185000656C3E20543C74726176656C2D616363E7
:10186000656C3E2900204A002054002053002020AF
:101870004D323035204200416476616E63656420EC
:1018800028423C6D696E5F7365676D656E745F7449
:10189000696D655F75733E20533C6D696E5F66656B
:1018A0006564726174653E20543C6D696E5F74724C
:1018B0006176656C5F66656564726174653E204A39
:1018C0003C6A756E635F6465763E290020440020A3
:1018D000490020204D333031205000486F74656E30
:1018E0006420504944002E0A00206E6F7420646901
:1018F0007361626C65642E20536861726564207741
:101900006974680020496E76616C6964206578743A
:1019100072756465722000536C6565702E2E2E0002
:101920005A2050726F626520506173742042656462
:101930000A005A2050726F62652050617374204211
:10194000656400205A3A200020593A20004265641C
:1019500020583A20004D65736820706F696E7420BE
:101960006F7574206F662072616E67650A00436C44
:1019700069636B20746F20526573756D652E2E2E12
:1019800000616C736F20656E61626C6564290A008A
:101990004E6F204D6F76652E004E6F206D65646929
:1019A000610A00456E642066696C65206C69737419
:1019B0000A00426567696E2066696C65206C697310
:1019C000740A00286E6F2066696C6529004E6F747A
:1019D000205344207072696E74696E670A00534424
:1019E000207072696E74696E672062797465200078
:1019F00043757272656E742066696C653A20002EBC
:101A00000A0044656C6574696F6E206661696C6577
:101A1000642C2046696C653A200046696C65206438
:101A2000656C657465643A002569730025696D20ED
:101A3000256973002569682025696D202569730073
:101A4000256964202569682025696D202569730052
:101A500025697920256964202569682025696D201C
:101A6000256973005072696E742074696D653A203F
:101A7000006F6B006F666600B514B014A914A21451
:101A8000941444454255473A004D31313220536851
:101A90007574646F776E004D3131332053004D659E
:101AA0006761205A65726F204F46462E00434F4EA5
:101AB0004649475F4558504F5254004D4541545098
:101AC00041434B00434F4F4C45525F54454D5045A9
:101AD000524154555245004348414D4245525F548E
:101AE000454D50455241545552450042414259538B
:101AF00054455050494E470041524353004D4F54B6
:101B0000494F4E5F4D4F44455300544845524D4157
:101B10004C5F50524F54454354494F4E0045585422
:101B2000454E4445445F4D3230004C4F4E475F4672
:101B3000494C454E414D45004155544F5245504F3B
:101B400052545F53445F5354415455530053445FC0
:101B5000575249544500524550454154005344435F
:101B60004152440050524F4D50545F535550504FC6
:101B7000525400484F53545F414354494F4E5F43C2
:101B80004F4D4D414E445300454D455247454E4300
:101B9000595F50415253455200434153455F4C49B0
:101BA0004748545F4252494748544E4553530054A6
:101BB0004F47474C455F4C494748545300534F46A5
:101BC00054574152455F504F574552004255494C7A
:101BD000445F50455243454E54004C4556454C4990
:101BE0004E475F44415441005A5F50524F424500B6
:101BF00052554E4F5554004155544F4C4556454C47
:101C0000005052494E545F4A4F420050524F475283
:101C1000455353004155544F5245504F52545F5411
:101C2000454D50004155544F5245504F52545F500E
:101C30004F5300564F4C554D45545249430045456E
:101C400050524F4D0042494E4152595F46494C4512
:101C50005F5452414E534645520053455249414C00
:101C60005F584F4E5F584F4646004649524D5741C8
:101C700052455F4E414D453A4D61726C696E20325E
:101C80002E302E392E332D6B61643120284465634C
:101C900020323720323032312031333A35303A3544
:101CA000392920534F555243455F434F44455F55B3
:101CB000524C3A6769746875622E636F6D2F6B6161
:101CC000642F4D61726C696E2050524F544F434FD8
:101CD0004C5F56455253494F4E3A312E30204D41BC
:101CE0004348494E455F545950453A4D6567612018
:101CF0005A65726F2045585452554445525F434FC0
:101D0000554E543A3120555549443A6462666363EE
:101D10006435352D656262612D343631352D616251
:101D200064372D3139366161343338663330340AE3
:101D3000002F2F004D31343520533C696E64657897
:101D40003E206F7574206F662072616E6765202873
:101D5000302D31290A003F4A206F7574206F6620AC
:101D600072616E67652028302E303120746F20300C
:101D70002E33290A0020580020204D61783A200097
:101D8000200020204D696E3A2000203B20002020BA
:101D90004D32313120530046523A0020466C6F7765
:101DA0003A200050726F6265204F6666736574203A
:101DB0005A0050726F6265204F6666736574205AD0
:101DC0000064697300656E0043290A0061626C65F6
:101DD0006420286D696E2074656D702000436F6CFF
:101DE0006420657874727564657320617265200083
:101DF0004F46460A00466164652048656967687415
:101E00002000426564204C6576656C696E67200031
:101E10004661696C656420746F20656E61626C65F3
:101E200020426564204C6576656C696E670A0049DE
:101E30006E76616C6964206D6573682E0A004D349E
:101E4000323120696E636F727265637420706172E3
:101E5000616D657465722075736167650A004D6513
:101E6000736820706F696E74206F7574206F6620C0
:101E700072616E67650A00454550524F4D204F4BC9
:101E80000A00290A0020746F20003F5A206F7574E1
:101E9000206F662072616E6765202800290A002085
:101EA000746F20003F59206F7574206F6620726137
:101EB0006E676520282D00290A0020746F20003FDE
:101EC00058206F7574206F662072616E67652028D8
:101ED0002D004D383400446F6E65207072696E7449
:101EE000696E672066696C650A004D3737004D33AF
:101EF0003100496E76616C6964206578747275642E
:101F000065720A004361703A00203B0020204D3882
:101F100035312058005A2D50726F6265204F666629
:101F200073657400436F6F6C696E672E2E2E0048C8
:101F3000656174696E672E2E2E0045312025530091
:101F400020573A0023646566696E65204445464122
:101F5000554C545F004B6420004B6920004B7020AF
:101F600000504944204175746F74756E6520666930
:101F70006E697368656421205075742074686520EB
:101F80006C617374204B702C204B6920616E64204F
:101F90004B6420636F6E7374616E74732066726F2E
:101FA0006D2062656C6F7720696E746F20436F6E71
:101FB00066696775726174696F6E2E680A005049B0
:101FC00044204175746F74756E65206661696C6537
:101FD00064212074696D656F75740A00504944204E
:101FE0004175746F74756E65206661696C656421F6
:101FF0002054656D706572617475726520746F6FC1
:1020000020686967680A00504944204379636C6519
:10201000730025532025692F256900204B643A2041
:1020200000204B693A2000204B703A200020436C7E
:10203000617373696320504944200A002054753A43
:102040002000204B753A2000206D61783A20002056
:102050006D696E3A200020643A2000206269617345
:102060003A20005761697420666F72206865617458
:102070002075702E2E2E00504944204175746F74C7
:10208000756E652073746172740A00504944204172
:1020900075746F74756E65206661696C6564212066
:1020A00054656D706572617475726520746F6F2010
:1020B000686967680A00504944204175746F7475F7
:1020C0006E65206661696C656421204261642068E8
:1020D00065617465722069640A0050494420417545
:1020E000746F74756E65004572723A207574663847
:1020F00020666F6E74206E6F7420696E69746961FA
:102100006C697A65642E004572723A20757466387F
:1021100020666F6E74206E6F7420696E69746961D9
:102120006C697A65642E004572723A20757466385F
:1021300020666F6E74206E6F7420696E69746961B9
:102140006C697A65642E002568753A2530326875A9
:102150000025303268753A253032687500253032F6
:10216000687527253032687500256875642025302C
:102170003268753A25303268750042656400456EF4
:10218000636C6F7375726500202020202020200072
:102190002020202000453A00523A00657272001F4C
:1021A000E0201020102010102010202010201030CF
:1021B000300840048003001FE03FF03FF03FF01F75
:1021C000E01FE03FF03FF03FF00FC0078003003F0B
:1021D000FFF038007030FC3020FC102078102030E8
:1021E000102C00D02E31D02F7BD02F7BD02E31D091
:1021F0002C00D020301020781020FC1030FC30381B
:1022000000703FFFF03FFFF03800703186302387C9
:10221000102787902F87D02F03D0203010207810E0
:102220002078102030102F03D02F87D027879023BD
:1022300087103186303800703FFFF0001DC43F002A
:1022400000000C86198000000D0E198000000F0B95
:10225000198000000D9F198000000DD399800000A7
:102260001CFBFF0000000000000000000000000058
:1022700000F380001F80007700001980005B1CF6CF
:10228000131DAE5B35AB0635FB5B3DA70CBD9B4B11
:1022900030EB19B19BE39D8E9F9D8E0001E0000005
:1022A000000001200000000001E0000000000C0F11
:1022B00000FE07022503BB017FFE08FE08FE05089D
:1022C0000806000040F0C8888898781005080806BD
:1022D0000000C0F88888888888F805050506000190
:1022E0002030F830200508080600002070F8202073
:1022F0002020E00509090600FF2070A8A8B88888FA
:102300007020070505070001D86C366CD80509094F
:102310000600FFF8A88888888888A8F8050A0A06B1
:1023200000FE205050505088A8A888700303030670
:10233000000340A040FFFFFFFFFFFFFFFFFFFFFF85
:10234000FFFFFFFFFFFFFFFFFFFFFF00000006058D
:10235000FF01070706020080808080800080030361
:1023600003060105A0A0A005060606000050F850CF
:1023700050F8500509090600FF2070A8A07028A891
:102380007020050707060000C8C81020409898056F
:10239000070706000040A0A040A8906801030306BC
:1023A00002058080800309090601FF2040408080EB
:1023B000804040200309090601FF80404020202082
:1023C00040408005070706000020A8702070A82064
:1023D0000505050600012020F82020020303060160
:1023E000FFC04080050101060003F8020202060159
:1023F00000C0C005070706000008101020404080FC
:10240000050707060000708898A8C88870030707AA
:1024100006010040C040404040E0050707060000BC
:10242000708808102040F8050707060000F808101B
:102430003008887005070706000010305090F8102B
:1024400010050707060000F880F0080888700507E7
:1024500007060000304080F08888700507070600F6
:1024600000F80810102020200507070600007088DB
:1024700088708888700507070600007088887808CB
:102480001060020505060100C0C000C0C0020606BB
:102490000601FFC0C000C040800305050601012001
:1024A00040804020050303060002F800F8030505FC
:1024B0000601018040204080050707060000708863
:1024C00010202000200507070600007088B8A8B873
:1024D0008070050707060000708888F888888805DE
:1024E0000707060000F04848704848F0050707064F
:1024F000000070888080808870050707060000F063
:102500004848484848F0050707060000F88080F072
:102510008080F8050707060000F88080F080808042
:1025200005070706000070888080988870050707F7
:10253000060000888888F888888803070706010055
:10254000E04040404040E00507070600003810101A
:10255000101090600507070600008890A0C0A090AA
:1025600088050707060000808080808080F80507C6
:102570000706000088D8A88888888805070706000D
:10258000008888C8A8988888050707060000708812
:102590008888888870050707060000F08888F08022
:1025A000808005070706000070888888A890680565
:1025B0000707060000F08888F0A090880507070646
:1025C000000070888070088870050707060000F812
:1025D0002020202020200507070600008888888802
:1025E0008888700507070600008888888850502072
:1025F00005070706000088888888A8A850050707EF
:1026000006000088885020508888050707060000CB
:1026100088885020202020050707060000F80810B1
:10262000204080F80309090601FFE0808080808057
:102630008080E00507070600008040402010100859
:102640000309090601FFE020202020202020E005CA
:1026500003030600052050880501010600FEF8036B
:1026600003030601058040200505050600007008EB
:102670007888780507070600008080F0888888F051
:1026800005050506000070808088700507070600B4
:102690000008087888888878050505060000708895
:1026A000F08070050707060000304840E0404040D9
:1026B0000507070600FE70888888780870050707F8
:1026C0000600008080F088888888030707060100DC
:1026D0004000C0404040E00409090601FE100030FF
:1026E0001010101090600507070600008080889089
:1026F000E09088030707060100C04040404040E0EA
:10270000050505060000D0A8A8A8A805050506002F
:1027100000B0C8888888050505060000708888888C
:10272000700507070600FEF0888888F0808005079E
:10273000070600FE788888887808080505050600E1
:1027400000B0C8808080050505060000788070080C
:10275000F00507070600002020F8202020180505B6
:102760000506000088888898680505050600008829
:10277000888850200505050600008888A8A850050F
:10278000050506000088502050880507070600FE52
:1027900088888850204080050505060000F8102034
:1027A00040F80309090601FF2040404080404040B6
:1027B000200109090602FF8080808080808080805F
:1027C0000309090601FF8040404020404040800549
:1027D000030306000248A890FF43616E6E6F7420E9
:1027E0006F70656E207375626469722000534420B7
:1027F00063617264206F6B0A006F70656E526F6F59
:1028000074206661696C65640A00766F6C756D652D
:102810002E696E6974206661696C65640A004E6F8A
:1028200020534420636172640A002E0A006F7065B1
:102830006E206661696C65642C2046696C653A207F
:102840000046696C652073656C65637465640A0095
:102850002053697A653A200046696C65206F70657F
:102860006E65643A2000454E4420535542524F5500
:1028700054494E450A002220706F73002220706177
:1028800072656E743A2200535542524F5554494E68
:10289000452043414C4C207461726765743A2200B4
:1028A00053756263616C6C204F766572666C6F77EE
:1028B000004578636565646564206D6178205355D3
:1028C00042524F5554494E452064657074683A0031
:1028D000667265736800646F696E67002066696C74
:1028E000653A20004E6F77200057726974696E67F1
:1028F00020746F2066696C653A20006D61726C69A6
:102900006E66772E6F726700322E302E392E332D81
:102910006B616431001FFFFFFFFFFFFF60000000DD
:102920000001FF400000000000FF800000000000E8
:102930007F83CF00000C303F87FF80000C301F8664
:102940007980000C000F8C30C7838C30E78C30CF3F
:10295000C7CC31F38C30DCECEC33B98C30D86C6CF8
:1029600033198C30D06C0C33198C30D86C0C331973
:102970008C30DC6C0E3B198C30CF7C079F198C306F
:10298000C77C038F194000000000000260000000B7
:102990000000061FFFFFFFFFFFF870012C019001F0
:1029A0002701B0012201C0011D01F0011801100230
:1029B000130130020E016002090190020401C002FD
:1029C000FF000003FA004003F5008003F000D0038D
:1029D000EB002004E6007004E100E004DC004005A8
:1029E000D700C005D2004006CD00D006C800800741
:1029F000C3003008BE00F008B900C009B400B00A36
:102A0000AF00B00BAA00D00CA500000EA000500F24
:102A10009B00C01096005012910000148C00C0154D
:102A20008700B0178200B0197D00D01B7800001E0F
:102A3000730040206E0090226900F024640040275B
:102A40005F0090295A00E02B5500102E50002030D6
:102A50004B0010324600E033410090353C00103707
:102A6000370070383200A0392D00B03A2800A03B62
:102A70002300603C1E00103D1900903D1400103EE4
:102A80000F00703E0A00C03E0500003F0000403FBE
:102A9000FBFF803FF6FFC03FF1FF2020506C616ECE
:102AA0006E657242756666657242797465733A2026
:102AB000002046726565204D656D6F72793A200081
:102AC00020436F6D70696C65643A20446563203201
:102AD0003720323032310A00204C61737420557037
:102AE00064617465643A20323032312D30392D30D2
:102AF00033207C20417574686F723A20286B6164C2
:102B00002C20416E796375626963204D6567612091
:102B10005A65726F2041424C20313256290A004DCD
:102B200061726C696E20322E302E392E332D6B611E
:102B300064310A0020536F667477617265205265B4
:102B40007365740A00205761746368646F6720526C
:102B5000657365740A002042726F776E206F75741A
:102B60002052657365740A002045787465726E6141
:102B70006C2052657365740A00506F7765725570EA
:102B80000A0073746172740A004732385859004D54
:102B900031303031006572726F72207772697469FA
:102BA0006E6720746F2066696C650A00446F6E65FD
:102BB00020736176696E672066696C652E0A004D28
:102BC000323900456E6473746F707300255320258D
:102BD0006320256320256320256300205A3A0020C6
:102BE000593A0020583A00656E6473746F70732010
:102BF0006869743A2000000000010200090A000020
:102C000000000403080700000000000000000000AE
:102C1000000000000000004D6F76652025736D6D8B
:102C2000004D6F766520302E316D6D004D6F7665ED
:102C300020316D6D004D6F76652031306D6D004D2A
:102C40006F76652041786973004D6F766520457811
:102C5000747275646572004D6F7665205A004D6F11
:102C600076652059004D6F76652058005072696E68
:102C7000742066726F6D204D6564696100FFFFFF0F
:102C8000205A3A200020593A200042656420583AE0
:102C900020004D656761205A65726F20526561643E
:102CA000792E005072696E74696E672E2E2E005058
:102CB00072696E742050617573656400220A005554
:102CC0006E6B6E6F776E20636F6D6D616E643A2010
:102CD00022006F6B00204500205A00205900202060
:102CE0004D3932205800537465707320706572201E
:102CF000756E6974003B2000DB0FC93F45BCDA3FAD
:102D00008FB30240FCF0274056946140FE4B9B403D
:102D100084A5D840E0231841346A5641E8599741C8
:102D200064DBD5416E271742B4B75542CE1A97429D
:102D3000C8AED542B5885A43D40684BFA65FA7BFA4
:102D40007443E0BF10B11AC01C2C58C0E8F697C0FD
:102D5000B849D6C04E4E17C124D355C1802497C15F
:102D6000A0B5D5C1121A17C244AE55C2781797C282
:102D70006CACD5C267885AC320746F6F206C6F6EBD
:102D80006720657874727573696F6E2070726576EE
:102D9000656E7465640A0020636F6C6420657874E6
:102DA000727573696F6E2070726576656E74656496
:102DB0000A006F6B0A00526573656E643A2000204A
:102DC000453A00205A3A0020593A00583A0000008B
:102DD0002200250028002B000000210024002700ED
:102DE0002A00020202020202020204040404040491
:102DF00004040303030303030303010101010101AD
:102E00000101010204081020408001020408102082
:102E100040800102040810204080804020100804F7
:102E200002014572726F722077726974696E672051
:102E3000746F20454550524F4D210A005448455269
:102E40004D414C2052554E415741590054686572CE
:102E50006D616C2052756E6177617900F0D02BD76F
:102E600011241FBECFEFD0E4DEBFCDBF84B7809367
:102E7000331514BE0FB6F894A89580916000886150
:102E800080936000109260000FBE12E0A0E0B1E0FD
:102E9000E4E8FAEC01E00BBF02C007900D92AC38F9
:102EA000B107D9F725E1ACE8B2E001C01D92A33328
:102EB000B207E1F717E1CFE2D7E104C02197FE01A5
:102EC0000E948AE2CE32D107C9F70E949AD10C94AF
:102ED00036E50C940000A0E1B0E0E1E7F7E10C94E6
:102EE000B9E28C01DC01ED91FC910280F381E02DCF
:102EF000BE016F5F7F4F0995882309F45DC089810A
:102F0000807C91F56F81637070E0762F6627770F74
:102F1000770F8885B4E08B9FC0011124682B792B33
:102F200089858295869586958370682B6F5F7F4F24
:102F300090E080E02A852370220F3B8537FB332702
:102F400030F9232B3E813F70230F3327331F275047
:102F5000310904C0660F771F881F991F2A95D2F781
:102F60006096E4E00C94D5E2803419F568856695A6
:102F7000669570E090E080E0CB01772766272A8590
:102F8000622B098510E0102F0027012E000C220B68
:102F9000330B602B712B822B932B6F5F7F4F8F4FE7
:102FA0009F4F4AE0660F771F881F991F4A95D1F7F8
:102FB000D7CF8BE0F801848360E070E0CB01D0CF05
:102FC0000895FC0182810895FC0190E1A0E7B4E03E
:102FD00001900D929A95E1F70895EF92FF920F9369
:102FE0001F93E0928F03F09290030093910310934C
:102FF0009203B62F172F022FF32E242F582FB093A2
:10300000930310939403509395036FEFFF27B01B26
:103010001F09520B30F450951095B195160B560BB5
:10302000662760939104A6E0BA9F00928504712DF3
:10303000EE271A9F700DE11D5A9FE00D70938604D4
:10304000E0938704AFE0BA9F00928904712DEE27C8
:103050001A9F700DE11D5A9FE00D70938A04E09352
:103060008B04AAE0BA9F00928D04712DEE271A9F5F
:10307000700DE11D5A9FE00D70938E04E0938F0454
:103080001F910F91FF90EF900895A5E0B0E0EBE461
:10309000F8E10C94B2E26F3671058105910578F480
:1030A000FB01EE0FFF1FEE0FFF1FE350F84F65917E
:1030B0007591859194912596EBE00C94CEE2F62ED5
:1030C000E72E282FEDEFF6E00027BB275F2D8E2D92
:1030D000922F992341F4982F852FB85F992319F4E3
:1030E000982F8827B85F903138F482959295582FA1
:1030F0005F70807F952BBC5F903428F4880F991FF8
:10310000880F991FBE5F903818F4880F991FB395E8
:10311000880F991FE90FF01F549181E09927B8504B
:1031200079F1C0F0B0FF02C0550F881FB1FF04C095
:10313000550F881F550F881FB2FF06C08295529504
:10314000152F1F70507F812BB3FF1AC0982F852F2A
:10315000552716C0B195B0FF02C085955795B1FFB0
:1031600004C08595579585955795B2FF05C0829502
:10317000507F5295582B8F70B3FF02C0582F88276D
:10318000BB247727AA27B2E0F59EB0187109A00BDF
:10319000B00BE59E7019A109B00B259FA019B109CC
:1031A000F89E7019A109B00BE89EA019B109289FDB
:1031B000B019F99EA019B109E99EB0195B9DA12C27
:1031C00099244427662733278B9DA00C911C401F10
:1031D000601F301F9B9D900C411D601F301F579F2B
:1031E000A00C911C401F601F301F879F900C411D39
:1031F000601F301F979F400D611D301F5A9F900C1C
:10320000411D601F301F8A9F400D611D301F9A9F16
:10321000600D311D5B9F400D611D301F8B9F600D48
:10322000311D9B9F300DB1E0AA277727BB24F49E68
:10323000B0187109A00BB00BE49E7019A109B00B76
:10324000249FA019B109F69E7019A109B00BE69E42
:10325000A019B109269FB019F39EA019B109E39EE8
:10326000B019BF187E09A20B20F0B1E04B0F601F10
:10327000301F1124762F642F90E0832F1CCFFC0188
:103280007081472F50E0062E02C0559547950A944D
:10329000E2F740FF14C04091080450E0062E02C03F
:1032A000559547950A94E2F740FF09C021E030E0C8
:1032B00001C0220F6A95EAF72095272320830895FD
:1032C0008F929F92AF92BF92CF92DF92EF92FF9236
:1032D000FC01C080D180E280F38020E030E048EC47
:1032E00052E4C701B6010E942ADC4B015C0120E0D8
:1032F00030E0A901C701B6010E94C5DB20E030E043
:1033000040EA50E487FF04C020E030E040EA50EC9F
:10331000C501B4010E94E3E22DEC3CEC4CEC5DE312
:103320000E942ADC0E94C2E39B018BE237FF05C0AA
:1033300022273327261B370B8DE280939502C90184
:1033400068EE73E00E945BE2CB01EAE0F0E0BF01CF
:103350000E945BE2805D80939602C90164E670E0A2
:103360000E945BE2CB01BF010E945BE2805D809323
:103370009702C901BF010E945BE29C01CB01BF0122
:103380000E945BE2805D809398028EE280939902B6
:10339000205D20939A0285E992E0FF90EF90DF9004
:1033A000CF90BF90AF909F908F9008954F925F9273
:1033B0006F927F928F929F92AF92BF92CF92DF9245
:1033C000EF92FF92FC01C080D180E280F38020E088
:1033D00030E04AE754E4C701B6010E942ADC4B0101
:1033E0005C0120E030E040E251ECC701B6010E94F0
:1033F000C5DB181654F420E030E048EC52E4C70175
:10340000B6010E9446E487FD8AC020E030E0A901B1
:10341000C701B6010E94C5DB87FF72C060E070E0A3
:1034200080EA90ECA50194010E94E3E22DEC3CECD3
:103430004CEC5DE30E942ADC0E94C2E36B017C013C
:10344000F7FC63C020E137E240E050E00E946EE20A
:10345000CA01B9012AE030E040E050E00E946EE28B
:10346000605D60939502C701B60128EE33E040E04D
:1034700050E00E946EE29AE0892E912CA12CB12C92
:10348000CA01B901A50194010E946EE2605D6093DA
:103490009602C701B60124E630E040E050E00E9409
:1034A0006EE2CA01B901A50194010E946EE2605D5D
:1034B000609397028EE280939802C701B601A5013E
:1034C00094010E946EE26B01CA01B901A501940149
:1034D0000E946EE2605D60939902F0E3CF0EC092AD
:1034E0009A0285E992E0FF90EF90DF90CF90BF9035
:1034F000AF909F908F907F906F905F904F900895C6
:1035000060E070E080EA90E48DCFF094E094D09495
:10351000C094C11CD11CE11CF11C6DE2A2CF20E0C3
:1035200030E0A901C701B6010E94C5DB87FF6BC06F
:1035300060E070E080EA90ECA50194010E94E3E273
:103540002DEC3CEC4CEC5DE30E942ADC0E94C2E3D3
:103550004B015C0120E030E0A901C701B6010E94E7
:10356000C5DB87FD0BC020E030E040E251E4C7013D
:10357000B6010E9446E460E287FD13C0B7FC48C074
:10358000C501B40128EE33E040E050E00E946EE255
:10359000CA01B9012AE030E040E050E00E946EE24A
:1035A000605D60939602C501B40124E630E040E01E
:1035B00050E00E946EE28AE0482E512C612C712C62
:1035C000CA01B901A30192010E946EE2605D60939D
:1035D00097028EE280939802C501B401A301920183
:1035E0000E946EE26B01CA01B901A30192010E941F
:1035F0006EE2605D6093990280E3C80EC0929A0209
:1036000086E992E070CF60E070E080EA90E494CFC9
:10361000B094A09490948094811C911CA11CB11C26
:103620006DE2BFCF282F81E3243609F080E280933A
:10363000970290E22A3040F03AE0822F632F0E94F6
:103640002EE20E942EE2905D90939802822F6AE013
:103650000E942EE2905D9093990285E280939A02F7
:1036600087E992E0089560912C0170912D01072E59
:10367000000C880B990B0E94CBDB2AE037ED43E26C
:103680005CE30E942ADC60936C0170936D0180936F
:103690006E0190936F010895CF93DF93EC01CB01FE
:1036A000BA010E94CBDB23E333E343E250E40E9400
:1036B0002ADC20E030E040E05FE30E94E3E20E9489
:1036C000C7E36883DF91CF9108950E94CBDB23E3AA
:1036D00033E343E250E40E942ADC20E030E040E0A3
:1036E0005FE30E94E3E20E94C7E324E6629FC00119
:1036F000112481589F4F6FEF70E00E945BE2862F8C
:1037000091CF80914707811104C080911E0780935B
:103710007D070895809178148823C1F081508093AB
:103720007814EFECF2E1882351F08150990B2BE1F2
:10373000289FF001299FF00D1124E659FC4E8BE1E2
:10374000A4EBB2E101900D928A95E1F720917814F3
:10375000211105C08091821480648093821481E0DD
:1037600090E0A0E0B0E0211103C080E090E0DC0137
:1037700080933D0790933E07A0933F07B093400787
:103780001092380781E080933A0783E080936701C5
:103790000895CF93DF93EC01CB01BA010E94CBDBFC
:1037A000688379838A839B83DF91CF910895CF9338
:1037B000DF93EC01CB01BA010E94CBDB2DEC3CEC9A
:1037C0004CEC5DE30E942ADC688379838A839B83C7
:1037D000DF91CF910895CF93DF93EC01CB01BA0134
:1037E0000E94CBDB2AE037ED43E25CE30E942ADC57
:1037F000688379838A839B83DF91CF910895CF92E9
:10380000DF92EF92FF92CF93DF9300D000D0CDB73D
:10381000DEB70E94CBDB2AE037ED43E25CE30E9497
:103820002ADC6B017C0120E030E0A9010E94C5DBAD
:103830002DEB37E346E055E387FF04C02DEB37E37C
:1038400046E055EBC701B6010E94E3E269837A8343
:103850008B839C83CE010196A9DD0F900F900F9072
:103860000F90DF91CF91FF90EF90DF90CF90089570
:10387000CF93DF93EC01CB01BA010E94CBDB0E9416
:10388000C2E379836883DF91CF9108958F929F92ED
:10389000AF92BF92CF92DF92EF92FF92FC01C08075
:1038A000D180E280F38020E030E0A901C701B601B9
:1038B0000E94C5DB87FD99C06DEB77E386E095E359
:1038C000A70196010E94E3E29F7720E030E048ECF8
:1038D00052E40E942ADC20E030E040EA50E40E94FA
:1038E000E3E22DEC3CEC4CEC5DE30E942ADC0E9410
:1038F000C2E36B017C0180E28093940260E2F0E11C
:10390000CF16F7E2DF06E104F1048CF0C701B6013F
:1039100020E137E240E050E00E946EE2CA01B901C6
:103920002AE030E040E050E00E946EE2605D60938B
:10393000950260E288EEC81683E0D806E104F1043F
:103940008CF0C701B60128EE33E040E050E00E9461
:103950006EE2CA01B9012AE030E040E050E00E9486
:103960006EE2605D6093960260E2E4E6CE16D104FA
:10397000E104F1048CF0C701B60124E630E040E038
:1039800050E00E946EE2CA01B9012AE030E040E056
:1039900050E00E946EE2605D609397028AE0882E9C
:1039A000912CA12CB12CC701B601A50194010E9454
:1039B0006EE26B01CA01B901A50194010E946EE299
:1039C000605D609398028EE280939902F0E3CF0EDF
:1039D000C0929A0284E992E0FF90EF90DF90CF903E
:1039E000BF90AF909F908F9008956DEB77E386E046
:1039F00095EB66CFA4E0B0E0E0E0FDE10C94BBE223
:103A00000E94CBDB2DEC3CEC4CEC5DE30E942ADC0D
:103A100069837A838B839C83CE01019637DF24965A
:103A2000E2E00C94D7E2CF93DF93EC018D810E940A
:103A3000718260E08B810E94F4C0DF91CF91089584
:103A4000CF92DF92EF92FF920F931F93CF938C014F
:103A5000C62F69017A01E7DF0E94FDC28C2F8064C6
:103A60000E9465828F2D0E9465828E2D0E94658244
:103A70008D2D0E9465828C2D0E94658287E8C11180
:103A800001C085E90E946582CC3011F40E946A82EF
:103A9000C0E00E946A82F801868387FF04C0CF3F9E
:103AA00011F0CF5FF6CFCF911F910F91FF90EF9064
:103AB000DF90CF90089561E0FC0183810E94F4C003
:103AC0008FEF0C9465820F931F93CF938C01ABDF24
:103AD0000E94FDC2C82F882369F08DEF0E94658285
:103AE0000E94FDC2C82FC801E6DF8C2FCF911F9125
:103AF0000F91089582E1F8018483F5CFB0E0A0E052
:103B0000E4E8FDE10C94B1E2EC016A017B014801BB
:103B1000590120E030E0A90167E392DFA501980197
:103B200067E1CE018DDF81111DC08F81833039F0B7
:103B300089E0CC0CDD1CEE1CFF1C8A95D1F7A70197
:103B4000960169E1CE017CDF11E0882319F010E0D5
:103B500087E08C83CE01AFDF812FCDB7DEB7ECE0FD
:103B60000C94CDE289E08C8310E0F4CFCF93DF9307
:103B7000EC016EBDFA01CA019E5F0DB407FEFDCFD8
:103B800020812EBD0DB407FEFDCF21812EBD3296C2
:103B9000E817F90791F70DB407FEFDCF8FEF0E94EC
:103BA00065828FEF0E9465820E946A828E838F7188
:103BB000853041F083E18C83CE017DDF80E0DF91B1
:103BC000CF91089581E0FBCF0F931F93CF93DF93A5
:103BD000EC018B0128DF0E94FDC281110BC085E141
:103BE0008C8310E0CE0167DF812FDF91CF911F9191
:103BF0000F910895A8016CEFCE01B8DF182F88232C
:103C000071F3F0CF0F931F93CF93DF93EC018901F2
:103C10008F81833039F089E0440F551F661F771F6D
:103C20008A95D1F79A01AB0168E1CE0109DF8111D4
:103C300027C0A8016EEFCE0199DF182F8823A9F0C5
:103C40000E94FDC2182F8823C1F020E030E0A901B6
:103C50006DE0CE01F5DE882321F086E18C8310E053
:103C600004C00E946A828111F8CFCE0124DF812F27
:103C7000DF91CF911F910F91089587E18C83F5CF4C
:103C800086E0ECCF1F93CF93DF93EC01CCDE20E0F6
:103C900030E0A9016CE0CE01D3DE11E0882319F0F9
:103CA00010E083E08C83CE0106DF812FDF91CF917E
:103CB0001F9108951F93CF93DF93EC018F81833081
:103CC00039F089E0440F551F661F771F8A95D1F799
:103CD0009A01AB0162E1CE01B3DE11E0882319F055
:103CE00010E085E08C83CE01E6DE812FDF91CF915D
:103CF0001F9108958F929F92AF92BF92EF92FF9281
:103D00000F931F93CF93DF938C01EB017A010E94F5
:103D1000DCC14B015C012CE2820E21E0921EA11C51
:103D2000B11C0E946A82F80186838F3F69F40E9469
:103D3000DCC1681979098A099B0997FDF2CF81E1F5
:103D4000F8018483C0E021C08E3F69F5F1E0EF1AED
:103D5000F1088FEF8EBDFE012FEF0DB407FEFDCFF2
:103D60008EB581932EBDCF018C1B9D0B8E159F05AB
:103D7000A0F30DB407FEFDCF8EB5CE0DDF1D8883F9
:103D80000E946A820E946A82C1E0C80194DE8C2F80
:103D9000DF91CF911F910F91FF90EF90BF90AF9067
:103DA0009F908F9008958FE0CBCF0F931F93CF9369
:103DB000DF93EC018B0137DE40E052E0B801CE0129
:103DC00099DFDF91CF911F910F9108950F931F936A
:103DD000CF93DF93EC0189018F81833039F089E043
:103DE000440F551F661F771F8A95D1F79A01AB01C3
:103DF00061E1CE0125DE882351F084E08C83CE0181
:103E00005ADE80E0DF91CF911F910F91089540E03D
:103E100052E0B801CE016EDFF5CFB0E0A0E0E3E103
:103E2000FFE10C94B1E2EC01162F1F821C824B8340
:103E30000E94DCC16B017C0120EDC20E27E0D21E86
:103E4000E11CF11CA89561E08B810E94F4C08B817C
:103E50000E94A8A7249A2C9A279A2698259A81E04E
:103E60000E94718285E08D830E9471820AE08FEF4B
:103E70000E9465820150D9F7A89520E030E0A901A1
:103E800060E0CE01DDDD8E83813079F00E94DCC1FF
:103E90006C197D098E099F0997FDEFCF81E08C8316
:103EA000CE0109DE1A8280E065C0A8952AEA31E0D9
:103EB00040E050E068E0CE01C3DD853031F581E0BF
:103EC0008F83A8958F81812C912C5401823029F405
:103ED000812C912CA12C80E4B82E20E030E0A901A7
:103EE00067E3CE01ADDDA501940169E2CE01A8DD55
:103EF0008E838823F1F00E94DCC16C197D098E0944
:103F00009F0997FDEACF8AE0CACF04E00E946A8247
:103F10008E830150D9F78A3A11F482E0D1CF0E9402
:103F2000DCC16C197D098E099F0997FDBFCF82E026
:103F3000B6CF8F818230B9F420E030E0A9016AE386
:103F4000CE017EDD882311F088E0A9CF0E946A822D
:103F5000807C803C11F483E08F830E946A820E94FF
:103F60006A820E946A82CE01A6DD81E08A831730D0
:103F700030F41D83CDB7DEB7ECE00C94CDE288E1E0
:103F80008C8391CF0F931F93CF93DF93EC018B0121
:103F900020E030E0A90169E053DD882351F080E1A1
:103FA0008C83CE0188DD80E0DF91CF911F910F914E
:103FB000089540E150E0B801CE019CDEF5CF0C94AD
:103FC000E8C140918D0321E042276CE070E00C9441
:103FD0007CA740918D0321E0422764E070E00C94BF
:103FE0007CA740918D0321E0422761E070E00C94B2
:103FF0007CA740918D0321E0422761E070E00C94A2
:104000007CA740918D0321E0422768E070E00C948A
:104010007CA740918D0321E042276CE070E00C9476
:104020007CA741E061E070E00C947CA740918D0397
:1040300021E042270C947CA76CE070E00C9483C1D3
:1040400061E070E00C9483C16CE070E00C9483C17B
:1040500064E070E00C9483C1CF93C82FCB010E9421
:10406000C47B89E396E00E94C47B8AE296E0CC237D
:1040700011F08FE296E00E946781CF9108959091B0
:10408000B80281E089270C94A27361E08EE197E089
:104090000C942E7420E030E0A901BC0182E791E08D
:1040A0000C94B6B780E090E0A0E8B0E480937A0189
:1040B00090937B01A0937C01B0937D0187E192E016
:1040C000E9DF80E090E0A0EFB1E48093720190938B
:1040D0007301A0937401B09375018093760190935E
:1040E0007701A0937801B0937901E091E503EE0F99
:1040F000FF0BE950FE4F808191818330910539F1AA
:1041000084309105C9F1029761F480E090E0A3E466
:10411000B3E48093720190937301A0937401B09300
:1041200075018FEF91E0B6DF10927A0110927B015A
:1041300010927C0110927D0187E192E0ABDF8091CB
:10414000E5038F5F8430ECF48093E503089580E00D
:1041500090E0A3E4B3E48093720190937301A09381
:104160007401B09375018093760190937701A093C9
:104170007801B0937901D5CF80E090E0A3E4B3E477
:10418000F2CF1092E5030895B0E0A0E0EAECF0E28F
:104190000C94BBE220E24F8158856E818D810E9494
:1041A000A7BCE2E00C94D7E280911E0790911F0714
:1041B0000C941DC26AEE78E482E00C94B5BE6EEEFB
:1041C00078E481E00C94B5BE62EF78E480E00C9472
:1041D000B5BE66EF78E483E00C94B5BE1092380764
:1041E0000C9433CD4FE350E06AE874E08DED96E037
:1041F0000C941CE58091041390910513891B8F701A
:1042000011F40C94827581E00895809167018823F0
:1042100041F06091DD037091DE0341E081E00C9498
:1042200047BC0895CF93DF93EC010E94E5C91B8240
:10423000DF91CF910895CF93DF93EC01462F41702A
:104240006C857D858E859F850E94F6C6882351F0FA
:10425000888920E2829FC001112485599F4EDF91F9
:10426000CF91089590E080E0FACFCF93DF93EB01F8
:10427000FC012381211104C080E0DF91CF910895DA
:104280002250223028F48FE28883198281E0F5CF12
:1042900060E0D1DF009781F3DC0160E080E09EE226
:1042A0002D91203299F0883031F49E01260F311D76
:1042B000F90190836F5F9E01260F311DAD014150C2
:1042C0005109FA014081F90140836F5F8F5F8B30A4
:1042D00039F7FE01E60FF11D1082D8CFACE0B0E057
:1042E000E4E7F1E20C94ACE25C01DC0159968D90BC
:1042F0009C90F40181859285A385B4859C01AD01D4
:104300002F5F3F4F4F4F5F4F29873A874B875C871F
:10431000D50114964D905D906D907C901797411447
:1043200051046104710409F459C0BFEF4B1A5B0AD0
:104330006B0A7B0A312C730162011D821E821F826F
:104340001886F40181859285A385B4852D813E81EF
:104350004F815885281739074A075B0708F056C070
:1043600089859A85AB85BC858C159D05AE05BF05F5
:1043700050F482E0C82ED12CE12CF12C92E0492E91
:10438000512C612C712C9E012F5F3F4FB701A6016C
:10439000C4010E9400C98823C9F189819A81AB8137
:1043A000BC81892B8A2B8B2B01F1260137019FEFD2
:1043B000491A590A690A790A2D813E814F81588527
:1043C0002F5F3F4F4F4F5F4F2D833E834F83588763
:1043D0003FEFC31AD30AE30AF30AB3CF40805180F8
:1043E0006280738033243394A6CFC414D504E604CA
:1043F000F70411F70FEF1FEF2FEF3FE0B701A60112
:10440000C4010E9486C8782E811106C0712C872DA8
:104410002C96E1E10C94C8E2F50144815581668156
:104420007781411551056105710539F097018601C4
:10443000C4010E9486C8882349F3D5011496CD9201
:10444000DD92ED92FC921797332051F0D701C6010F
:104450000196A11DB11DF40180839183A283B383D2
:10446000F50185899689A789B08D892B8A2B8B2B9D
:1044700071F6C58AD68AE78AF08E81818068818349
:10448000C6CF40E050E0BA010C942ECA4F925F9222
:104490006F927F92AF92BF92CF92DF92EF92FF9294
:1044A0000F931F93CF93DF931F92CDB7DEB78C018D
:1044B0007B015A01C22EDB0159968D919C91F80126
:1044C000928F818FCB01DDDF712CF7018085918583
:1044D000A285B385418952896389748984179507B8
:1044E000A607B70708F052C055E0B695A79597956F
:1044F00087955A95D1F7F82FFF70DF2ED7011396C5
:104500008C91823010F480E0DAC041E050E0BE01CE
:104510006F5F7F4FC7010E9429CB0197A1F7F70179
:1045200080859185A285B3854F96A11DB11D808799
:104530009187A287B387F0E2DF9EB001112465590D
:104540007F4E61157105F9F2DB018C91882341F0F2
:10455000853E09F04BC0772029F077247394B5CFBE
:1045600071100EC080916B1290916C12A0916D121F
:10457000B0916E12F80184879587A687B787D08A95
:10458000DB018C918111E9CF772473948C2D827497
:10459000823409F0B8CF772009F4A1C0F801D0889F
:1045A00061E0C80148DE009709F4ADCF20E2DC01EC
:1045B0001D922A95E9F72BE0F501DC0101900D929F
:1045C0002A95E1F721E238E2FC01318B208B40E0B3
:1045D00058E057874687338B228B318F208F578B3C
:1045E000468B0E94ADC6811109C08DCF4BE050E0D3
:1045F000C5010E94CCE4892B09F067CFF0E2DF9E71
:10460000D00111249D0125593F4EF9018385817107
:1046100021F08C2D827109F000C1F801818D928DFD
:1046200040916B1250916C1260916D1270916E12EC
:104630004487558766877787D08AFD01E559FF4E05
:1046400044885588712C612C320155244424D801AA
:1046500055964D925D926D927C925897428D538DF6
:1046600070E060E0442955296629772955964D93D5
:104670005D936D937C935897D9011B962C9128716B
:1046800009F0BDC0848D958DA68DB78DF801818B05
:10469000928BA38BB48B81E083838C2D8F70F80178
:1046A00081831482158216821782108611861286E3
:1046B000138681E0C4FE03C0C8010E94B3CA0F90F4
:1046C000DF91CF911F910F91FF90EF90DF90CF90EE
:1046D000BF90AF907F906F905F904F900895D701FB
:1046E00013968C911397823009F40DCF51968D91CA
:1046F0009D910D90BC91A02D803E9F4FAF41B10583
:1047000008F001CFC701EADD882309F4FCCE0E943E
:10471000ADC6882309F4F7CED7015996ED91FC91E7
:104720005A9714964D905D906D907C901797B2E0DB
:104730004B1A510861087108858504C0440C551C4A
:10474000661C771C8A95D2F786859785A089B189E2
:10475000480E591E6A1E7B1E81E080936F124092A4
:104760006B1250926C1260926D1270926E12EBE6A8
:10477000F0E180E092E0DF019C011D922150304089
:10478000E1F7DD24D394D7015996ED91FC91848112
:10479000D816C0F48091701290917112DC01ED91E5
:1047A000FC910288F389E02D2BE630E1B301A201F0
:1047B0004D0D511D611D711D0995882309F4A3CE6E
:1047C000D394E1CF258580E092E0A0E0B0E004C082
:1047D000880F991FAA1FBB1F2A95D2F7F70141899D
:1047E000528963897489840F951FA61FB71F818B17
:1047F000928BA38BB48B8BE690E1D12CD7CE20315A
:1048000061F498012F5E3F4F0E947CC9882329F0F4
:1048100084E0D80113968C9340CFD80113961C9254
:1048200072CEFC0123812111FDCC0895A1E4B0E0FA
:10483000ECE1F4E20C94ABE24C015B017A01222E34
:1048400019821C821C8E1F8E6115710569F410E09F
:10485000CE014C96E6DFCE010196E3DF812FCF5BE0
:10486000DF4FE2E10C94C7E2FC0183818111EFCFBD
:10487000FA0180818F3251F18B01CE0101966C01DA
:104880002C0180E2382E360122963FAE22972196E7
:104890003FAE21973FAE3EAE3DAE3CAE3BAE3AAEF4
:1048A00039AE38AE3FAA970190E047E0D9018D912B
:1048B000882309F447C08F3209F444C08E3209F5C9
:1048C0004A3029F298E04AE09D01F0CFFB01838154
:1048D00082508230A0F0618D728DCE014C960E9484
:1048E000E4CC882309F4B3CF8E01045E1F4FC701C7
:1048F0007C010196F70120812F32D1F3BECF8B01CD
:10490000F6CFE4E8F4E12491222321F031968213DA
:10491000FACF9DCF491708F49ACF813208F497CF88
:104920008F3709F494CF3FE9380F3A3108F420EE7D
:10493000E7E3F0E0EC0FFD1FE90FF11D820F80832C
:104940009F5FC2CF8FA9803209F481CF7901F9012D
:1049500080812F5F3F4F8F32C9F38823C1F021E060
:10496000AE01495C5F4FB801C60190DD882309F4B0
:104970006ECF0A151B0511F0C80154DCCE014C9610
:104980004C145D0409F0C30186016C017DCF222D1A
:10499000AE01495C5F4FB801C40178DD182F58CFD4
:1049A0008F929F92AF92BF92CF92DF92EF92FF923F
:1049B0000F931F93CF93C82F00E812E1F801608591
:1049C0007185072E000C880B990B0E94CBDB6B01C5
:1049D0007C01F80184809580A680B78080E20E94E7
:1049E000A37B84E50E94A37B8AE30E94A37B42E031
:1049F000C501B4010E94C7A78DE794E10E94C47B62
:104A000042E0C701B6010E94C7A762E070E080E003
:104A100090E00E9450C187E1C802F0011124E058E3
:104A2000FD4E628570E080E894E10E945A81CF914A
:104A30001F910F91FF90EF90DF90CF90BF90AF90BC
:104A40009F908F9008950F930FB70F9300916E0072
:104A50000B7F00936E0078940F930BB70F930CB7F6
:104A60000F921F922F933F934F935F936F937F9378
:104A70008F939F93AF93BF93EF93FF9311240E9463
:104A80006F58FF91EF91BF91AF919F918F917F915F
:104A90006F915F914F913F912F911F900F900CBF9D
:104AA0000F910BBF0F910460F89400936E000F916B
:104AB0000FBF0F911895CF93DF9310929703C0E823
:104AC000D2E1198618860E94E8C11A865D98DF91A6
:104AD000CF910895EF92FF920F931F93CF93C82F1A
:104AE0007B018A0180911D078330E0F00E94F180F4
:104AF000C7010E94C47B83E094E10E94C47BC7FD90
:104B00000EC081E094E10E94C47B6C2FCC0F770B28
:104B1000880B990B0E947DA58AE00E94A37B8AE006
:104B20000E94A37BC8DFA89580918004811128C0D2
:104B300081E08093800482E080931D07BCDFC5E1A3
:104B4000C150149AB9F069E170E080E090E00E94F1
:104B500050C1A895149868E270E080E090E00E944F
:104B600050C1A89568E270E080E090E00E9450C1DA
:104B7000A895E6CF40E06EEF73E1C8010E949681F0
:104B8000CF911F910F91FF90EF900895CF93DF93F6
:104B9000A89580918212909183120E94F5A660934D
:104BA0008412709385128093861290938712C0911D
:104BB0008212D09183128091600190916101C81797
:104BC000D90734F44FE354E16CE474E180E082DF10
:104BD0008091881290918912181619066CF48091B0
:104BE0005E0190915F018C179D0734F44EE554E10E
:104BF0006BE674E180E06EDFDF91CF9108958F92D4
:104C00009F92AF92BF92CF92DF92EF92FF92CF939B
:104C1000DF9300D000D0CDB7DEB780911D078111A2
:104C200010C0A8950F900F900F900F90DF91CF912B
:104C3000FF90EF90DF90CF90BF90AF909F908F90BC
:104C40000895809181048111EDCF81E080938104EA
:104C500080919803811103C010928104E3CF96DF05
:104C6000109298030E94DCC16B017C010E9498A500
:104C70004B015C016091640170916501072E000C8D
:104C8000880B990B0E94CBDB9B01AC01C501B401E1
:104C90000E9446E418160CF469C060918812709165
:104CA0008912072E000C880B990B0E94CBDB6983BD
:104CB0007A838B839C83CE0101960E9427C28090C9
:104CC000841290908512A0908612B0908712609105
:104CD000620170916301072E000C880B990B0E94F2
:104CE000CBDB9B01AC01C501B4010E9446E4181660
:104CF000CCF46091640170916501072E000C880B63
:104D0000990B0E94CBDB9B01AC01C501B4010E9451
:104D1000C5DB87FF07C00E94A1A50E94C2E375956D
:104D2000679501C060E060938A1280917C12909137
:104D30007D12A0917E12B0917F120097A105B1055E
:104D400009F48ACFC81AD90AEA0AFB0AF7FC84CF09
:104D50000E9498A50E94C2E320917A1230917B12A2
:104D60006217730754F00E94E8C176CF4FE354E115
:104D70006CE474E180E0AEDE90CF41E254E160E3A8
:104D800074E180E0A7DE68CFCF92DF92EF92FF92CE
:104D9000CF93DF93EC01C880D980EA80FB8084EF59
:104DA00093E10E94C47BC701B6010E94E96FCC80E9
:104DB000DD80EE80FF8087EC9DE20E94C47BC7010E
:104DC000B6010E94E96FC884D984EA84FB8483EC2D
:104DD0009DE20E94C47BC701B6010E94E96F8AE090
:104DE0000E94A37BDF91CF91FF90EF90DF90CF9057
:104DF0000895BC01209161043091620440916104E6
:104E0000509162042417350731F481E026173707E3
:104E100009F080E008959A01F1CF0F930FB70F9337
:104E200000916E000F930B7F00936E0000916F0056
:104E30000D7F00936F000F930BB70F930CB70F927A
:104E40001F922F933F934F935F936F937F938F9313
:104E50009F93AF93BF93EF93FF931124BCD5FF9122
:104E6000EF91BF91AF919F918F917F916F915F91E2
:104E70004F913F912F911F900F900CBF0F910BBF3F
:104E80000F910260F89400936F000F9100936E00F1
:104E90000F910FBF0F91189500C000C08091D906E7
:104EA00080FF1FC0459A8FEF80931A048091D90626
:104EB00081FF1AC0479A8FEF80931B048091D90617
:104EC00082FF15C02A988FEF80931C048091D90629
:104ED00083FF10C028988FEF80931D0400C000C08E
:104EE0000895459881E0E0CF479881E0E5CF2A9A80
:104EF00081E0EACF289A81E0EFCF80918E03982F4E
:104F0000977F90938E03982F937081E011F080E04B
:104F100008955E9A08955E9880918E0388608093CC
:104F20008E030895E82FF0E021E030E0082E02C063
:104F3000220F331F0A94E2F72095309590918E034B
:104F4000922390938E03ED50FE4F2081922321E017
:104F500019F020E0822F0895813079F038F0823006
:104F6000C9F7159A90914B079B7F04C05E9A909168
:104F70004B079E7F90934B07EDCF5E9A90914B0726
:104F80009D7FF8CF80E0CEDF81E0CCDF82E0CADF1A
:104F9000B4CF813079F070F0823071F021E030E0F0
:104FA00001C0220F8A95EAF780918E03822B8093AD
:104FB0008E0308955E98F2CF1598F0CFB0E0A0E090
:104FC000E4EEF7E20C94B5E2C82F67EC7BE00E94B8
:104FD000F4B7C11102C00E94F4808FEB9BE00E94E5
:104FE000C47B8BE29BE00E9467816DEA7BE08C2FA3
:104FF0000E94F4B7C11102C00E94F48080E99BE0D6
:105000000E94C47B8C2F0E9414B88C2F0E94328087
:105010008C2F0E9459808C2F0E9412808C2F0E940E
:10502000DE7F67E47BE08C2F0E940BB8D091B80242
:105030008EE39BE00E94C47B6D2F70E090E080E0E7
:105040000E947DA54091B4025091B5026091B602D4
:105050007091B70288ED9CE20E94EF7B81E39BE0B8
:105060000E94C47B8091B8020E94E78020E030E07B
:10507000A9016091B9027091BA028091BB0290912E
:10508000BC020E94C5DB8823A1F189ECE82E82E0F6
:10509000F82E10E0670100E0C11102C00E94F48008
:1050A00086E89BE00E94C47B802F0E94C57183E844
:1050B0009BE00E94C47B812F0E94C57188ED9CE219
:1050C0000E94C47BF601608171818281938145E0F9
:1050D0000E94C7A78AE00E94A37B0F5FFCE1CF0E6E
:1050E000D11C0730C9F61F5F84E0E80EF11C1730B1
:1050F00089F668E67BE08C2F0E94F4B701EC12E0A1
:10510000D0E0C11102C00E94F4808FE59BE00E94B4
:10511000C47B8D2F0E94C571F80160817181072EBB
:10512000000C880B990B0E94CBDBAB01BC018CE51A
:105130009BE00E94EF7BF801E280F38089E59BE031
:105140000E94C47BC7010E947D758AE00E94A37BF8
:105150000C5F1F4FD13059F48C2F0E941C818C2F73
:105160000E946A81CDB7DEB7E8E00C94D1E2D1E0CD
:10517000C8CFB0E0A0E0EFEBF8E20C94B3E2CFE3ED
:10518000DDE005E617E08FE4A82E8DE0B82EC12CF7
:10519000D12C7601C39469917991899199910E945A
:1051A000C9DB288939894A895B890E942ADC0E94E7
:1051B000C7E3F80161937193819391938F01C616B0
:1051C000D706E806F90610F46B017C01AC16BD06A3
:1051D00011F76FEF7FEFCB01A70196010E94F3E17A
:1051E000209375073093760740937707509378079D
:1051F000CDB7DEB7EAE00C94CFE20F931F93CF93C5
:10520000DF9303E51DE0CEE7D7E0F801219131916E
:10521000419151918F0160E070E080E89FE30E942E
:105220005AE36993799389939993F7E0CE38DF072E
:1052300061F70E94D9B79DDFDF91CF911F910F9148
:105240000895DBCFDACFD9CFD8CF909104138091D6
:105250000513981306C08091870D9091880D892BB6
:1052600021F080E00E948282F0CF08959091041393
:1052700080910513981307C08091870D9091880D38
:10528000892B09F47FCE80E00E948282EFCFCF92FB
:10529000DF92EF92FF92CF93DF932091B802222307
:1052A00019F1EC0108960E944D716B017C0120E020
:1052B00030E0A9010E94C5DB20E030E0A90188238D
:1052C00049F0CE010E94CB71A70196010E942ADC11
:1052D0009B01AC01688579858A859B850E94E2E205
:1052E000688779878A879B87DF91CF91FF90EF90BE
:1052F000DF90CF900895CF92DF92EF92FF92CF93FD
:10530000DF932091B802222319F1EC0108960E9444
:105310004D716B017C0120E030E0A9010E94C5DBEA
:1053200020E030E0A901882349F0CE010E94CB7132
:10533000A70196010E942ADC9B01AC016885798552
:105340008A859B850E94E3E2688779878A879B87A5
:10535000DF91CF91FF90EF90DF90CF900895AEE175
:10536000B0E0E5EBF9E20C94ADE29E8F8D8F5B012E
:105370008A01FC01EA5BFF4F208131814281538128
:10538000298B3A8B4B8B5C8BCA01B9010E94C9DB1C
:105390006B017C01D5012D913D914D915C910E9455
:1053A0002ADC0E9447E32B013C01F8012081318176
:1053B00042815381C701B6010E942ADC0E9447E363
:1053C0004B015C01C301B2010E94C7E36D8B7E8B70
:1053D0008F8B988F683771058105910540F428E718
:1053E00030E040E050E02D8B3E8B4F8B588FC50155
:1053F000B4010E94C7E3698F7A8F8B8F9C8F6837C7
:1054000071058105910540F488E790E0A0E0B0E0E7
:10541000898F9A8FAB8FBC8FED8DFE8DEE5AFF4F2B
:10542000208131814281538129873A874B875C876C
:10543000CA01B9010E94CBDB2B013C016D897E8939
:105440008F89988D0E94C9DB6D837E838F839887B7
:1054500020E030E0A901C301B2010E94C5DB88232E
:1054600009F4BBC1A7019601C701B6010E942ADC5D
:105470004B015C012D813E814F815885CA01B901E4
:105480000E942ADC9B01AC01C501B4010E94E2E24A
:105490004B015C01A3019201C301B2010E94E3E24E
:1054A0009B01AC01C501B4010E945AE30E9447E38D
:1054B0000E94C7E369837A838B839C8369857A859D
:1054C0008B859C8590958095709561957F4F8F4FCA
:1054D0009F4F0E94CBDB4B015C01698D7A8D8B8DD8
:1054E0009C8D0E94C9DB69877A878B879C8720E027
:1054F00030E0A901C501B4010E94C5DB882309F48D
:1055000070C129853A854B855C85CA01B9010E9425
:105510002ADC6D877E878F87988BA7019601C7014C
:10552000B6010E942ADC9B01AC016D857E858F85CA
:1055300098890E94E2E26B017C01A5019401C501FA
:10554000B4010E94E3E29B01AC01C701B6010E94D5
:105550005AE30E94F3E3AD8DBE8D95962D913D915A
:105560004D915C9198972D873E874F87588B6901A5
:105570007A0129813A814B815C81C21AD30AE40AFB
:10558000F50A0E94C7E3C61AD70AE80AF90AF7FE25
:105590008CC02D813E814F815885CA01B9010E947E
:1055A0002ADC6B017C0120E030E0A901C301B201DB
:1055B0000E94C5DB882309F418C16D857E858F851F
:1055C00098890E94C9DB9B01AC010E94E3E2A30120
:1055D00092010E942ADC4B015C0129853A854B85AA
:1055E0005C85CA01B9010E942ADC9B01AC01C5019E
:1055F000B4010E94E3E2A70196010E94E2E24B019E
:105600005C0120E030E040E850E4C301B2010E94B8
:105610002ADC9B01AC01C501B4010E945AE30E943F
:1056200047E34B015C0120E030E0A9010E9446E421
:1056300087FF03C0812C912C5401C501B4010E9445
:10564000C7E369837A838B839C832D853E854F8551
:105650005889261737074807590720F429833A83C2
:105660004B835C8369817A818B819C810E94C9DB39
:105670004B015C01A3019201C301B2010E94E3E26C
:105680009B01AC01C501B4010E942ADCA70196016F
:105690000E94E3E20E947FE40E94C7E3698B7A8B59
:1056A0008B8B9C8BC12CD12C760169897A898B8953
:1056B0009C892D893E894F89588D621B730B840B01
:1056C000950B0E94C9DBA30192010E945AE320E0DE
:1056D00034E244EF59E40E942ADC0E94C7E34B0104
:1056E0005C0169897A898B899C89298D3A8D4B8DDA
:1056F0005C8D621B730B840B950B0E94C9DBA301AD
:1057000092010E945AE320E034E244EF59E40E94FF
:105710002ADC0E94C7E36D837E838F839887C5014F
:10572000B4010E9445182B013C016D817E818F815F
:1057300098850E94451829813A814B815C81AD8D05
:10574000BE8D99962D933D934D935C939C978901C3
:105750009A010C0D1D1D2E1D3F1DFD0105A716A74D
:1057600027A730ABE65BFF4F2D893E894F89588DC7
:105770002083318342835383D5968D929D92AD923F
:10578000BC92D8972D813E814F815885D9962D9313
:105790003D934D935C93DC973D97408251826282AA
:1057A00073823496608371838283938329893A89D3
:1057B0004B895C89D1962D933D934D935C93D497FF
:1057C0003D96298D3A8D4B8D5C8D208331834283AC
:1057D00053836E96E0E10C94C9E260E070E0CB0187
:1057E00065CE60E070E0CB01B4CE60E070E0CB014C
:1057F00016CF90916F0081E091FD02C080E0089586
:1058000090916F009D7F90936F000895EFE6F0E018
:105810008081826080830895CF93C82FEADF94E06F
:10582000C99F90011124F901EC59FB4F20593B4FBE
:10583000D9014D915D916D917C914083518362833B
:10584000738391E0909363048111E0DFCF91089519
:10585000CF93DF938091D806811105C08091DA063D
:10586000882309F44EC08091F503329B4DC08160BE
:105870008093F5038091F503339B48C08260809349
:10588000F5038091F503349B43C084608093F50356
:10589000C0915404C0FF0FC08091D90680FF0BC097
:1058A0008091F50380FF07C080914A078160809353
:1058B0004A0780E0B1DFC1FF0FC08091D90681FFA8
:1058C0000BC08091F50381FF07C080914A07826079
:1058D00080934A0781E0A0DFC2FF13C08091D90600
:1058E00082FF0FC08091DA06882359F08091F5037A
:1058F00082FF07C080914A07846080934A0782E054
:105900008BDFDF91CF9108958E7FB2CF8D7FB7CFA0
:105910008B7FBCCF6EDF1092790710927A071092BE
:105920007B0710927C07811171CF08950F931F930D
:105930008091041390910513891B8F7009F449C05D
:1059400090910113992361F0833040F48FEF890F18
:1059500029F08093011390E080E038C01092011389
:10596000809105132BE5829FC00111248257984F27
:10597000FC01208120FDEFCF4091790750917A07FB
:1059800060917B0770917C07E95AFF4F008111817C
:1059900022813381401B510B620B730B40937907BB
:1059A00050937A0760937B0770937C0720910513CF
:1059B0002F5F2F7020930213309105132091031352
:1059C000321304C020910213209303131F910F91EF
:1059D0000895A0DFC0CFA3E1B0E0E1EFFCE20C94BA
:1059E000ABE28FEF9FEF90938900809388002AE0CD
:1059F0002983312C212C789480915D0490915E0450
:105A0000A0915F04B0916004892B8A2B8B2B09F045
:105A1000C2C1809163048823D1F080916104909188
:105A2000620410926304892B91F010926204109228
:105A300061041092540490910413809105139817F7
:105A400031F0809105138F5F8F70809305138091E3
:105A5000610490916204892B09F49DC1409159041D
:105A600050915A0460915B0470915C0480915504DC
:105A700090915604A0915704B091580400914B04A2
:105A800010E030E020E0841B950BA60BB70B081745
:105A900019072A073B0710F4D901C8018A8B840F24
:105AA000951FA61FB71F8093590490935A04A09383
:105AB0005B04B0935C04E1E0C0902204D090230426
:105AC000E0902404F09025048091320490913304F6
:105AD000A0913404B0913504C80ED91EEA1EFB1EF5
:105AE000C0923204D0923304E0923404F092350430
:105AF000F7FC33C040911A04042E000C550B660BC2
:105B0000770B8091700490917104A0917204B09110
:105B10007304840F951FA61FB71F80937004909382
:105B20007104A0937204B093730480911E04909149
:105B30001F04A0912004B0912104B701A601481BC5
:105B4000590B6A0B7B0BDB01CA01809332049093E3
:105B50003304A0933404B0933504009126041091CB
:105B600027042091280430912904809136049091D3
:105B70003704A0913804B0913904080F191F2A1F67
:105B80003B1F00933604109337042093380430935E
:105B9000390437FD33C040911B04042E000C550B13
:105BA000660B770B8091740490917504A091760434
:105BB000B0917704840F951FA61FB71F80937404BC
:105BC00090937504A0937604B093770480911E049B
:105BD00090911F04A0912004B09121042801390163
:105BE000481A590A6A0A7B0AD301C2018093360413
:105BF00090933704A0933804B093390440912A0459
:105C000050912B0460912C0470912D0480913A04E2
:105C100090913B04A0913C04B0913D04480F591F62
:105C20006A1F7B1F40933A0450933B0460933C04EB
:105C300070933D0477FD33C080901C04082C000C49
:105C40009908AA08BB088091780490917904A091E2
:105C50007A04B0917B04880D991DAA1DBB1D809309
:105C6000780490937904A0937A04B0937B04809194
:105C70001E0490911F04A0912004B09121043A01C8
:105C80004B01681A790A8A0A9B0AD401C3018093DE
:105C90003A0490933B04A0933C04B0933D0480905D
:105CA0002E0490902F04A0903004B0903104809185
:105CB0003E0490913F04A0914004B0914104880DAE
:105CC000991DAA1DBB1D80933E0490933F04A09391
:105CD0004004B0934104B7FD33C040901D04042C30
:105CE000000C55086608770880907C0490907D042D
:105CF000A0907E04B0907F04840C951CA61CB71C59
:105D000080927C0490927D04A0927E04B0927F04E5
:105D100080901E0490901F04A0902004B090210455
:105D20002C013D01481859086A087B0853014201BB
:105D300080923E0490923F04A0924004B0924104AD
:105D4000E11104C0E0918400F0918500F7FE5F9AB4
:105D500037FF469A77FF2B9AB7FF299AE091840084
:105D6000F0918500E0918400F0918500F7FE5F9846
:105D700037FF469877FF2B98B7FF29985A88552008
:105D800021F080918400909185002A8921502A8BEE
:105D9000E0E0211191CE80915D0490915E04A0918C
:105DA0005F04B0916004892B8A2B8B2B09F0B0C65D
:105DB00040906104509062045B8A4A8A4114510405
:105DC00009F402C78091590490915A04A0915B0490
:105DD000B0915C0440915504509156046091570471
:105DE0007091580484179507A607B70708F449C0AF
:105DF0001092620410926104109254049091041362
:105E000080910513981709F4DFC6809105138F5F01
:105E10008F7080930513A0EDCA2EA7E0DA2EE12C37
:105E2000F12C8091610490916204892B09F068C67D
:105E30007DDD9093620480936104892B09F460C630
:105E400040906104509062045B8A4A8AD2018C912E
:105E500083FF08C5C20145960E94E41710926204B0
:105E600010926104109254049091041380910513D0
:105E70009817F1F2809105138F5F8F70809305134F
:105E8000D7CF4091500450915104609152047091C9
:105E90005304481759076A077B0708F40FC240915B
:105EA0004C0450914D0460914E0470914F04EA8966
:105EB000FB8985A996A9A7A9B0AD481759076A0714
:105EC0007B0708F0D0C1411551056105710509F046
:105ED00066C08090930390909403A0909503B09037
:105EE000960384ED93E1A1E0FC01059115912591C4
:105EF0003491081519052A053B0558F4B694A79462
:105F000097948794AA0F0496E0EFF3E1E817F90756
:105F100059F7A0934B04F0E28F169104A104B10449
:105F200028F4E0E28E2E912CA12CB12C20E2821AD2
:105F30009108A108B108811438E09306A104B104C6
:105F400008F49AC1A4E09A9EC00111248C52904F8B
:105F5000FC01329625913491B82DEE27B39F800134
:105F6000B29F010D1E1F06940E1F1E1F112430E04C
:105F700020E0FC01C590D490F12CE12CC01AD10A8C
:105F8000E20AF30A4C0D5D1D6E1D7F1D40934C040B
:105F900050934D0460934E0470934F0442CF10E031
:105FA0000A81942F852E862FBC81AD81FE81EF81E1
:105FB000388529854B80E0918F03E99FA12DFF272C
:105FC00030919003399FA00DF11D10909103199EFF
:105FD000F00DE89DA00DF11D389DF00DE89FF00D2E
:105FE0004A2EBF2F4A9EE12D332722274F9EE00DD8
:105FF000311D211FBA9FE00D311D211FBF9F300DA4
:10600000211D432EB22F4A9E012D332722274F9E5A
:10601000000D311D211FBA9F000D311D211FBF9F93
:10602000300D211D432EB22FEE27909193038090C7
:1060300094038091950300909104012A09F483C090
:1060400030918D04349DE119910B810A810B2091CF
:106050008E04249DE0199109810A810B00918F041F
:10606000049D90198108810B3B9FE0199109810AD9
:10607000810B2B9F90198108810B0B9F8018810940
:106080004A9E012D332722274F9E000D311D211FCF
:10609000BA9F000D311D211FBF9F300D211D432EC2
:1060A000B22F30918904349DE10D911F811E811F13
:1060B00020918A04249DE00D911D811E811F009175
:1060C0008B04049D900D811C811F3B9FE00D911D51
:1060D000811E811F2B9F900D811C811F0B9F800CA7
:1060E000811D4A9E012D332722274F9E000D311D11
:1060F000211FBA9F000D311D211FBF9F300D211D93
:10610000432EB22F30918504349DE119910B810A01
:10611000810B20918604249DE0199109810A810B4D
:1061200000918704049D90198108810B3B9FE01921
:106130009109810A810B2B9F90198108810B0B9F7C
:106140008018810982C030918D04349DE10D911F2A
:10615000811E811F20918E04249DE00D911D811EC2
:10616000811F00918F04049D900D811C811F3B9F16
:10617000E00D911D811E811F2B9F900D811C811FA1
:106180000B9F800C811D4A9E012D332722274F9E95
:10619000000D311D211FBA9F000D311D211FBF9F12
:1061A000300D211D432EB22F30918904349DE11909
:1061B000910B810A810B20918A04249DE019910999
:1061C000810A810B00918B04049D90198108810B39
:1061D0003B9FE0199109810A810B2B9F901981083F
:1061E000810B0B9F801881094A9E012D332722279E
:1061F0004F9E000D311D211FBA9F000D311D211F23
:10620000BF9F300D211D432EB22F30918504349D48
:10621000E10D911F811E811F20918604249DE00DB8
:10622000911D811E811F00918704049D900D811C8A
:10623000811F3B9FE00D911D811E811F2B9F900DA3
:10624000811C811F0B9F800C811D11244B820A83AE
:10625000BC83AD83FE83EF8338872987982C892EF2
:10626000B12CA82E3ECEAA89BB89D1968D909D9047
:10627000AD90BC90D49735CED501C401B695A79505
:10628000979587958C7F8C52944FFC01C590D49044
:10629000FC01329625913491E82DE7708E2EE29F15
:1062A000C001E39F900D112433E0969587953A95B0
:1062B000E1F7C81AD90AF12CE12C64CE40914704C9
:1062C000509148046091490470914A044817590755
:1062D0006A077B0708F030C2809042049090430424
:1062E000A0904404B090450480914604EA89FB895B
:1062F00081117CC0EF5BFF4FE080F1800281138150
:10630000EA89FB89E25BFF4F208131814281538121
:10631000AA89BB89D1966D917D918D919C91D497DD
:106320000E94ED17B1E0B0934604EA89FB8941A9C8
:1063300052A963A974A984ED93E1A1E0FC01059140
:10634000159125913491041715072607370758F43E
:106350007695679557954795AA0F0496E0EFF3E178
:10636000E817F90759F7A0934B044032510561052E
:10637000710520F440E250E060E070E040525109C5
:10638000610971094115F8E05F076105710508F4BD
:10639000B3C124E0529FC00111248C52904FFC01E4
:1063A000329625913491AA27439FF001429FE10D37
:1063B000FA1F0694EA1FFA1F1124AF0170E060E093
:1063C000FC01C590D490F12CE12CC41AD50AE60A40
:1063D000F70A8C0C9D1CAE1CBF1C8092420490924C
:1063E0004304A0924404B09245041BCD81AD92AD0C
:1063F000A3ADB4AD88169906AA06BB0608F072C113
:1064000081149104A104B10449F440919303509183
:10641000940360919503709196038DCFA0E0BA85A7
:10642000982D492D8A2DFB85EC857D856E855F85B0
:106430003889298950918F03599F712D6627309192
:106440009003399F700D611D10909103199E600D8E
:10645000549F700D611D349F600D589F600DF72F84
:10646000E62FF79F512D33272227F69F500D311D20
:106470002A1FE79F500D311D2A1FE69F300D211D59
:10648000F32FE22FF79FB12D33272227F69FB00D70
:10649000311D2A1FE79FB00D311D2A1FE69F300DC9
:1064A000211DF32FE22F55279091930340919403E0
:1064B00080919503009091040A2A09F483C03091D9
:1064C0008D043F9F51199A0B4A0B8A0B20918E0421
:1064D0002F9F501991094A0B8A0BB0918F04BF9FCF
:1064E000901941098A0B3E9F501991094A0B8A0B5A
:1064F0002E9F901941098A0BBE9F40198109F79F71
:10650000B12D33272227F69FB00D311D2A1FE79F9B
:10651000B00D311D2A1FE69F300D211DF32FE22FF4
:10652000309189043F9F510D9A1F4A1F8A1F209165
:106530008A042F9F500D911D4A1F8A1FB0918B0412
:10654000BF9F900D411D8A1F3E9F500D911D4A1FF8
:106550008A1F2E9F900D411D8A1FBE9F400D811DD9
:10656000F79FB12D33272227F69FB00D311D2A1F2B
:10657000E79FB00D311D2A1FE69F300D211DF32F1F
:10658000E22F309185043F9F51199A0B4A0B8A0BD9
:10659000209186042F9F501991094A0B8A0BB091C4
:1065A0008704BF9F901941098A0B3E9F501991099A
:1065B0004A0B8A0B2E9F901941098A0BBE9F4019E6
:1065C000810982C030918D043F9F510D9A1F4A1F4F
:1065D0008A1F20918E042F9F500D911D4A1F8A1FE4
:1065E000B0918F04BF9F900D411D8A1F3E9F500D9B
:1065F000911D4A1F8A1F2E9F900D411D8A1FBE9F0D
:10660000400D811DF79FB12D33272227F69FB00D36
:10661000311D2A1FE79FB00D311D2A1FE69F300D47
:10662000211DF32FE22F309189043F9F51199A0BBE
:106630004A0B8A0B20918A042F9F501991094A0B0B
:106640008A0BB0918B04BF9F901941098A0B3E9F22
:10665000501991094A0B8A0B2E9F901941098A0BF8
:10666000BE9F40198109F79FB12D33272227F69F3E
:10667000B00D311D2A1FE79FB00D311D2A1FE69F67
:10668000300D211DF32FE22F309185043F9F510DD6
:106690009A1F4A1F8A1F209186042F9F500D911D1B
:1066A0004A1F8A1FB0918704BF9F900D411D8A1F0A
:1066B0003E9F500D911D4A1F8A1F2E9F900D411D18
:1066C0008A1FBE9F400D811D1124BA87FB87EC876E
:1066D0007D876E875F87388B298B542F492F70E019
:1066E000682F29CE2A893B89225B3F4FD9014D91E2
:1066F0005D916D917C911FCEDB01CA01B695A79586
:10670000979587958C7F8C52944FFC01C590D490BF
:10671000FC013296259134914770429FC001439FFE
:10672000900D1124A3E096958795AA95E1F7C81AD4
:10673000D90AF12CE12C4DCE80912E0190912F01A0
:10674000A0913001B0913101B7FF61C0EA89FB89A6
:10675000EA5BFF4FC080D180E280F38084ED93E15B
:1067600021E0FC0145915591659174914C155D05B1
:106770006E057F0558F4F694E794D794C794220FDA
:10678000049640EF53E14817590759F720934B04FB
:1067900050E2C516D104E104F10428F470E2C72EDA
:1067A000D12CE12CF12C60E2C61AD108E108F108E5
:1067B000C11478E0D706E104F10408F431C0A4E084
:1067C000DA9EC00111248C52904FFC013296259123
:1067D0003491BC2D6627B39FA001B29F410D561F77
:1067E0000694461F561F112470E060E0FC0185915D
:1067F0009491B0E0A0E0841B950BA60BB70B80939F
:106800002E0190932F01A0933001B0933101C090DD
:106810002E01D0902F01E0903001F090310101CB9A
:10682000D701C601B695A795979587958C7F8C5211
:10683000944FFC0125913491FC013296459154917D
:10684000EC2DE770E49FC001E59F900D112463E0FB
:10685000969587956A95E1F7281B390BC901B0E039
:10686000A0E0CDCFEA89FB8985889688A788B08C7F
:1068700081E081149104A104B10409F480E0AA89A3
:10688000BB895996CD90DD90ED90FC905C97C1143A
:10689000D104E104F10409F08260EA89FB89458DA5
:1068A000568D678D70A1411551056105710509F07F
:1068B0008460809354041092420410924304109216
:1068C00044041092450410924C0410924D0410920E
:1068D0004E0410924F04EA89FB8985A196A1A7A1D5
:1068E000B0A58093550490935604A0935704B09399
:1068F0005804442455243201481A590A6A0A7B0A6A
:106900004092320450923304609234047092350401
:1069100040923604509237046092380470923904E1
:1069200040923A0450923B0460923C0470923D04C1
:1069300041A052A063A074A0440C551C661C771C97
:10694000880C991CAA1CBB1C8092220490922304E0
:10695000A0922404B0922504CC0CDD1CEE1CFF1C7C
:10696000C0922604D0922704E0922804F0922904D1
:10697000440F551F661F771F40932A0450932B0422
:1069800060932C0470932D0440922E0450922F0497
:106990006092300470923104880F991FAA1FBB1FA8
:1069A00080931E0490931F04A0932004B0932104AD
:1069B0001092590410925A0410925B0410925C04D5
:1069C00081A592A5A3A5B4A58093500490935104EA
:1069D000A0935204B093530485A596A5A7A5B0A98A
:1069E0008093470490934804A0934904B0934A04C9
:1069F000EB5BFF4F80819091D906891721F080933E
:106A0000D9060E944C270E94282C44244A94542CD6
:106A1000320140922E0150922F016092300170920B
:106A20003101EA89FB89FD96E080F18002811381C2
:106A3000AA89BB89D1962D913D914D915C91D497B6
:106A40006D01BAE4CB0ED11CF601608171818281A7
:106A500093810E94ED1710924604D6014D915D91ED
:106A60006D917C9184ED93E1A1E0FC01059115917C
:106A700025913491041715072607370758F47695A2
:106A8000679557954795AA0F0496E0EFF3E1E8174D
:106A9000F90759F7A0934B04403251056105710580
:106AA00020F440E250E060E070E04052510961099A
:106AB00071094115F8E05F076105710508F462C0CE
:106AC00024E0529FC00111248C52904FFC01329659
:106AD00025913491AA27439FF001429FE10DFA1FAF
:106AE0000694EA1FFA1F1124AF0170E060E0FC0178
:106AF000C590D490F12CE12CC41AD50AE60AF70A05
:106B0000C0925D04D0925E04E0925F04F092600453
:106B100080915D0490915E04A0915F04B091600447
:106B2000AC01BD01009731E0A307B10520F04FEFA4
:106B30005FEF60E070E0841B950BA60BB70B8093B2
:106B40005D0490935E04A0935F04B0936004F89496
:106B500080918400909185004096A981A150A983DD
:106B6000AA2381F1240E351E2816390610F40C9440
:106B7000FB2C309289002092880078946396E2E1A1
:106B80000C94C7E2DB01CA01B695A7959795879546
:106B90008C7F8C52944FFC01C590D490FC013296AE
:106BA000259134914770429FC001439F900D11245D
:106BB00033E0969587953A95E1F7C81AD90AF12CF2
:106BC000E12C9ECF1C01D5CF80EDC82E87E0D82EBA
:106BD000E12CF12C2DC9CF93DF9380910413909178
:106BE0000513891B80958F7019F40E948282F5CF5E
:106BF000809104138F5F8F70A09104139BE5A99F70
:106C0000D0011124FD01E257F84FEF0119929A9536
:106C1000E9F798E09083AD55B84F90E1E6E0F3E1F5
:106C200001900D929A95E1F720910413909105132C
:106C3000291303C094E690930113809304130E94D8
:106C4000062CDF91CF910895FC0120813181428192
:106C5000538160915F0D7091600D8091610D9091F5
:106C6000620D0E942ADC0E944BE460931213709321
:106C70001313809314139093151390910413809120
:106C80000513981709F0A7CF0E9425290E94F92B18
:106C900040911213509113136091141370911513B6
:106CA00040937C0450937D0460937E0470937F0432
:106CB00081110C94062C08954F925F926F927F92EF
:106CC0008F929F92AF92BF92CF92DF92EF92FF92FC
:106CD000CF93DF93EC0120915F0D3091600D4091D7
:106CE000610D5091620D6C857D858E859F850E941A
:106CF0002ADC0E944BE46B017C0120915B0D3091FA
:106D00005C0D40915D0D50915E0D688579858A8599
:106D10009B850E942ADC0E944BE44B015C01209180
:106D2000570D3091580D4091590D50915A0D6C816D
:106D30007D818E819F810E942ADC0E944BE42B0181
:106D40003C012091530D3091540D4091550D5091BF
:106D5000560D688179818A819B810E942ADC0E947C
:106D60004BE460930613709307138093081390937A
:106D7000091340920A1350920B1360920C137092F5
:106D80000D1380920E1390920F13A0921013B092D5
:106D90001113C0921213D0921313E0921413F092B5
:106DA00015139091041380910513981781F013DF48
:106DB000DF91CF91FF90EF90DF90CF90BF90AF9099
:106DC0009F908F907F906F905F904F9008950E945A
:106DD00025290E94F92BC82F86E093E10E94E41731
:106DE000CC2331F30E94062CE3CFCF92DF92EF92B7
:106DF000FF92CF93DF93C82F0E94F92B94E0C99F95
:106E0000E0011124FE01E059FB4FC080D180E280F7
:106E1000F38081110E94062CC258D84FC701B601D9
:106E20000E94CBDB288139814A815B810E942ADC68
:106E3000DF91CF91FF90EF90DF90CF900895CF92A8
:106E4000DF92EF92FF92CF93DF93C82F0E94F92B2E
:106E500094E0C99FE0011124FE01EC59FB4FC08072
:106E6000D180E280F38081110E94062CC258D84F55
:106E7000C701B6010E94CBDB288139814A815B8141
:106E80000E942ADCDF91CF91FF90EF90DF90CF90AE
:106E90000895A1E0B0E0EFE4F7E30C94BBE289834E
:106EA00060E0CE0101960E943F1961E0CE0101969B
:106EB0000E943F1962E0CE0101960E943F1989812C
:106EC0002196E2E00C94D7E2A2E1B0E0EAE6F7E333
:106ED0000C94B7E2DEDF8823C1F1EDB6FEB64AE8D6
:106EE00052E082FF02C041E852E02AE832E081FF2E
:106EF00002C023E832E080FD25C08AE892E05F937B
:106F00004F933F932F939F938F9382EA96E09F93A3
:106F10008F938E010F5F1F4F1F930F930E945EDBB5
:106F20000E94F480C8010E94B57BC8010E9422B76C
:106F30000FB6F894DEBF0FBECDBF81E06296E6E0EB
:106F40000C94D3E285E892E0DACF80E0F7CFA0E2BC
:106F5000B0E0EDEAF7E30C94ABE2809112018823F4
:106F600009F4BEC080910804082F10E080FF3CC0E7
:106F7000C0901401D0901501E0901601F090170117
:106F800020919C0230919D0240919E0250919F025F
:106F9000C701B6010E9446E4181644F4C0929C0250
:106FA000D0929D02E0929E02F0929F02C09020013A
:106FB000D0902101E0902201F090230120919C02C9
:106FC00030919D0240919E0250919F02C701B601EF
:106FD0000E94C5DB87FF08C0C0929C02D0929D0230
:106FE000E0929E02F0929F0201FF3CC0C090180107
:106FF000D0901901E0901A01F0901B012091A0029D
:107000003091A1024091A2025091A302C701B601A2
:107010000E9446E4181644F4C092A002D092A10245
:10702000E092A202F092A302C0902401D090250128
:10703000E0902601F09027012091A0023091A1025A
:107040004091A2025091A302C701B6010E94C5DB84
:1070500087FF08C0C092A002D092A102E092A202D3
:10706000F092A30202FF3CC0C0901C01D0901D0111
:10707000E0901E01F0901F012091A4023091A50222
:107080004091A6025091A702C701B6010E9446E4B2
:10709000181644F4C092A402D092A502E092A6026F
:1070A000F092A702C0902801D0902901E0902A0117
:1070B000F0902B012091A4023091A5024091A602EC
:1070C0005091A702C701B6010E94C5DB87FF08C027
:1070D000C092A402D092A502E092A602F092A7026A
:1070E00080913E0D83FD61C020917E0130917F0132
:1070F00040918001509181016091A8027091A90294
:107100008091AA029091AB020E94C5DB882309F40A
:107110004CC00E9475A8182F882331F00E94F4807B
:1071200087E896E00E94C47B20917E0130917F0128
:1071300040918001509181016091A8027091A90253
:107140008091AA029091AB020E94E2E29F77209187
:107150006C0130916D0140916E0150916F010E9460
:107160002ADC20E030E046E154E40E9446E41816B0
:10717000D4F40E94F48088E696E00E94C47B80915B
:10718000A8029091A902A091AA02B091AB028093AB
:107190007E0190937F01A0938001B093810188EAE2
:1071A00092E052DD02C01111EACF2AE037ED43E24E
:1071B0005CE360910C0170910D0180910E01909142
:1071C0000F010E942ADC6B017C016091100170911B
:1071D0001101072E000C880B990B0E94CBDB9B0141
:1071E000AC01C701B6010E942ADC698B7A8B8B8BBC
:1071F0009C8B8091B802882309F18090B402909012
:10720000B502A090B602B090B702C090A402D09090
:10721000A502E090A602F090A70220E030E0A901CC
:10722000C501B4010E94C5DB8823F9F0A7019601CE
:10723000C501B4010E9446E41816BCF020E030E01D
:10724000A901BE016F5E7F4F8CE992E00E94B6B744
:1072500080E1ECE9F2E0A2E7B1E001900D928A95BD
:10726000E1F7A096E2E10C94C7E22091720130911F
:107270007301409174015091750160919C0270916D
:107280009D0280919E0290919F020E94E2E24B013A
:107290005C01209176013091770140917801509105
:1072A00079016091A0027091A1028091A202909157
:1072B000A3020E94E2E26D8B7E8B8F8B988F2091D0
:1072C0007A0130917B0140917C0150917D01C70191
:1072D000B6010E94E2E26D8F7E8F8F8F98A320917E
:1072E0007E0130917F014091800150918101609138
:1072F000A8027091A9028091AA029091AB020E940B
:10730000E2E2698F7A8F8B8F9C8F20E030E0A901B9
:10731000C501B4010E94C5DB81110CC020E030E042
:10732000A9016D897E898F89988D0E94C5DB88238C
:1073300009F484CFA5019401C501B4010E942ADC9F
:107340006B017C012D893E894F89588DCA01B90195
:107350000E942ADC9B01AC01C701B6010E94E3E256
:107360006B017C012D8D3E8D4F8D58A1CA01B90155
:107370000E942ADC9B01AC01C701B6010E94E3E236
:107380006B017C01298D3A8D4B8D5C8DCA01B90151
:107390000E942ADC9B01AC01C701B6010E94E3E216
:1073A0006B017C010E947FE42B013C012CEC3CEB47
:1073B0004CE85BE2C701B6010E94C5DB87FF06C04F
:1073C000498C5A8C6B8C7C8CE89477F82DEB37E3E6
:1073D00046E855E3C301B2010E94C5DB87FD38CF03
:1073E0002DEC3CEC4CE45EE3C301B2010E942ADCCC
:1073F0000E94C7E31B01672B19F422242394312C2C
:10740000B10190E080E00E94C9DB9B01AC0160E02B
:1074100070E080E89FE30E945AE36B017C01AC01BD
:107420009B01C301B2010E942ADC2B013C01A70190
:107430009601C501B4010E942ADC4B015C01A70141
:1074400096016D897E898F89988D0E942ADC6D8BCB
:107450007E8B8F8B988FA70196016D8D7E8D8F8D82
:1074600098A10E942ADC6D8F7E8F8F8F98A3A70131
:107470009601698D7A8D8B8D9C8D0E942ADC698F97
:107480007A8F8B8F9C8F80E1E2E7F1E08E010F5FB6
:107490001F4FD80101900D928A95E1F70E94DCC13F
:1074A0006B017C0128ECC20ED11CE11CF11C81E0B7
:1074B000281A310809F454C00E94DCC19B01AC01B8
:1074C0002C193D094E095F0957FD4DC06B017C0128
:1074D00028ECC20ED11CE11CF11C80E00E948282CB
:1074E000A501940169817A818B819C810E94E3E2EC
:1074F00069837A838B839C832D893E894F89588D3C
:107500006D817E818F8198850E94E3E26D837E8309
:107510008F8398872D8D3E8D4F8D58A169857A85F3
:107520008B859C850E94E3E269877A878B879C879D
:10753000298D3A8D4B8D5C8D6D857E858F859889E3
:107540000E94E3E26D877E878F87988BA30192016B
:10755000BE016F5E7F4FC8010E94B6B78111A7CFF1
:10756000A30192016ECE0E94FF25BACF8091040440
:1075700090910504A0910604B091070480930C013A
:1075800090930D01A0930E01B0930F01809102041E
:1075900090910304909311018093100108958091BC
:1075A0000C0190910D01A0910E01B0910F018093FB
:1075B000040490930504A0930604B09307048091FB
:1075C000100190911101909303048093020484E6CA
:1075D00090E090931101809310010895ACE0B0E029
:1075E000E4EFFAE30C94ADE22B013C0129873A87E2
:1075F0004B875C8747015801D601CD90DD90ED9017
:10760000FC9020E030E0A901C701B6010E94C5DB73
:10761000811171C08091680190916901A0916A0106
:10762000B0916B0189839A83AB83BC8320E030E007
:10763000A901C701B6010E94C5DB811106C0C12C9A
:10764000D12C80E8E82E80E4F82ECD82DE82EF8215
:10765000F886A501940160917A0170917B01809177
:107660007C0190917D010E94C5DB87FF0CC0809258
:107670007A0190927B01A0927C01B0927D01CE01B3
:1076800005960E944A2040927201509273016092C6
:1076900074017092750189859A85AB85BC8580934C
:1076A000760190937701A0937801B0937901CE0190
:1076B00001960E944A20A501940160917A0170917F
:1076C0007B0180917C0190917D010E9446E4181617
:1076D00064F480927A0190927B01A0927C01B09236
:1076E0007D01CE0105960E944A200E9425292C96F4
:1076F000E0E10C94C9E2D701C60194CFCF92DF92AA
:10770000EF92FF920F931F936B01FC01E080F180D9
:1077100002811381E2E7F1E02481358146815781BE
:10772000608171818281938159DF1F910F91FF9058
:10773000EF90DF90CF9008958F929F92AF92BF927B
:10774000CF92DF92EF92FF921F93CF93DF93CDB74B
:10775000DEB760970FB6F894DEBF0FBECDBF182F0F
:1077600080E043DB4B015C018092F6039092F703CB
:10777000A092F803B092F90381E037DB6B017C0142
:10778000C092FA03D092FB03E092FC03F092FD0357
:1077900082E02BDB6093FE037093FF038093000471
:1077A000909301041D861E861F86188A89829A82FC
:1077B000AB82BC82CD82DE82EF82F88669877A87CF
:1077C0008B879C8783E011DB6D877E878F87988B03
:1077D000CE0101960E9447291E3FD9F480E1FE01A7
:1077E0003196A2E7B1E001900D928A95E1F760969B
:1077F0000FB6F894DEBF0FBECDBFDF91CF911F91C2
:10780000FF90EF90DF90CF90BF90AF909F908F90C0
:10781000089584E0189FF0011124DF01AE58BE4F97
:1078200081E090E08C0F9D1FE80FF91F408151818E
:10783000628173814D935D936D937C931397D7CF42
:107840000C94D9B7CF930E94F92BC82F80910513C0
:1078500080930413809303138093021384E6809330
:1078600001130E948A2C80ED93E09093880D809301
:10787000870DC1110E94062C81E0809363040E9451
:1078800025298EEF59DFDCDFCF910895ACE0B0E021
:10789000ECE4FCE30C94BBE20E9434A80E94F92BB8
:1078A0009CE0E0E7F4E0DE01119601900D929A95DC
:1078B000E1F781110E94062CCE0101960E94C42698
:1078C0002C96E2E00C94D7E2B0E0A0E0EAE6FCE31C
:1078D0000C94ADE24090720150907301609074017D
:1078E000709075018090760190907701A09078015A
:1078F000B0907901C0907A01D0907B01E0907C013A
:10790000F0907D010E94B92860912C0170912D01A9
:10791000072E000C880B990B0E94CBDB2AE037ED79
:1079200043E25CE30E942ADC60936C0170936D017A
:1079300080936E0190936F0104E111E0D0E0C0E00C
:10794000CE018F51964F0E944771F8016193719358
:10795000819391938F01CE018B52964F0E94477174
:10796000F80160877187828793872496CC30D10590
:1079700039F760E086E194E00E942E740E94FB7467
:107980000E94FD28A3019201609172017091730120
:1079900080917401909175010E94C5DB81111BC01B
:1079A000A501940160917601709177018091780131
:1079B000909179010E94C5DB81110DC020917A015F
:1079C00030917B0140917C0150917D01C701B6014E
:1079D0000E94C5DB81115ADFCDB7DEB7E0E10C9420
:1079E000C9E28EE496E00E94C47B86B168E476E04A
:1079F00082FB882780F90E942C2086B162E476E021
:107A000083FB882780F90E942C2086B16CE376E006
:107A1000829581700C942C208091D806811103C02E
:107A20008091DA0681110C94282C0895ACE0B0E026
:107A3000ECE1FDE30C94BBE2AFE3BDE090E080E05D
:107A4000FC01E55EF44F45915591659174914D931C
:107A50005D936D937D93FC01E55FF44F45915591E6
:107A60006591749150964D935D936D937C9353976C
:107A7000FC01E550F54F45915591659174919096B3
:107A80004D935D936D937C9393970496803191050C
:107A9000B9F680E29EE4A0E0B0E080934F0D9093B1
:107AA000500DA093510DB093520D80E090E0AAEFDD
:107AB000B3E48093730D9093740DA093750DB09300
:107AC000760D8093770D9093780DA093790DB093F8
:107AD0007A0D80937B0D90937C0DA0937D0DB093D8
:107AE0007E0D10927F0D1092800D1092810D1092DC
:107AF000820D1092830D1092840D1092850D1092BC
:107B0000860D8AE097EDA3EABDE380936107909329
:107B10006207A0936307B093640780E090E0A0E25F
:107B2000B1E48093160490931704A0931804B093C3
:107B300019040E94E4738CE0E2E8F1E0DE011196A2
:107B400001900D928A95E1F789819A81AB81BC8180
:107B50008093F3129093F412A093F512B093F6125F
:107B60008D819E81AF81B8858093F7129093F81232
:107B7000A093F912B093FA1289859A85AB85BC85DA
:107B80008093FB129093FC12A093FD12B093FE120F
:107B90008EEB90E09093C2028093C1021092C402D7
:107BA0001092C30286EE90E09093C6028093C502C5
:107BB0001092C8021092C7028FE892ECADE8B1E4CF
:107BC00080938B1290938C12A0938D12B0938E128F
:107BD0008CE998EFA5E4BEE380938F129093901206
:107BE000A0939112B093921281E49CEBABECB3E4BE
:107BF0008093931290939412A0939512B09396123F
:107C00001092D8061092D70607DF5EDE0E94F4803D
:107C100088ED9AE00E94C47B2C96E2E00C94D7E2B7
:107C200080914A07882319F010924A07089540E08E
:107C300070E060E08CE196E00E9496811F920F92C6
:107C40000FB60F9211240BB60F922F933F934F93C1
:107C50005F936F937F938F939F93AF93BF93EF93B4
:107C6000FF930E94282CFF91EF91BF91AF919F91BC
:107C70008F917F916F915F914F913F912F910F90D5
:107C80000BBE0F900FBE0F901F9018950F931F9370
:107C900080915B07813019F50E94DCC10091ED03F2
:107CA0001091EE032091EF033091F003601B710BF4
:107CB000820B930B28EE33E040E050E00E94F3E1AA
:107CC0006091E9037091EA038091EB039091EC03DA
:107CD000620F731F841F951F1F910F91089560916C
:107CE000F1037091F2038091F3039091F403D6CFE6
:107CF00010925B071092ED031092EE031092EF03C7
:107D00001092F0031092F1031092F2031092F30319
:107D10001092F4031092E9031092EA031092EB031D
:107D20001092EC03089580915B078130E1F082307E
:107D3000C1F4ACDF6093E9037093EA038093EB0333
:107D40009093EC0381E080935B070E94DCC1609319
:107D5000ED037093EE038093EF039093F00381E0C3
:107D60000895C6DFEFCF80E008950E9454B80E94C6
:107D70009575882351F08091821482FD06C087EEAC
:107D800091E09093DC068093DB06CDCF80915B077A
:107D9000813079F482E080935B070E94DCC16093BC
:107DA000F1037093F2038093F3039093F40381E063
:107DB000089580E0089580915B078150823070F4CF
:107DC00010925B070E94DCC16093F1037093F20391
:107DD0008093F3039093F40381E0089580E0089585
:107DE0009C0197FF26C0EE27FF27E81BF90B2D39D2
:107DF0008FEF38070CF05DC08DE280939702CF01C2
:107E000064E670E00E945BE2CB012AE030E0B90159
:107E10000E945BE2805D80939802CF01B9010E94CD
:107E20005BE2CB01B9010E945BE2805D8093990225
:107E30002AC0283E83E03807B4F1C90168EE73E038
:107E40000E945BE2CB01EAE0F0E0BF010E945BE24E
:107E5000805D80939702C90164E670E00E945BE256
:107E6000CB01BF010E945BE2805D80939802C90153
:107E7000BF010E945BE2CB01BF010E945BE2805D1B
:107E800080939902F901CF016AE070E00E945BE201
:107E9000805D80939A0287E992E008958DE237FD34
:107EA000C5CF80E2C3CFF90180E2243631050CF062
:107EB000A4CF80E28093970280939802EA30F10584
:107EC0006CF38DE237FF80E280939802CF016AE085
:107ED00070E00E945BE2605D60939902D4CF9C01E8
:107EE00097FD2DC080E2243631055CF0C90164E6BF
:107EF00070E00E945BE2CB016AE070E00E945BE20E
:107F0000805D8093980280E22A3031055CF0EAE0DF
:107F1000F0E0C901BF010E945BE2CB01BF010E94FA
:107F20005BE2805D80939902C9016AE070E00E9483
:107F30005BE2805D80939A0288E992E00895319532
:107F4000219531098DE2DDCFCF92DF92EF92FF9242
:107F5000FC01C080D180E280F38020E030E0A90104
:107F6000C701B6010E94C5DB87FD26C06DEB77E334
:107F700086E095E3A70196010E94E3E26B017C0194
:107F800020E030E0A9010E94C5DB20E030E040E0C5
:107F90005FE387FF04C020E030E040E05FEBC70113
:107FA000B6010E94E3E20E94C2E3CB0198DFFF909A
:107FB000EF90DF90CF9008956DEB77E386E095EB3F
:107FC000D9CFA4E0B0E0E7EEFFE30C94BBE20E945F
:107FD000CBDB69837A838B839C83CE010196B4DFEC
:107FE0002496E2E00C94D7E2FC01608171818281E9
:107FF00093810E94C2E3CB0172CFA4E0B0E0E3E042
:10800000F0E40C94BBE20E94CBDB69837A838B8320
:108010009C83CE010196E8DF2496E2E00C94D7E23F
:108020000F931F930E94DCC10091D3061091D406D8
:108030002091D5063091D60601151105210531058F
:10804000D9F5209118132223A1F1E09116132150A4
:108050002093181321E02E0F20931613309119133B
:10806000231302C01092161324E0E29FF0011124A2
:10807000E65EFC4E00811181228133810093CF06A0
:108080001093D0062093D1063093D206600F711F53
:10809000811D911D6093D3067093D4068093D506FD
:1080A0009093D6068091D1069091D206892B09F043
:1080B000149A1F910F910895601B710B820B930B03
:1080C00097FDF7CF14981092D3061092D406109211
:1080D000D5061092D606EDCF0F931F93CF93DF9363
:1080E0008C01EB019091181320911913921304C085
:1080F00097DF0E94FF25F6CF8091171334E0839F0E
:10810000F0011124E65EFC4E11830083D383C28309
:108110009F5F909318138F5F281739F08093171380
:10812000DF91CF911F910F91089510921713F8CFFF
:10813000882351F063E972E084E690E0CDDF6AEBDA
:1081400072E084E690E0C8CF68EB71E084E190E0F3
:10815000FACF6CDC81E0ECCF8F929F92AF92BF920E
:10816000EF92FF920F931F93CF93DF93EC018B015C
:10817000E42EF22E80912A1390912B138C179D07D9
:10818000C9F125E5C03CD20709F03FC0835A9547A5
:1081900071F40E94DCC16E517B4F8F4F9F4F6093F3
:1081A000D9037093DA038093DB039093DC03D093BD
:1081B0002B13C0932A1330E020E000933D07109367
:1081C0003E0720933F0730934007E0923807F09234
:1081D0003907C35AD54721F4109293021092D8035D
:1081E00082E08093670181E080933A0710929202C7
:1081F0001092E403DF91CF911F910F91FF90EF90C8
:10820000BF90AF909F908F90089525E7C33AD20713
:1082100071F6805C9545D9F40E94DCC18090D90349
:108220009090DA03A090DB03B090DC036819790921
:108230008A099B0997FF0BC080914B078770873095
:1082400031F40E94FA20CFEADCE48111B0CFC3EA16
:10825000D5E7ADCF20E040E070E060E089EE90E24D
:108260007BCF0E9475A8882339F020E040E070E0C1
:1082700060E081ED9BE470CFEDCF21E0209393028D
:10828000FC0180819181A281B38180930801909348
:108290000901A0930A01B0930B0120E040E070E0D7
:1082A00060E0809127079091280756CFA4E0B0E0C6
:1082B000ECE5F1E40C94BBE28DEC9CECACECBCE3A3
:1082C00089839A83AB83BC83CE010196D6DF249643
:1082D000E2E00C94D7E2A4E0B0E0E1E7F1E40C9432
:1082E000BBE28DEC9CECACECBDE389839A83AB8361
:1082F000BC83CE010196C1DF2496E2E00C94D7E264
:10830000A4E0B0E0E6E8F1E40C94BBE280E090E0A9
:10831000A0E8BFE389839A83AB83BC83CE01019637
:10832000ACDF2496E2E00C94D7E2A4E0B0E0EBE905
:10833000F1E40C94BBE280E090E0A0E2B1E4898338
:108340009A83AB83BC83CE01019697DF2496E2E04B
:108350000C94D7E281E08093930280914B07877061
:10836000873051F010924B071092080486EB95E08D
:108370009093DC068093DB068091B8028093E6033D
:1083800080E00E94A27320E040E070E060E08AECB0
:1083900091E4E2CE80916701882331F041E062EA06
:1083A00073E082E00E9447BC8091080487708730A8
:1083B00071F41092E50320E040E070E060E081E5B8
:1083C0009CE4CADE81E08093E4030C94522008957B
:1083D00020E040E070E060E083EA95E7BDCE1092D7
:1083E0007D070E945B25F4CFCF93DF93C0911E07DA
:1083F000C7FD1FC084E0C802E0011124FE01EF5355
:10840000FD4F80819181181619063CF4863F910535
:1084100014F085EF90E00E941DC2CF53DD4F8A819A
:108420009B818F3F910519F010F08FEF90E08093C2
:108430007D07CEDFDF91CF910895B0E0A0E0E3E2C9
:10844000F2E40C94B5E2CDB6DEB6EEE4F7E0DF017F
:108450000D900020E9F7CD01865497402DB73EB727
:10846000281B390B0FB6F8943EBF0FBE2DBF0DB7BA
:108470001EB70F5F1F4FFF93EF9389E195E09F9326
:108480008F931F930F930E945EDB780134E0E30E1D
:10849000F11C0F900F900F900F900F900F90D7013D
:1084A0008D917D01882349F0082E000C990B0E94C4
:1084B000C4E4F70131978083F2CF64E175E0C8012D
:1084C0000E94F7DA4FE350E0B8018DED96E00E948C
:1084D0001CE50FB6F894DEBE0FBECDBE79DF0E945C
:1084E00054B8E8E00C94D1E280931E0720E040E00D
:1084F00070E060E08FE69CE42FCECF93DF93C091D5
:10850000D803CC23B1F0C150C093D80389E0C89FF1
:10851000E0011124CE55DC4F6A817B812F814E8191
:108520008881998119DE888580939302DF91CF91AC
:1085300008954EDFFBCFA4E0B0E0E1EAF2E40C9452
:10854000AFE20E945BBDF090380785E0782E7F0C8B
:1085500085E0E82EEF1884E0D82EDF18AA24AA942C
:10856000B12C83E0C82ECF1882E0982E9F1881E0AE
:10857000882E8F186F2C6194F11027C080913B07D3
:108580008823A1F080916701882359F081E09091C0
:108590003B07911180E024E047E156E0662D0E9400
:1085A000A7BC80917D0780931E0768C08091220739
:1085B00010922207882331F3A0DF80913A078823A5
:1085C00009F32496EEE00C94CBE221E0F21276C09F
:1085D00080913B07813009F458C08091670188235E
:1085E00001F311E080913B07813009F010E06091C8
:1085F000100170911101072E000C880B990B0E943D
:10860000CBDB69837A838B839C83CE010196ECDC80
:1086100000E09C0141E156E0682D812F0E944B6FE4
:1086200080917D0780931E0723E0F2129CC0109278
:10863000470780913B07833009F482C0809167012E
:108640008823E1F011E080913B07833009F010E0CE
:1086500080911E0724E6829FC001112481589F4FFC
:10866000B5010E945BE2862F0E94121B00E09C0174
:1086700040E056E06C2D812F0E944B6FF394F71071
:108680007BCF86E0809339079CCF809122071092A0
:108690002207882309F4A1CF10E000E027EE33E0A1
:1086A0004AE050E060E171E081E196E00E9420BE86
:1086B00080913A07882309F490CF83CF82E0F812A3
:1086C000AFCF80913B07823011F180916701882301
:1086D00009F467CF11E080913B07823009F010E088
:1086E0006091881270918912072E000C880B990BEB
:1086F0000E94CBDB69837A838B839C83CE010196B6
:1087000073DC00E09C014AE056E0692D86CF809141
:108710002207109222078823C1F20E944FBD0FED5D
:108720001FE125EF30E050E040E068E872E18AE0C8
:1087300096E00E9420BE80913A07882331F241CF13
:108740008091220710922207882309F477CF0E9494
:108750004FBD80E096E00E9495C080913A07882343
:1087600009F46CCF2ECF84E0F8123DC080913B0716
:10877000843011F180916701882309F47FCF11E0E3
:1087800080913B07843009F010E060912C017091DA
:108790002D01072E000C880B990B0E94CBDB6983FF
:1087A0007A838B839C83CE0101961EDC00E09C01C2
:1087B0004BEF55E06D2D5FCF80912207109222077D
:1087C0008823C1F203E31BE127EE33E04AE050E0E7
:1087D0006CE271E08BEF95E00E9420BE80913A0739
:1087E000882341F2EECE25E0F21248CF80913B077C
:1087F000853091F080916701882309F43FCF81E0B3
:1088000090913B07953009F080E023E04CEE55E075
:108810006E2D0E94A7BC32CF8091220710922207B2
:10882000882341F38FEA9CE40E94B1BD80913A070E
:10883000882301F3C6CEA7E0B0E0E1E2F4E40C94B3
:10884000ABE2A0908812B09089120E945BBD70903C
:1088500038077E8225E0270D2D8388248A94912C69
:1088600082E087198F8381E0682E6718472C419436
:1088700054EFE52E51E4F52E6CECC62E65E0D62EB5
:1088800085E0582E5718711015C080913B0788233A
:1088900009F4DBC080916701882309F433C181E0CA
:1088A00090913B07911180E024E047EE55E0642D64
:1088B0000E94A7BC809188129091891290931F0703
:1088C00080931E0781E0781229C080913B07813098
:1088D00009F4CCC080916701882309F44DC011E0F0
:1088E00080913B07813009F010E060911E07709184
:1088F0001F07072E000C880B990B0E94CBDB6983A6
:108900007A838B839C83CE0101966EDB00E09C0111
:1089100040EE55E0662D812F0E944B6F80917D07C0
:1089200080931E0792E0791227C01092470780912A
:108930003B07823009F4B5C0809167018823E1F0DC
:1089400011E080913B07823009F010E080911E0712
:1089500024E6829FC001112481589F4FB4010E94D8
:108960005BE2862F0E94121B00E09C0146ED55E061
:108970006F81812F0E944B6F10E000E033E0332EB7
:10898000272C8E81281A00931E07731027C0F80128
:10899000EE0FFF1FE154FA4F859194919093490790
:1089A0008093480780913B07871509F48DC080911B
:1089B0006701882399F0FF92EF92DF92CF922F9276
:1089C00081E090913B07931180E08F930E94C42037
:1089D0000F900F900F900F900F900F90832D0F5FBF
:1089E0001F4F94E0392E843071F6A114B10409F4BC
:1089F00087C095E0791221C080913B07853009F44A
:108A000071C0809167018823C1F08FEE91E49F933C
:108A10008F9383EC95E09F938F935F9281E0909189
:108A20003B07953009F080E08F930E94C4200F909F
:108A30000F900F900F900F900F9086E073942D8100
:108A4000271121CF809339070DC080912207109202
:108A50002207882309F41ECF50DD80913A0788232E
:108A600009F418CF2796E2E10C94C7E2809122071F
:108A700010922207882309F42DCF0E944FBD04EDE8
:108A800010E225EF30E050E040E06EE177E080EE6C
:108A900095E00E9420BE80913A07882309F41ACFFE
:108AA000E1CF8091220710922207882309F444CF56
:108AB0000E944FBD86ED95E00E9495C080913A07D7
:108AC000882309F439CFCECF809122071092220754
:108AD000882309F46CCF88DC80913A07882309F455
:108AE00066CFC0CF8091220710922207882309F415
:108AF00088CF75DC80913A07882309F482CFB2CF02
:108B000085E09CCF809188129091891290931F07E5
:108B100080931E0703CFB0E0A0E0E1E9F5E40C94F8
:108B2000B2E20E945BBDC091380785E0E82EEC0EF2
:108B30009BE9C92E95E0D92ED4E0DC1B13E01C1B69
:108B400026EBA22E25E0B22E02E00C1B81E0F82ECF
:108B5000FC1A9C2E9194C1112AC080913B07882356
:108B6000B1F080916701882359F081E090913B0733
:108B7000911180E024E04AEB55E0692D0E94A7BCEA
:108B8000CF5FEC12E8CF85E0809339070BC080916E
:108B9000220710922207882321F3AFDC80913A0745
:108BA0008823F9F2CDB7DEB7EBE00C94CEE2C1300A
:108BB00011F580913B07813079F08091670188231E
:108BC000F9F281E090913B07913009F080E023E0D9
:108BD0004FE35CE26F2DD2CF8091220710922207E3
:108BE000882359F388E696E40E94B1BD80913A0744
:108BF000882319F3D7CFC23009F053C090913B07B7
:108C0000923071F080916701882309F4B9CF81E037
:108C1000923009F080E020E24CEA55E0602FAECFC0
:108C20008091220710922207882361F3B092DC061C
:108C3000A092DB0680913A07882321F3B3CF80917D
:108C40003B07833081F080916701882309F498CF36
:108C500081E090913B07933009F080E023E04FE9F9
:108C600055E0612F8BCF8091220710922207882335
:108C700051F381EC9CE50E94B1BD80913A078823B5
:108C800011F390CF8091220710922207882391F050
:108C9000D092DC06C092DB0680913A07882351F01F
:108CA00081CFC33061F2C43009F06ACF90913B07A5
:108CB000943041F380916701882309F461CF81E00A
:108CC000943009F080E020E24AE855E06D2F56CF5D
:108CD000B0E0A0E0EEE6F6E40C94B6E20E945BBDE4
:108CE000C091380785E0E82EEC0ED4E0DC1B13E0E1
:108CF0001C1B02E00C1B81E0F82EFC1ADC2ED19428
:108D0000C1112AC080913B078823B1F0809167018F
:108D1000882359F081E090913B07911180E024E095
:108D200043E855E06D2D0E94A7BCCF5FEC12E8CF61
:108D300085E0809339070BC08091220710922207AB
:108D4000882321F3DADB80913A078823F9F2CDB743
:108D5000DEB7E7E00C94D2E2C13011F580913B0719
:108D6000813079F0809167018823F9F281E0909158
:108D70003B07913009F080E023E045E65CE26F2D8F
:108D8000D2CF8091220710922207882359F384EED4
:108D900090E20E94B1BD80913A07882319F3D7CFA2
:108DA000C23009F055C080913B07823081F080913C
:108DB0006701882309F4B9CF81E090913B07923095
:108DC00009F080E023E04EE55CE2602FACCF8091BB
:108DD000220710922207882351F38FED90E20E9420
:108DE000B1BD80913A07882311F3B1CF80913B0741
:108DF000833081F080916701882309F496CF81E068
:108E000090913B07933009F080E023E047E55CE276
:108E1000612F89CF8091220710922207882351F376
:108E20008AED90E20E94B1BD80913A07882311F348
:108E30008ECF8091220710922207882391F081E340
:108E400091E40E94B1BD80913A07882351F07FCF11
:108E5000C33061F2C43009F068CF80913B078430A1
:108E600041F380916701882309F45FCF81E09091FD
:108E70003B07943009F080E023E049E45CE26D2F89
:108E800052CFACE0B0E0E7E4F7E40C94ACE29C87AE
:108E90008B87362E8091220710922207882339F083
:108EA000109293022ADB2C96E1E10C94C8E26091C7
:108EB0003D0770913E0780913F07909140076115F3
:108EC00071058105910509F45CC0209112012223EE
:108ED00009F4AEC0209113012111AAC021E032167D
:108EE00009F484C0E2E03E1609F491C0C090140178
:108EF000D0901501E0901601F090170140902001EC
:108F00005090210160902201709023010E94CBDBE0
:108F1000209108013091090140910A0150910B0103
:108F20000E942ADC6F83788789879A87F4E03F9EC6
:108F300080011124C8018E589E4F9E838D83FC01B1
:108F400020813181428153816F81788589859A851D
:108F50000E94E3E24B015C01A3019201C701B6014B
:108F60000E94C5DB811173C0F801EE58FE4F80826C
:108F70009182A282B382832D0E94F46781E0809364
:108F8000670110923D0710923E0710923F07109222
:108F9000400780916701882309F485CF24E0329E41
:108FA000F0011124EE58FE4FC080D180E280F380A2
:108FB000C982DA82EB82FC822DEC3CEC4CEC5DE366
:108FC000609108017091090180910A0190910B0153
:108FD0000E9446E487FD65C0CE0101960E9460199B
:108FE000BC018B859C850E94E46E5DCFC09018010A
:108FF000D0901901E0901A01F0901B0140902401DB
:109000005090250160902601709027017FCFC0907D
:109010001C01D0901D01E0901E01F0901F014090B6
:1090200028015090290160902A0170902B016ECF89
:10903000412C20E5522E23EC622E27E4722EC12C07
:1090400030E5D32E33ECE32E37ECF32E5FCF20E068
:1090500030E0A9016F81788589859A850E94C5DBFA
:1090600087FF0FC0A7019601C501B4010E94C5DBAF
:1090700087FF7ACFED81FE81C082D182E282F382C6
:109080007ACFA3019201C501B4010E9446E41816EB
:109090000CF06ACFED81FE81408251826282738240
:1090A0006ACF20E030E44CE156E4C701B6010E94EB
:1090B0002ADC4B015C0120E030E0A901C701B601C8
:1090C0000E94C5DB20E030E040EA50E487FF04C0A6
:1090D00020E030E040EA50ECC501B4010E94E3E238
:1090E0002DEC3CEC4CEC5DE30E942ADC0E94C2E3D8
:1090F0006B017C01F7FC64C020EA36E841E050E0F7
:109100000E946EE2CA01B9012AE030E040E050E07E
:109110000E946EE2605D60939402C701B60120E197
:1091200037E240E050E00E946EE28AE0882E912C07
:10913000A12CB12CCA01B901A50194010E946EE2D3
:10914000605D60939502C701B60128EE33E040E010
:1091500050E00E946EE2CA01B901A50194010E948B
:109160006EE2605D609396028EE280939702C70183
:10917000B60124E630E040E050E00E946EE2CA0111
:10918000B901A50194010E946EE2605D60939802AE
:10919000C701B601A50194010E946EE26B017C013A
:1091A000CA01B901A50194010E946EE2605D60935D
:1091B000990280E3C80EC0929A0284E992E010CF2F
:1091C000F094E094D094C094C11CD11CE11CF11C1B
:1091D0006DE2A1CF62E087E59CE253CE61E08EE5CF
:1091E0009CE24FCE60E085E69CE24BCEA4E0B0E08E
:1091F000ECEFF8E40C94BBE2809122071092220776
:10920000882339F01092930278D92496E2E00C94E6
:10921000D7E260913D0770913E0780913F079091A2
:109220004007611571058105910561F10E94CBDB55
:10923000209108013091090140910A0150910B01E0
:109240000E942ADC20917E0130917F0140918001B3
:10925000509181010E94E3E260937E0170937F014F
:10926000809380019093810183E00E94F46781E004
:109270008093670110923D0710923E0710923F07BE
:109280001092400780916701882309F4BECF209196
:1092900023073091240740912507509126076091BC
:1092A0007E0170917F0180918001909181010E94E7
:1092B000E2E269837A838B839C83CE0101960E94CC
:1092C0006019BC0189E49CE20E94E46E9ECFB0E08C
:1092D000A0E0EDE6F9E40C94B6E20E94FA20082F33
:1092E0000E945BBDC0913807FC2E85E0E82EEC0E95
:1092F00011E01C1BDC2ED194C11114C080913B07DE
:109300008823F9F080916701882309F473C081E014
:1093100090913B07911180E024E04CE753E06D2DE4
:109320000E94A7BC011139C0D2E0C130B9F58091CB
:109330003B078130B1F080916701811121C0D2E0FB
:1093400043C080912207109222078823D9F2D5D8F2
:1093500080913A078823B1F2CDB7DEB7E7E00C94ED
:10936000D2E28091220710922207882321F386E11E
:109370009AE40E94B1BD80913A078823E1F2ECCFD4
:1093800081E090913B07913009F080E023E043E7D2
:1093900053E0612F0E94A7BCD2CFD1E0DC1314C0F0
:1093A00080913B078D17B9F080916701882361F0A8
:1093B0006C2F6F1981E090913B079C1380E023E0B4
:1093C00047E653E00E94A7BCCF5FCE1195CFDF5F89
:1093D000D0933907C1CF80912207109222078823AA
:1093E00019F388E39FE40E94B1BD80913A07882376
:1093F000D9F2B2CFD1E0002309F4A1CFE5CF80E0CC
:1094000090E0A0E8B0E480937A0190937B01A09370
:109410007C01B0937D0187E192E00E944A20809117
:10942000E6030E94A2731092930267C8B0E0A0E026
:10943000ECE1FAE40C94B4E20E945BBDC091380701
:1094400085E0C82ECC0ED4E0DC1B13E01C1B82E0B0
:10945000F82EFC1A81E0E82EEC1ABC2EB194C11152
:109460002AC080913B078823B1F08091670188234F
:1094700059F081E090913B07911180E024E045E5AF
:1094800053E06B2D0E94A7BCCF5FCC12E8CF85E0E4
:10949000809339070BC080912207109222078823FE
:1094A00021F32BD880913A078823F9F2CDB7DEB7A4
:1094B000E9E00C94D0E2C13089F580913B0781301E
:1094C000C1F0809167018823F9F2DD24D394809163
:1094D0003B07813009F0D12C83E59DE00E94461CBA
:1094E00000E09C014AE453E06E2D8D2D0E944B6FED
:1094F000CBCF8091220710922207882311F30E947C
:109500004FBD44E259E263E57DE08AE493E00E94C6
:10951000C0BD80913A078823A1F2C8CFC23009F0BC
:1095200073C080913B078230B1F08091670188233E
:1095300009F4AACFDD24D39480913B07823009F04F
:10954000D12C87E59DE00E94461C00E09C014FE382
:1095500053E06F2DCACF80912207109222078823F3
:1095600021F30E944FBD43E259E267E57DE08FE3BE
:1095700093E00E94C0BD80913A078823B1F296CF54
:1095800080913B078330B1F080916701882309F413
:109590007BCFDD24D39480913B07833009F0D12C1D
:1095A0008BE59DE00E94461C00E09C0144E353E0F3
:1095B000612F9BCF8091220710922207882321F3ED
:1095C0000E944FBD42E259E26BE57DE084E393E007
:1095D0000E94C0BD80913A078823B1F267CF809185
:1095E0002207109222078823C9F00E944FBD41E252
:1095F00059E26FE57DE089E293E00E94C0BD809171
:109600003A07882359F052CFC33009F4B9CFC43098
:1096100009F03ACF80913B07843009F380916701CC
:10962000882309F431CFDD24D39480913B07843023
:1096300009F0D12C8FE59DE00E94461C00E09C01C2
:1096400049E253E06D2F51CFA3E0B0E0EAE2FBE442
:109650000C94ABE24C013B015A011901280181E055
:109660008093930240913D0750913E0760913F07E0
:1096700070914007411551056105710571F014168F
:1096800015060CF080E08093E40310923D071092E1
:109690003E0710923F07109240071091E40380911B
:1096A00022078B8310922207811105C080916701E8
:1096B000882309F46FC0C2010E949C68082F80E0D3
:1096C000C114D10419F0C6010E949C681A82198243
:1096D000E114F104B1F4402F50E0282F30E0CA012A
:1096E000820F931F46976CF485E190E0841B950BE5
:1096F000821B930B97FD0196959587958A8381E050
:10970000898301E028E332E6A201BE016F5F7F4F4B
:10971000CE0102960E94F469E114F10491F08A816D
:10972000882321F01A8289818F5F898300E02BE3EF
:1097300032E6A701BE016F5F7F4FCE0102960E9405
:10974000F469C114D10459F000E028E332E6A6011F
:10975000BE016F5F7F4FCE0102960E94F46941E027
:109760004127B30181E00E94EEC4C4010E949C68BD
:10977000412FB40194E1981B892F0E94EEC4EB8124
:10978000EE2341F0111101C05101A114B10431F0D7
:10979000F50109952396E2E10C94C7E20E947D420F
:1097A000F9CFCF92DF92EF92FF920F931F9384E64F
:1097B000C82E85E0D82EF12CE12C06E615E030E02D
:1097C00020E04AE251E466E775E08BE795E03CDF94
:1097D0001F910F91FF90EF90DF90CF900895B0E030
:1097E000A0E0E5EFFBE40C94B3E2ADB6BEB6809129
:1097F000F90F6EE477E0882311F069EF7FE0FB0159
:1098000001900020E9F7CF01861B970B01962DB739
:109810003EB7281B390B0FB6F8943EBF0FBE2DBFC5
:109820008DB79EB701967C0180E2EDB7FEB78183CC
:10983000C70101960E9407E580E2C82E85E0D82E78
:1098400002E215E030E020E04DE152E46EE275E026
:1098500085E395E0F9DE0FB6F894BEBE0FBEADBE4F
:10986000EAE00C94CFE2CF92DF92EF92FF920F9357
:109870001F938EE7C82E84E0D82EF12CE12C01EF47
:1098800014E030E020E04CE058E560E874E085E862
:1098900094E0DADE1F910F91FF90EF90DF90CF9070
:1098A0000895CF92DF92EF92FF920F931F938AE871
:1098B000C82E83E0D82EF12CE12C0CE813E02FEF1A
:1098C00039E442E550E268E973E08DE993E0BCDEFB
:1098D0001F910F91FF90EF90DF90CF900895B0E02F
:1098E000A0E0E5E7FCE40C94B3E2ADB6BEB683E3DA
:1098F00092E00E949C6890E001962DB73EB7281B2D
:10990000390B0FB6F8943EBF0FBE2DBF8DB79EB773
:1099100001967C0163E372E00E940DDB80911E07DB
:1099200000E012E0813031F00BEE11E0823011F0F6
:1099300003E112E084E2C82E82E0D82E28EE31E462
:1099400043ED53E566E272E08DE292E07DDE0FB614
:10995000F894BEBE0FBEADBEEAE00C94CFE28F928B
:109960009F92AF92BF92CF92DF92EF92FF920F93AE
:109970008091220710922207882371F0109293029F
:109980000E947D420F91FF90EF90DF90CF90BF90AB
:10999000AF909F908F90089581E080939302809183
:1099A0003D0790913E07A0913F07B0914007009777
:1099B000A105B10509F44AC05C01AA0CBB1CAA0CA4
:1099C000BB1C10923D0710923E0710923F07109269
:1099D0004007B5010B2C000C880B990B0E94CBDBC8
:1099E0002091860730918707409188075091890719
:1099F0000E942ADC2091FB123091FC124091FD1252
:109A00005091FE120E94E3E26B017C0120E030E005
:109A100040EA51EC0E9446E487FD18C020E030E0A7
:109A200040EA51E4C701B6010E94C5DB181674F084
:109A3000C5010E94C5B8C092FB12D092FC12E09200
:109A4000FD12F092FE1282E080936701809167011F
:109A5000882309F497CFC090FB12D090FC12E090BD
:109A6000FD12F090FE1220E030E44CE156E4C70114
:109A7000B6010E942ADC4B015C0120E030E0A90124
:109A8000C701B6010E94C5DB20E030E040EA50E4A7
:109A900087FF04C020E030E040EA50ECC501B4018B
:109AA0000E94E3E22DEC3CEC4CEC5DE30E942ADCEE
:109AB0000E94C2E36B017C018BE2F7FE09C0F094C7
:109AC000E094D094C094C11CD11CE11CF11C8DE227
:109AD00080939402C701B60120E137E240E050E0F4
:109AE0000E946EE26AE0862E912CA12CB12CCA0154
:109AF000B901A50194010E946EE2605D6093950238
:109B0000C701B60128EE33E040E050E00E946EE26B
:109B1000CA01B901A50194010E946EE2605D6093E3
:109B200096028EE280939702C701B60124E630E0E8
:109B300040E050E00E946EE2CA01B901A501940123
:109B40000E946EE2605D60939802C701B601A501B4
:109B500094010E946EE26B01CA01B901A501940152
:109B60000E946EE2605D6093990260E36C0D609309
:109B70009A0264E972E084EF92E00E94E46EC09081
:109B8000FB12D090FC12E090FD12F090FE1280903B
:109B9000E0039090E103A090E203B090E303A501FD
:109BA0009401C701B6010E94C5DB8823E9F020E0DB
:109BB00030E0A901C701B6010E94C5DB882309F482
:109BC00079C0A5019401C701B6010E94C5DB87FDDC
:109BD00073C081E08093DF03C092E003D092E10381
:109BE000E092E203F092E303D090DF0380916413EC
:109BF000813188F480916613833068F044E04D1918
:109C00005CEDE52E52E0F52E0CE022E062E480E30C
:109C100093E10E942AC680916413853180F480917B
:109C20006613843160F049EDE42E42E0F42E01E049
:109C300023E044E16CE380E393E10E942AC6809133
:109C400064138F3308F09ECE809166138F3208F430
:109C500099CE40E34D198FEBE82E82E0F82E0DE00F
:109C600022E06AE580E393E10E942AC641E34D19B0
:109C700095EAE92E92E0F92E22E065E080E393E197
:109C80000E942AC625E7E22E22E0F22E00E123E020
:109C90004FE262E180E393E10E942AC635E4E32EBD
:109CA00032E0F32E23E04FE267E680E393E10E9487
:109CB0002AC668CE80E08ECF8FEF8CCF0F931F9394
:109CC000CF93DF93FC01EB0180913D0790913E071C
:109CD000A0913F07B0914007B7FF08C010923D0721
:109CE00010923E0710923F071092400780912C0778
:109CF00090912D07A0912E07B0912F0740913D071D
:109D000050913E0760913F07709140078417950777
:109D1000A607B70744F480933D0790933E07A093AE
:109D20003F07B0934007809167018823E1F060917D
:109D30003D0770913E0780913F0790914007009149
:109D40003007109131072091320730913307600FAF
:109D5000711F821F931F0995BC0180913607909156
:109D600037070E94E46E80912207811108C080911C
:109D700029078823A9F180916701882389F18091BF
:109D80003407909135070097B1F040913D0750910D
:109D90003E0760913F077091400700913007109196
:109DA00031072091320730913307400F511F621F56
:109DB000731FFE010995E0912A07F0912B07309758
:109DC00041F080912907811103C080912207811100
:109DD0000995809122071092220781110E947D42ED
:109DE000DF91CF911F910F9108956CE47BE185E69F
:109DF0009BE164CF69EC7BE181EE9FE35FCF67ED90
:109E00007BE18AEF9CE15ACF6BEE7BE18FEF9BE128
:109E100055CF68E37CE18DEF9FE350CFE091D8030D
:109E2000E63028F581E08E0F8093D80340913D07FE
:109E300050913E0760913F0770914007209138078D
:109E4000909139078091930239E0E39FF00111244A
:109E5000EE55FC4FA0912A13B0912B13B183A08330
:109E60004283538364837583268397838087089511
:109E7000A7E0B0E0EEE3FFE40C94ABE20E945BBD30
:109E8000F09038072F2C85E08F0D8D833324339489
:109E900083E0E82E98EE892E93E0992EA12CB12C28
:109EA00084E08F198E839E2D9F199F8382E0D82E88
:109EB000DF18C32CCF18F1102CC080913B078823EA
:109EC000C1F080916701882361F0622D619581E086
:109ED00090913B07911180E024E045E553E00E941A
:109EE000A7BCF3949D81F912E6CF85E080933907F2
:109EF0000CC08091220710922207882311F30E9440
:109F00007D4280913A078823E1F22796E2E10C94A2
:109F1000C7E281E0F8122DC090913B079130B9F073
:109F2000809167018823E9F281E0913009F080E0B7
:109F3000909197032DE133E0911102C029E133E0C4
:109F400001E040E253E06C2D0E944B6FCACF80913C
:109F5000220710922207882319F3809197038F25F7
:109F600080939703E092670180913A078823C1F2BA
:109F7000CCCF92E0F912D1C080913B07823021F121
:109F800080916701882309F4ACCF11E080913B07F1
:109F9000823009F010E06091060170910701072EF0
:109FA000000C880B990B0E94CBDB69837A838B832F
:109FB0009C83CE0101960E94F43F00E09C0142E1A7
:109FC00053E06D2D812FC0CF809122071092220780
:109FD0008823B1F210E000E025EF30E050E040E0EF
:109FE00066E071E082E193E00E9420BE80913A0732
:109FF000882331F28ACF80913B07833019F1809119
:10A000006701882309F46DCF11E080913B0783300D
:10A0100009F010E06091040170910501072E000C19
:10A02000880B990B0E94CBDB69837A838B839C839B
:10A03000CE0101960E94F43F00E09C014BE053E00A
:10A040006F81C0CF80912207109222078823B9F236
:10A0500010E000E025EF30E050E040E064E071E027
:10A060008BE093E00E9420BE80913A07882339F26A
:10A070004CCF8091220710922207882309F459C0FF
:10A0800020E030E048EC52E4609100017091010161
:10A0900080910201909103010E942ADC0E94C7E393
:10A0A0002B0130923A07BADEE092670183E093E039
:10A0B000909337078093360780E091E090933507BF
:10A0C00080933407109230071092310710923207B4
:10A0D0001092330780922C0790922D07A0922E07A2
:10A0E000B0922F07712C612C40923D0750923E0791
:10A0F00060923F077092400784E09FE490932B1397
:10A1000080932A1310922B0710922A071092290786
:10A1100080913A07882369F0F8CE83E0F81609F4B5
:10A120006ACF94E0F912DDCE80913B07843009F4C8
:10A13000A0CF80916701882309F4D3CE11E08091EC
:10A140003B07843009F010E040900001509001017D
:10A15000609002017090030120E030E0A901C3018A
:10A16000B2010E94C5DB2DEB37E346E055EB87FDDE
:10A1700004C02DEB37E346E055E3C301B2010E9472
:10A18000E3E269837A838B839C83CE0101960E94EC
:10A19000D61900E09C0143E053E06E8113CFB0E09C
:10A1A000A0E0E5EDF0E50C94BBE28D8190916A10A2
:10A1B000891778F080936A109E01285F3F4F4E8187
:10A1C0005F8164E570E085E190E10E948DDB109293
:10A1D0001410E2E00C94D7E20F931F93CF93DF9318
:10A1E0008C016F3F19F410926A1060E020916A10A0
:10A1F000862F062E000C990B2817190609F004F576
:10A2000060936A10C8010E9414DB800F911FEC015B
:10A21000C01BD10BC535D1053CF00197FC01249141
:10A22000207C2038D1F3F3CFDD27AE01B80185E1E2
:10A2300090E10E9435DBCB5EDF4E18821092141045
:10A24000DF91CF911F910F9108958F929F92AF92BE
:10A25000BF92DF92EF92FF920F931F93CF93DF9302
:10A26000CDB7DEB7C658D1090FB6F894DEBF0FBE22
:10A27000CDBFC358DF4F188219821A821B82CD5777
:10A28000D0408091870290918802A0918902B0917C
:10A290008A02CF57DF4F88839983AA83BB83C15833
:10A2A000D04084E690E090937412809373121092E1
:10A2B0009812109297121092150464E070E0CE018B
:10A2C0008F579F4F0E9483C1809173129091741297
:10A2D00002969093741280937312109298121092B7
:10A2E000971281E0CA57DF4F8883C658D040CE010D
:10A2F0008A579F4F0E94202068E470E08FE39DE022
:10A300000E9483C180E1EEE8F1E08E010F5F1F4FF4
:10A31000D80101900D928A95E1F760E170E0C801E3
:10A320000E9483C181E697E00E9428208CE0F8011A
:10A3300011928A95E9F7C8010E9424207E01FDE66A
:10A34000EF0EF11C8FEFF7018083C7010E942020E0
:10A3500019821A821B821C82C8010E9428208091C7
:10A36000B4029091B502A091B602B091B702898370
:10A370009A83AB83BC83C8010E942820C358DF4F57
:10A38000188219821A821B82CD57D04083E0F701D0
:10A3900080838983CE0183589F4F0E942820C70164
:10A3A0000E942020C8010E9420203AE0D32EDA9497
:10A3B000DD2031F0CE0183589F4F0E942820F7CF37
:10A3C00083EF92E10E942420C358DF4F1882198244
:10A3D0001A821B82CD57D0402AE0D22EDA94DD209B
:10A3E00031F0CE0183589F4F0E942820F7CF87E09D
:10A3F0008983F7018083C8010E942020C7010E9441
:10A40000202068E070E089EB92E00E9483C168E060
:10A4100070E08CEA92E00E9483C164EC70E089EC09
:10A4200092E00E9483C11982BB24BA94F701B082E2
:10A43000C8010E94D9C1C7010E94202080E1D82E06
:10A44000F8018D2D11928A95E9F760E170E0C8015D
:10A450000E9483C11982C8010E94D9C168E070E0DE
:10A4600081EC92E00E9483C1198A1A8A1B8A1C8A95
:10A4700080E090E0A0E8BFE38D879E87AF87B88B30
:10A4800080918B1290918C12A0918D12B0918E12AE
:10A4900089839A83AB83BC8320E030E543EC50E4AE
:10A4A00060918F12709190128091911290919212FE
:10A4B0000E942ADC6D837E838F8398872CEA35EC9B
:10A4C00047E25EE36091931270919412809195122D
:10A4D000909196120E942ADC69877A878B879C87E5
:10A4E00064E170E0C8010E9483C184E190E09A8336
:10A4F000898362E070E0C8010E9483C18CE0EEE9CC
:10A50000F1E0D80101900D928A95E1F7C8010E940F
:10A510001C208CE0EEE9F1E0D80101900D928A95C3
:10A52000E1F7C8010E941C201982C8010E94202066
:10A530008FE78983C8010E942020B982C8010E9448
:10A54000202085E0EAEAF1E0D80101900D928A9599
:10A55000E1F765E070E0C8010E9483C11982C8017B
:10A560000E94D9C180E2EFEAF1E0D80101900D929A
:10A570008A95E1F760E270E0C8010E9483C1F701AB
:10A580001082C7010E94D9C11982C8010E94D9C195
:10A5900080E090E0A0EEBFE3C358DF4F888399834B
:10A5A000AA83BB83CD57D040CE0183589F4F0E94D2
:10A5B0002820C358DF4F188219821A821B82CD5778
:10A5C000D040CE0183589F4F0E94282082E1F8019D
:10A5D00011928A95E9F762E170E0C8010E9483C197
:10A5E00084E2EFECF1E0D80101900D928A95E1F759
:10A5F00064E270E0C8010E9483C1F8011192DA940C
:10A60000E9F760E170E0C8010E9483C189E0F801C8
:10A6100011928A95E9F769E070E0C8010E9483C150
:10A62000C358DF4F188219821A821B82CD57D0403F
:10A63000CE0183589F4F0E9428209CE0D92EF8011C
:10A640008D2D11928A95E9F76CE070E0C8010E94A7
:10A6500083C18CE6F80111928A95E9F76CE670E007
:10A66000C8010E9483C189E094E00E941C20F70188
:10A67000108211821282138214821582168217822E
:10A6800068E070E0C7010E9483C1F7011192DA947B
:10A69000E9F7CB57DF4F1882C558D04080E090E0F3
:10A6A000A0E4B0E4ED968CAF9DAFAEAFBFAFED9739
:10A6B000C7010E942420CE018B579F4F0E9420206B
:10A6C000CE0187589F4F0E942820D0901504D110AA
:10A6D00048C00091731210917412045611098091B0
:10A6E000971290919812F7019183808384E690E00D
:10A6F000909374128093731264E070E08FE192E0A3
:10A700000E9483C162E070E0C7010E9483C10E9481
:10A71000F4808DE09AE00E94C47BC8010E947D75A0
:10A72000F70180809180B12CA12C80E09AE00E94FA
:10A73000C47BC501B4010E9420A58DEF99E00E9461
:10A74000C47B0431134041F00E94F1808FE19AE014
:10A750000E94C47BDD24D394809115048D298093BD
:10A76000150480911504811104C060E08DEE99E01C
:10A7700033DD9091150481E08927CA57DF4F0FB66A
:10A78000F894DEBF0FBECDBFDF91CF911F910F9127
:10A79000FF90EF90DF90BF90AF909F908F900895C3
:10A7A00054DD0C949840CF930E94163D4EDDC82F87
:10A7B000882319F080E00E94DE278C2F0E949840A9
:10A7C0000E94E841CF910895A4E0B0E0EAEEF3E5FD
:10A7D0000C94ACE29091DA06981709F474C0382E04
:10A7E00080E090E0A0E2B1E489839A83AB83BC83EC
:10A7F0004090FB125090FC126090FD127090FE127F
:10A8000020E030E0A901C301B2010E94C5DB87FF4F
:10A810000CC0A301920160E070E080E291E40E942C
:10A82000E2E269837A838B839C83CE0101960E9446
:10A8300077B84090720150907301609074017090ED
:10A8400075018090760190907701A0907801B0908A
:10A85000790163E972E084E690E00E946C406AEB63
:10A8600072E084E690E00E946C4009EB19E033202E
:10A8700011F006EC19E00E94E84163E6C801ACDC87
:10A88000C8010E94678160E070E0CB010E94C6C2EF
:10A890000E9454B819821A821B821C82E0907A01AD
:10A8A000F0907B0100917C0110917D01CE01019619
:10A8B0006C01A5019401C301B2010E94EE3A3092ED
:10A8C000DA060E940C3D80E02496E1E10C94C8E297
:10A8D0004F925F926F927F928F929F92AF92BF92B0
:10A8E000DF92EF92FF920F931F93CF93DF93D82EB7
:10A8F000C82FD0E0FE01E358F34DF49082E0D81663
:10A9000009F4E4C06F2DFF0C770B880B990B0E94A4
:10A91000CBDB2B013C01CE01880F991F880F991FBB
:10A920008F50994F0E9447714B015C01A301920126
:10A93000C501B4010E942ADC4B015C017E01EE0CD2
:10A94000FF1CEE0CFF1CC7018B51994F0E944771F1
:10A950009B01AC01C301B2010E942ADC20E030E07F
:10A9600040EC5FE30E942ADCAB01BC0100E010E098
:10A9700098018D2D0E949ABB20E030E0A901C5010D
:10A98000B4010E94C5DB882309F440C082E000E0E6
:10A9900010E020E830E4D81619F000E010E098014B
:10A9A000B501A40170588D2D0E949ABBA501940198
:10A9B000C501B4010E94E3E24B015C0182E000E0CA
:10A9C00010E020E030E4D816E1F0FE01EA52F94F41
:10A9D0006491611107C00E94F48084EB96E00E94AC
:10A9E000C47B6AE070E090E080E00E94C9DB9B01DC
:10A9F000AC0161E070E088E492E40E945AE38B01CC
:10AA00009C01B501A4018D2D0E949ABB81E090E0CC
:10AA10000D2C01C0880F0A94EAF790914B07982BF0
:10AA200090934B0790910804892B80930804C701E9
:10AA30008752994F0E944771F701EE58FE4F60838D
:10AA400071838283938382E0D8121AC02091FB1213
:10AA50003091FC124091FD125091FE1260917A01EA
:10AA600070917B0180917C0190917D010E94E2E2D6
:10AA700060937A0170937B0180937C0190937D01B8
:10AA80000E94203CF701E456FD4FD701AE58BE4F5F
:10AA90008D919D910D90BC91A02D80839183A28377
:10AAA000B38382E0D81202C080E08EDEDF91CF91C6
:10AAB0001F910F91FF90EF90DF90BF90AF909F900C
:10AAC0008F907F906F905F904F90089581E07CDE33
:10AAD0008111ECCF89EF96E00E94477120E030E0D1
:10AAE000A9010E94C5DB882309F40CCF6F2DFF0C50
:10AAF000770B880B990B0E94CBDB2B013C0189EF74
:10AB000096E00E9447714B015C0120E030E040EA92
:10AB100050E40E9446E487FF09CF812C912C90EAF3
:10AB2000A92E90E4B92E02CFCF9380919A03811180
:10AB300009C08CED91E09093DE038093DD0381E00A
:10AB400080939A036BD920E040E070E060E085E0FC
:10AB500091E20E94AC40C1E0C09393020E9425297B
:10AB60000E947D42C093930260E08FEA9CE234DB56
:10AB700088ED91E09093DC068093DB06CF910895F9
:10AB8000A6E0B0E0E6ECF5E50C94ABE20E9482753D
:10AB9000382E8091821484FB662460F8412C84FF57
:10ABA00003C00E949575482E0E945BBD2091380716
:10ABB0002D83522E2B5F298380E00FED14E091E06E
:10ABC000792E7518952D91959A8394E9E92E95E53E
:10ABD000F92E2CEFC22E24E0D22E92E095199B8301
:10ABE00093E095199C833BE9832E34E0932E40EB50
:10ABF000A42E44E0B42E9D812981921709F409C244
:10AC0000992349F131106AC00E94907B882309F48E
:10AC10007AC19D81913009F444C122E02E832D81B7
:10AC20008E8128135FC180913B07281709F46EC1FC
:10AC300080916701882309F455C16D81651981E010
:10AC400090913B072D81921380E023E048ED54E082
:10AC50000E94A7BC47C180913B07882379F180916E
:10AC60006701882379F281E090913B07911180E0A0
:10AC700024E048E055E06A810E94A7BC332021F21D
:10AC800024E02E839D812E8192134AC080913B0740
:10AC9000981709F44CC180916701882309F440C0DA
:10ACA0006D81651981E090913B072D81921380E0C1
:10ACB00023E04CEC54E00E94A7BC32C080912207F4
:10ACC00010922207882359F20E947D4280913A0710
:10ACD000882329F22696E2E10C94C7E28D81813027
:10ACE00009F47FC0823009F4A6C09D81933041F6FB
:10ACF00080913B07833009F4C3C0809167018823AA
:10AD000009F4BECF81E090913B07933009F080E0D9
:10AD100023E04CEE54E06C810E94A7BC84E08E835B
:10AD20008E818F5F9D81981316C080913B07981785
:10AD300009F40EC180916701882369F06D8165195E
:10AD400081E090913B072D81921380E023E04EEB50
:10AD500054E00E94A7BC8E818E5F662009F430C14A
:10AD600041103BC09D8198131BC020903B0792155A
:10AD700009F4FFC080916701882391F01F92BF9270
:10AD8000AF928D8185198F9381E02D81221180E012
:10AD90008F930E94C4200F900F900F900F900F90F0
:10ADA0008E818D5F9D81981316C080913B07981707
:10ADB00009F4F5C080916701882369F06D816519F8
:10ADC00081E090913B072D81921380E023E04FE9D1
:10ADD00054E00E94A7BC8E818C5F9D819F5F9D8304
:10ADE0000ACF80913B078130D1F0809167018823A1
:10ADF00009F446CFFF92EF92DF92CF927F9281E0EB
:10AE000090913B07913009F080E08F930E94C4201D
:10AE10000F900F900F900F900F900F9031CF809167
:10AE2000220710922207882301F37EDE80913A07E1
:10AE30008823D9F24FCF80913B07823091F08091E7
:10AE40006701882309F41CCF81E090913B07923081
:10AE500009F080E023E041EF54E06B810E94A7BC41
:10AE60000FCF8091220710922207882341F383E3BA
:10AE70009CE40E94B1BD80913A07882301F32ACF58
:10AE80008091220710922207882309F436CF8BE99C
:10AE900092E40E94B1BD80913A07882309F42DCF36
:10AEA00019CF80913B07813009F180916701882398
:10AEB00009F4B3CE85EB9EE39F938F931F930F937B
:10AEC0007F9281E090913B07913009F080E08F9371
:10AED0000E94C4200F900F900F900F900F900F9032
:10AEE00082E08E838E818F5F8E83CCCE809122070D
:10AEF000109222078823C9F20E94B53E80913A073A
:10AF0000882399F2E7CE91E09E8389CE8091220733
:10AF100010922207882309F48BCE8BE895E40E94D7
:10AF2000B1BD80913A07882309F482CED3CE8091B7
:10AF3000220710922207882309F4ADCE8BE194E416
:10AF40000E94B1BD80913A07882309F4A4CEC2CEF5
:10AF50008091220710922207882309F4EBCE83E325
:10AF60009FE50E94B1BD80913A07882309F4E2CEA3
:10AF7000B1CE8091220710922207882309F4FACEDD
:10AF80004FE350E06AE874E08DED96E00E941CE526
:10AF900080913A07882309F4EDCE8D811ECF8091F0
:10AFA000220710922207882309F404CF89E690E64D
:10AFB0000E94B1BD80913A07882309F4FBCEEDCF02
:10AFC0009D81981314C090913B072D81291791F012
:10AFD00080916701882359F06D81651981E02D8189
:10AFE000291380E020E24EE854E00E94A7BC8E8145
:10AFF0008D5FF3CE8091220710922207882341F3C0
:10B000009092DC068092DB0680913A07882301F358
:10B01000C4CF809339075ECE10925F07109266010D
:10B020000E9495759091821480FB97F990938214F9
:10B0300060E08AEC91E0D0D80C94E8410F931F9324
:10B040000E94DCC100918E0210918F02209190022B
:10B0500030919102601B710B820B930B97FD0CC01A
:10B0600089B183FB882780F991E089274A9B826018
:10B07000309B846080938D0280918D0281709091CD
:10B080008D0291FD826090919903981749F081306B
:10B0900009F148F0823079F0833091F08093990380
:10B0A0001F910F910895913079F09230B9F79091F6
:10B0B0008C0291500CC0992339F09330C1F3EECF3C
:10B0C0009130A9F3923051F790918C029F5F909349
:10B0D0008C02E4CF992359F3933001F7F5CF1F93F6
:10B0E000CF93DF93809134018F3708F468C08F5776
:10B0F00090918A1290938404992309F465C05D9A13
:10B100008F5F809334018091830491E0892780933D
:10B110008304811193DF8091330191E0980F833094
:10B120000CF090E0813009F485C00CF04FC088230A
:10B1300009F462C090933301C0914C07D0914D0740
:10B14000209709F42DC0F89413B1147082E00E9486
:10B15000C92700C000C01C161D060CF08BC02A9A1F
:10B1600000C000C02B9A00C0000082E090E0019770
:10B17000F0F72B9800C000C0112309F47DC02A9A73
:10B1800000C000C0789480914C0790914D071C1628
:10B190001D060CF073C0019790934D0780934C07E8
:10B1A0008091870D9091880D009729F001979093D9
:10B1B000880D8093870DDF91CF911F910895909115
:10B1C0008404891708F49CCF5D989ACF8230E9F106
:10B1D000833009F0AFCF80918204811103C087E0F2
:10B1E000809382048091820481508093820488231A
:10B1F00009F4A0CF93E09ECF809132018F5F803120
:10B200001CF48093320196CF109232018091980302
:10B2100081110BC0209180123091811230938312E2
:10B220002093821281E080939803109281121092F1
:10B23000801280CF10927B0087E480937C00809105
:10B240007A00806480937A0075CF80917A0086FDC1
:10B250000FC0409178005091790020918012309178
:10B260008112240F351F309381122093801262CFF8
:10B2700092E060CF2A9874CF2A9882CF01968CCF23
:10B28000A4E8B0E0E6E4F9E50C94ABE22DB73EB7F4
:10B29000CD57DF4F39832883C358D04084E690E0F0
:10B2A00090937412809373121092981210929712C6
:10B2B00041E064E070E0CE0187589F4F0E947CA778
:10B2C00043E050E0BE0167587F4F8FE192E00E945B
:10B2D0000EE5892BF1F1ED968FADED97882339F0CE
:10B2E0008FE3EA968FAFEA97EB961FAEEB970E943B
:10B2F000F480BE0167587F4F87EB9AE00E94D17BB4
:10B3000089EA9AE00E94C47B82E00E94744281E054
:10B310008093150480918D03811107C080911D07D2
:10B32000833018F080E00E94DE279091150481E0C0
:10B330008927CD57DF4F28813981C358D0400FB6B8
:10B34000F8943EBF0FBE2DBFCC57DF4FE2E10C9407
:10B35000C7E241E062E070E0CE0183589F4F0E9457
:10B360007CA7E9961CAE1DAE1EAE1FAEE9971092EB
:10B37000981210929712CE018F579F4F0E94112062
:10B38000EDB6FEB6CF57DF4FC880C158D040D12CA4
:10B3900033E0C30ED11CCC0CDD1CCC0CDD1C8DB7F6
:10B3A0009EB78C199D090FB6F8949EBF0FBE8DBF36
:10B3B000EDB7FEB731963F012DB73EB72C193D09C9
:10B3C0000FB6F8943EBF0FBE2DBF8DB79EB7019646
:10B3D0004C01EDB7FEB7EC19FD090FB6F894FEBFAE
:10B3E0000FBEEDBF0DB71EB70F5F1F4FB601C301F4
:10B3F0000E94162040918D0381E0482764E070E0B0
:10B400008FE49DE00E947CA7B601C4010E94162033
:10B41000B601C8010E941620F0918D03CE57DF4F70
:10B42000F883C258D040F1114FC0CF57DF4F888109
:10B43000C158D04090E00296AFE3BDE050E040E05C
:10B4400030E020E067E27BE0E7E1CE2EEBE0DE2EAD
:10B45000F7E0AF2EFBE0BF2E821793070CF495C0E8
:10B46000F301E40FF51F20803180428053802D923C
:10B470003D924D925D92821793070CF48CC0F401BB
:10B48000E40FF51F208031804280538050962D922A
:10B490003D924D925C925397821793070CF481C0B2
:10B4A000F801E40FF51F2080318042805380909690
:10B4B0002D923D924D925C9293972F5F3F4F4C5F40
:10B4C0005F4F2430310541F683E79DE00E94E91F7C
:10B4D00087E79DE00E94E91F8BE79DE00E94E91F3E
:10B4E0008FE79DE00E94E91F83E89DE00E94E91F2D
:10B4F000CE018B589F4F0E94E91FCE018B589F4F62
:10B500000E94E91FCE018B589F4F0E94E91FCE0178
:10B510008B589F4F0E94E91F81E697E00E94E91F28
:10B520000FB6F894FEBE0FBEEDBE8E010F5F1F4F2B
:10B53000C8010E940920CE0183599F4F0E94F11F2C
:10B54000C8010E94E91F86E194E00E94E91FCE0134
:10B550008B589F4F0E94E91FCE0183599F4F0E9435
:10B560001120C8010E941120AE96CFACAE97898100
:10B57000C89E6001112421E0C21AD108C0F0CE019A
:10B580008B589F4F0E94E91FF6CFFB012590359005
:10B59000459054906CCFF60125903590459054908D
:10B5A00075CFF501259035904590549080CF83EF6D
:10B5B00092E10E9409208AE0D82EDA94CE01DD20A3
:10B5C00029F08B589F4F0E94E91FF7CF80589F4F5B
:10B5D0000E941120CE0181589F4F0E941120C05817
:10B5E000DF4F8881C058D040873009F046C1C1582C
:10B5F000DF4F8881CF57D040873009F03EC1CE570A
:10B60000DF4F8881C258D040811102C00E94A273CE
:10B6100089EB92E00E9401208CEA92E00E940120D6
:10B6200040918D0381E0482764EC70E089EC92E062
:10B630000E947CA7CE0183599F4F0E94F91FC80129
:10B640000E94F11F40918D03FF24F3944F2560E188
:10B6500070E0C8010E947CA7C8010E94F91F4091B8
:10B660008D034F2568E070E081EC92E00E947CA79A
:10B6700040918D034F2564E170E0C8010E947CA7D2
:10B68000D0908D03D11030C089819A81AB81BC816B
:10B6900080938B1290938C12A0938D12B0938E1284
:10B6A0002CEA35EC47E25EE36D817E818F819885DF
:10B6B0000E942ADC60938F127093901280939112F3
:10B6C0009093921220E030E543EC50E469857A854E
:10B6D0008B859C850E942ADC609393127093941250
:10B6E0008093951290939612FF24F3944D2D4F253D
:10B6F00062E070E0C8010E947CA7C8010E94E11FBF
:10B70000C8010E94E11FC8010E94F11FC8010E94E8
:10B71000F11FC8010E94F11F85E0F80111928A957E
:10B72000E9F740918D034F2565E070E0C8010E9464
:10B730007CA7C8010E94F91F40918D034F2560E24C
:10B7400070E0C8010E947CA7CE0183599F4F0E94E0
:10B75000F91F40918D034F2569E070E0C8010E94F8
:10B760007CA740918D034F2562E170E0C8010E94E3
:10B770007CA740918D034F2564E270E0C8010E94D0
:10B780007CA740918D034F2560E170E0C8010E94C5
:10B790007CA740918D034F2569E070E0C8010E94AD
:10B7A0007CA7C8010E94E91F40918D034F256CE0E2
:10B7B00070E0C8010E947CA740918D034F256CE684
:10B7C00070E0C8010E947CA719821A821B821C8229
:10B7D0001D821E821F82188619861A861B861C8669
:10B7E000C8010E94E11F40918D034F2568E070E081
:10B7F000C8010E947CA7C8010E940920CE0181587F
:10B800009F4F0E94F11FCE0183599F4F0E94E91F55
:10B8100080917312909174128837934009F44DC04F
:10B820000E94F1808FE19AE00E94C47BF09215049F
:10B830000E94F480609173127091741264567109C1
:10B8400081EA9AE00E945A8189E99AE00E94C47BC9
:10B8500084E193E00E947D758AE00E94A37B81E0F1
:10B860000E94744280918D03811154CD8091150402
:10B87000811150CD0E94643C4DCDCE0183599F4F24
:10B880000E940120C8010E940120C058DF4FC880DB
:10B89000C058D040C158DF4F8881CF57D040C89E94
:10B8A0006001112491E0C91AD10808F4C3CECE0179
:10B8B0008B589F4F0E94E91FF5CF109215042091DD
:10B8C000971230919812EF968EAD9FADEF97281793
:10B8D000390701F1F09215040E94F180EF960EAD48
:10B8E0001FADEF9789E79AE00E94C47BC8010E94D0
:10B8F0007D75009197121091981284E79AE00E944A
:10B90000C47BC8010E947D7584E69AE00E94C47BD6
:10B9100080E0A6CF80918D038111A4CF0E94F48096
:10B920008FE192E00E94AA7B609173127091741271
:10B930006456710987E49AE00E945A8180909712B8
:10B9400090909812B12CA12C8AE39AE00E94C47BBB
:10B95000C501B4010E9420A587E39AE00E94C47B40
:10B9600081CF81E080938D038BDC10928D0388233F
:10B9700009F086CC0E94163D80E00895F2DF0C9419
:10B980009840A7E0B0E0E7ECFCE50C94ABE28091D6
:10B990004B07877089838090B9029090BA02A0907B
:10B9A000BB02B090BC020E945BBD209138072E8381
:10B9B0003981373009F075C085E194E09B838A8333
:10B9C0001E81312F3B5F3C8333243394812F81953B
:10B9D0008D83232C211A84E6482E512C612C712C46
:10B9E0002E81222309F462C03981373009F434C230
:10B9F0002E81213009F029C290913B07913009F442
:10BA000045C180916701811154C182E0F82E81E027
:10BA10008F0D8F839981973009F063C020E030E06B
:10BA2000A901C501B4010E94C5DB882309F459C0EE
:10BA30003F818E81381331C09091B8029F838091ED
:10BA40003B072E81821311C080912207109222079A
:10BA5000882359F093259F8383E0809367010E9498
:10BA60003F2080913A0781110DC1809167018823A1
:10BA7000A1F06E81611B81E090913B073E819313A1
:10BA800080E09F8126EF33E0911102C022EF33E086
:10BA900001E049EF53E00E944B6FF394F394FF826F
:10BAA00020C020E134E03B832A838ACF80913B078A
:10BAB000882309F4D9C080916701882309F494CFC1
:10BAC00081E090913B07911180E024E043E254E053
:10BAD0006D810E94A7BC8981873009F41DC193E064
:10BAE0009F838091B4029091B502A091B602B0916B
:10BAF000B70280931E0790931F07A0932007B0936F
:10BB000021072F813E8123131EC080913B0782179E
:10BB100009F407C1809167018823A9F0EE80E11A3A
:10BB2000FF24F39480913B073E818313F12C8EE137
:10BB300097E00E94A43F00E09C0146EE53E06E2D8A
:10BB40008F2D0E944B6F8F818F5F9E81891316C04E
:10BB500080913B07891709F439C1809167018823D7
:10BB600069F06E81611B81E090913B072E819213F9
:10BB700080E023E047ED53E00E94A7BC8F818E5FF9
:10BB80003E81831316C080913B07831709F42FC1B0
:10BB900080916701882369F06E81611B81E090913B
:10BBA0003B072E81921380E023E04AEC53E00E9491
:10BBB000A7BC8F818D5F3E81831323C080913B079B
:10BBC000831709F425C1809167018823D1F08EEB9A
:10BBD0009CE59F938F938CEB93E09F938F938E8143
:10BBE000811B8F9381E090913B073E81931380E00E
:10BBF0008F930E94C4200F900F900F900F900F9082
:10BC00000F908F818C5F9E81891323C080913B07A9
:10BC1000891709F40BC1809167018823D1F080ED69
:10BC200093E59F938F938DEA93E09F938F938E81FB
:10BC3000811B8F9381E090913B072E81921380E0CE
:10BC40008F930E94C4200F900F900F900F900F9031
:10BC50000F903E813F5F3E838C818313C1CE9F81D5
:10BC60009B5F909339070EC08091220710922207A4
:10BC7000882309F420CF0E947D4280913A078823CF
:10BC800009F419CF2796E2E10C94C7E280912207CC
:10BC900010922207882309F4B4CE26EB35E03093C6
:10BCA000DC062093DB0680913A07882309F4A9CEAD
:10BCB000E9CF81E0913009F080E020E249E154E0F1
:10BCC000622D0E94A7BCA1CE90913B073E819317A5
:10BCD00031F080916701811113C08E8197CE8091E0
:10BCE0002207109222078823A1F32A813B813093F7
:10BCF000DC062093DB0680913A07882351F3C2CFFC
:10BD00006E81611B81E03E81931380E020E246E07A
:10BD100054E00E94A7BCE1CF22E02F83FF24F394DC
:10BD20007DCE8091220710922207882309F4F2CE5B
:10BD30000E944FBD60911E0770911F0780912007E0
:10BD4000909121070E94C7E36B0130923A070E944D
:10BD50000E4F83E08093670186EE93E09093370760
:10BD6000809336072EE137E0309335072093340770
:10BD70001092300710923107109232071092330759
:10BD800040922C0750922D0760922E0770922F0739
:10BD9000F12CE12CC0923D07D0923E07E0923F0784
:10BDA000F09240078AEF9EE490932B1380932A131E
:10BDB00025E430E230932B0720932A0710922907BD
:10BDC00080913A07882309F4A5CE5CCF80912207A1
:10BDD00010922207882309F4C0CE8FEA9CE40E94C7
:10BDE000B1BD80913A07882309F4B7CE4BCF80913B
:10BDF000220710922207882309F4CACE8AEA91E426
:10BE00000E94B1BD80913A07882309F4C1CE3ACF90
:10BE10008091220710922207882309F4D4CEAEDD48
:10BE200080913A07882309F4CECE2CCF8091220747
:10BE300010922207882309F4EECE0E94D0538091FD
:10BE40003A07882309F4E7CE1DCF2E81223009F46A
:10BE50003BCF33E03F8345CE8E81813009F434CF30
:10BE600092E09F835BCFB0E0A0E0E9E3FFE50C94B4
:10BE7000AEE20E94FA20D82F0E945BBDC091380725
:10BE80005C2E85E0682E6C0E9EEBE92E9CE5F92E6B
:10BE90002BE3C22E24E0D22E14E01C1B39EAA32E81
:10BEA00030E4B32E05E00C1B83E0982E9C1A82E050
:10BEB000882E8C1A81E0782E7C1AC11141C08091A5
:10BEC0003B07882361F180916701882361F0652D2C
:10BED000619581E090913B07911180E024E049E772
:10BEE00054E00E94A7BCD111EDC0C43009F0A0C03D
:10BEF00080913B07843009F480C0809167018823DA
:10BF000009F4B6C0FF92EF92DF92CF921F9381E0C7
:10BF100090913B07943009F4A2C080E0A0C08091CA
:10BF2000220710922207882371F20E947D4280919D
:10BF30003A07882341F2CDB7DEB7EFE00C94CAE2AE
:10BF4000C13031F580913B07813099F080916701D4
:10BF5000882361F081E090913B07913009F080E007
:10BF600023E047E654E0672D0E94A7BCD111AAC088
:10BF70007FC08091220710922207882339F387E639
:10BF800099E40E94B1BD80913A078823F9F2D3CF9A
:10BF9000C23009F06FC080913B07823081F0809100
:10BFA0006701882309F48BC081E090913B079230B0
:10BFB00009F080E023E048E554E0682DD5CF80917A
:10BFC000220710922207882351F38FEA9CE40E94F3
:10BFD000B1BD80913A07882311F3ADCF809122073C
:10BFE00010922207882309F44DC00E94D0538091FB
:10BFF0003A07882309F446C09ECF80912207109209
:10C000002207882309F479CFB9DC80913A07882385
:10C0100009F473CF90CF80912207109222078823D2
:10C0200069F00E94A94080913A07882339F083CFB4
:10C03000C530F1F480913B07853069F38091670149
:10C040008823B1F0BF92AF928AE294E09F938F93DE
:10C050000F9381E090913B07953009F05ECF8F936D
:10C060000E94C4200F900F900F900F900F900F9090
:10C0700086E029C0C33009F036CF80913B0783307A
:10C0800009F4ACCF809167018823C9F080ED93E576
:10C090009F938F9389E494E09F938F939F9281E085
:10C0A00090913B07933009F080E08F930E94C42069
:10C0B0000F900F900F900F900F900F9057CFDD23A0
:10C0C00009F4B6CF84E0CF5F6C12F7CE80933907C6
:10C0D00032CFACE3B0E0EFE6F0E60C94ABE2809157
:10C0E0003C07882369F18091821410E000E084FF0E
:10C0F00023C084EB92E10E9441228BE1E4EBF2E168
:10C10000DE01919601900D928A95E1F710E000E032
:10C11000BE016F5F7F4FCE0181960E9407CC18163B
:10C120003CF4CE0101960E947AC6080F111DF0CF93
:10C13000CE0181960E9411241093E8030093E70337
:10C140000E945BBD10913807312E85E0810F8CAFC6
:10C15000212E21948AE8A82E8BE1B82E91E5892E14
:10C1600095E0992E01E0011B26E5622E25E0722E56
:10C17000111113C080913B07882391F180916701D1
:10C18000882359F081E090913B07911180E024E0F1
:10C190004FE555E0622D0E94A7BC8091821486FF76
:10C1A0003EC01130D9F480913B07813049F1809134
:10C1B0006701882309F43EC11F927F926F920F930B
:10C1C00081E090913B07913009F080E08F930E94CD
:10C1D000C4200F900F900F900F900F9082E04FC0EF
:10C1E0008091220710922207882341F20E947D420B
:10C1F00080913A07882311F2EC96E2E10C94C7E2B1
:10C200008091220710922207882389F21092380722
:10C210000E9433CD80913A07882349F2EDCF84FF05
:10C220002DC01130D9F680913B078130D1F080913B
:10C230006701882309F4FEC0BF92AF929F928F924C
:10C240000F9381E090913B07913009F080E08F934C
:10C250000E94C4200F900F900F900F900F900F909E
:10C26000BDCF8091220710922207882301F30E94FC
:10C270008A1B80913A078823D1F2BECF81E090914A
:10C280006701992309F4D7C0582ED12CC12C412E17
:10C290004318852DE090E703F090E803CE14DF0407
:10C2A00008F0C9C05112A5C091E0E91AF108EC18D4
:10C2B000FD0884EB92E10E9441228BE1E4EBF2E184
:10C2C000DE01919601900D928A95E1F7F12CBE0165
:10C2D0006F5F7F4FCE0181960E9407CC18167CF4C9
:10C2E000CE0101960E947AC6882389F3EF106BC0B5
:10C2F000BE016F5F7F4F8EE497E00E9495C6CE012E
:10C3000081960E9411248091821490913B0785FFB1
:10C3100075C0911363C08091220710922207882371
:10C3200009F45CC019821C828091B7126FEC72E133
:10C33000882311F064EB72E121E04EE457E0CE0176
:10C3400001960E941624882309F43FC08BE1FE0168
:10C350003196A4EBB2E101900D928A95E1F78091BC
:10C3600082148F7B80938214A0917814AA3080F479
:10C3700081E08A0F809378148BE18A9FD001112489
:10C38000A659BC4EE4EBF2E101900D928A95E1F7DB
:10C39000CE0101960E9411241092380782E090E0AD
:10C3A000A0E0B0E080933D0790933E07A0933F0745
:10C3B000B093400781E080933A071092920283E0A5
:10C3C0008093670119CFF39482CF0E94F4806EE4CA
:10C3D00077E08BE395E00E9490CEDACF8091670101
:10C3E000882339F081E0911380E041E0642D0E94C0
:10C3F000E5BC8FEFC81AD80A53944BCF911759F068
:10C40000809167018823A9F381E090913B07911304
:10C4100080E040E0EBCF8091220710922207882332
:10C4200079F38FEE9BE40E94B1BD80913A07882397
:10C4300039F3E2CE82E01F5F9CAD911399CE8093D9
:10C440003907DACEFC01A081B1811C92A281B381AF
:10C450008C918F5F8C930280F381E02D90818CE032
:10C46000989F800D1124ECE2F3E113AE84AF0895A0
:10C47000FC0184910895FC0180810895009751F09A
:10C48000FC0180E09191992331F0907C9038D1F3B8
:10C490008F5FF8CF80E00895119800C087FD43C0FA
:10C4A000419800C0119A00C000C0119800C086FDDC
:10C4B00046C0419800C0119A00C000C0119800C049
:10C4C00085FD3BC0419800C0119A00C000C0119882
:10C4D00000C084FD30C0419800C0119A00C000C067
:10C4E000119800C083FD25C0419800C0119A00C07A
:10C4F00000C0119800C082FD1AC0419800C0119A76
:10C5000000C000C0119800C081FD0FC0419800C05C
:10C51000119A00C000C0119800C0419800C0119A43
:10C5200000C000C00895419ABCCF419AF0CF419A13
:10C53000E5CF419ADACF419ACFCF419AC4CF419A01
:10C54000B9CF90E080E00895CF93DF93DB01F9014C
:10C550009C919130C1F0943080F094509C9388303D
:10C56000D1F480819181009771F00197918380834C
:10C57000480F591FEA01188206C08C3539F49C5FB8
:10C580009C93943041F4DF91CF9108958B3339F728
:10C5900081E08C93F8CF20813181B9016F5F7F4FAB
:10C5A00071836083420F531FEA01888380819181E8
:10C5B0008F3591056CF7E7CF0F931F9381E00091C2
:10C5C0007E1410917F142091801430918114409139
:10C5D0007A1450917B1460917C1470917D1404172F
:10C5E00015072607370708F480E01F910F9108957B
:10C5F00090E080E008952091E705833021F425FD47
:10C600000CC024FD0CC030E0A90102C0559547952F
:10C610008A95E2F7CA018170089581E0089580E06B
:10C6200008958091020684FD0BC08091040687FD69
:10C6300007C090910506937081E019F480E0089599
:10C6400081E008952FEB280F2A3108F047C0E22F30
:10C65000F0E08091020690910306A0910406B0914B
:10C66000050604C0B695A795979587952A95D2F7A4
:10C6700080FD02C081700895E851FA4FE081EE23F9
:10C6800041F180915D0790915E07E80FF92FF11D50
:10C69000808190ED980F9A3030F08E3251F4818184
:10C6A00080538A3098F4F093D805E093D70581E061
:10C6B00008958D3211F08B3249F4818190ED980FFD
:10C6C0009A3088F38E3211F48281EACFF0E0E0E014
:10C6D000EACF1092D8051092D705E9CF80E00895EF
:10C6E000CF93DF9385E4AEDF882309F188E04091A2
:10C6F0000206509103066091040670910506972F7B
:10C700009170C92F90E0D92FCC0FDD1F71FB22272C
:10C7100020F930E0220F331F220F331FC22B67FB9B
:10C72000442740F9C42B8C2BDF91CF91089580E0F2
:10C73000DECF88DF882341F081E02091D70530915A
:10C74000D805232B09F480E00895B0E0A0E0EBEADF
:10C75000F3E60C94B4E26B01E9014A3009F4D5C068
:10C76000453109F081C0DB011296ED91FC91F28018
:10C7700096818781139A00C00000E6E2F0E03197CD
:10C78000F0F7092F182FEF2CE29420EFE22230E18E
:10C79000B32EBF0CE80188EF7FDE00C0000086E208
:10C7A00090E00197F0F7BFE1BF1508F49BC08F2D13
:10C7B0008077806871DE8E2D6FDE00C0000086E21B
:10C7C00090E00197F0F780E867DE80E065DE00C06A
:10C7D000000086E290E00197F0F78AEF5DDE00C08E
:10C7E000000086E290E00197F0F7005F1F4F88811C
:10C7F000807F52DE89918295807F4EDEC017D107FF
:10C80000B1F700C0000086E290E00197F0F7F394E2
:10C81000E0E1EE0EFB10BECF1398D6011296ED911B
:10C82000FC9180819281980F92832181921708F068
:10C830009FC194819F5F94839381890F821710F029
:10C840008FEF820F8383458150E0440F551F70E0C6
:10C8500060E0868197810E94E2E481E0CDB7DEB797
:10C86000E9E00C94D0E2DEC1FB0102811381423386
:10C8700009F485C108F48DC1463409F475C1473403
:10C8800009F482C14B3349F789812B81D801129673
:10C890007C91129713963C91213009F4BFC123304B
:10C8A00009F0A0C148EF480F582F91E0341708F461
:10C8B00090E031E0541708F030E0492F432B61E05D
:10C8C000571708F460E0462311F4932331F2FA80FD
:10C8D00030E0F901E95CFD4FD0802D5C3D4FF9015E
:10C8E000E08099C180EE8F0D8068807FD5DD8F2D2F
:10C8F0008295807FD1DD00C0000086E290E0019744
:10C90000F0F780E8C9DD80E861CF0B9A1398399A77
:10C910004198099A119A139A00C0000086E290E0AB
:10C920000197F0F788E790E0CEE9DFE0FE0131976C
:10C93000F1F70197D9F788EFAFDD00C0000086E27C
:10C9400090E00197F0F780E2A7DD80E0A5DD00C070
:10C95000000086E290E00197F0F780E09DDD80E83E
:10C960009BDD00C0000086E290E00197F0F780E0D8
:10C9700093DD80E191DD00C0000086E290E0019748
:10C98000F0F7CE010197F1F7CE010197F1F7CE0153
:10C990000197F1F7CE010197F1F7CE010197F1F779
:10C9A000CE010197F1F7CE010197F1F7CE01019782
:10C9B000F1F7CE010197F1F7CE010197F1F7CE0122
:10C9C0000197F1F7CE010197F1F7CE010197F1F749
:10C9D000CE010197F1F72197F1F780E25DDD80E468
:10C9E0005BDD00C0000086E290E00197F0F780E296
:10C9F00053DD80E651DD00C0000086E290E0019743
:10CA0000F0F7D0E0C0E08C2F8077806845DD8D2F77
:10CA100043DD00C0000086E290E00197F0F780E877
:10CA20003BDD80E039DD00C0000086E290E0019748
:10CA3000F0F78AEF31DD00C0000086E290E0019758
:10CA4000F0F780E2119800C0419800C0119A00C030
:10CA500000C0119800C0419800C0119A00C000C0E9
:10CA6000119800C0419800C0119A00C000C01198F0
:10CA700000C0419800C0119A00C000C0119800C0C9
:10CA8000419800C0119A00C000C0119800C04198A0
:10CA900000C0119A00C000C0119800C0419800C0A9
:10CAA000119A00C000C0119800C0419800C0119AAE
:10CAB00000C000C0119800C0419800C0119A00C089
:10CAC00000C0119800C0419800C0119A00C000C079
:10CAD000119800C0419800C0119A00C000C0119880
:10CAE00000C0419800C0119A00C000C0119800C059
:10CAF000419800C0119A00C000C0119800C0419830
:10CB000000C0119A00C000C0119800C0419800C038
:10CB1000119A00C000C0119800C0419800C0119A3D
:10CB200000C000C000C00000E6E2F0E03197F0F77E
:10CB3000815009F087CF88EFAFDC00C0000086E2AB
:10CB400090E00197F0F7CF5FD05FC03209F05BCF84
:10CB500080E0A2DC80ECA0DC00C0000086E290E077
:10CB60000197F0F7139879CEF8018581888375CE07
:10CB700080E0CDB7DEB7E9E00C94D0E253C0B90154
:10CB8000C8010E9467C369CED80111968C91888331
:10CB900064CE443191F0473109F05FCE1882D8015C
:10CBA00012968C911297898315968C9115978150C6
:10CBB0008A8313968C918B8350CED80115964C9115
:10CBC000159750E0440F551F70E060E016968D9168
:10CBD0009C910E94E2E4F80112828081815083835B
:10CBE00014823BCE381708F438CE871708F435CEB8
:10CBF000FA80E12CD12C243070F46ACEBE01C80139
:10CC00000E9467C3898198819D0D98838E0D8983C9
:10CC1000FF0C09F422CEF7FEF6CFF0CF58E0580F04
:10CC2000482F43CEEF92FF920F931F93CF93DF9342
:10CC3000EC018B017A018A859B858617970731F075
:10CC4000888199810E9454C51B870A87B701888112
:10CC500099810E941DBD2E813F81820F932F911DCE
:10CC60009F838E8390E080E0CDB7DEB7E6E00C9442
:10CC7000D3E2B0E0A0E0EFE3F6E60C94B3E2EC011F
:10CC80007B018A018A859B858617970731F0888109
:10CC900099810E9454C5FB86EA868885998501960C
:10CCA00009F5CC80DA808E81D80EA880B980D501B4
:10CCB0005596ED91FC91C5010995C80E780110E0DB
:10CCC000F70121917F0121111FC08E819F81810F6A
:10CCD000911D9F838E8390E080E0CDB7DEB7EAE0C0
:10CCE0000C94CFE2EE80FF80B801888199810E9488
:10CCF0001DBD8E0D9F2D911D28853985281739075B
:10CD000080F681E090E0E9CF4C2D6D2DC5010E94A9
:10CD1000ACC5D80E180FD4CFB0E0A0E0E2E9F6E63B
:10CD20000C94B6E2EC01D62E1CAD0BAD7C0184E078
:10CD3000E80EF11CE98DFA8DC7010995412F480FC6
:10CD40002D2D602FC7010E94ACC59BAD890F8BAF05
:10CD500081E090E0CDB7DEB7E7E00C94D2E2A6E048
:10CD6000B0E0E5EBF6E60C94ACE27E836D83342E06
:10CD7000FC014080518062807380C301B20120E1D8
:10CD80003EE040E050E00E94F3E149015A01890190
:10CD90008CE3C82ED12CE12CF12CC301B201A701E8
:10CDA00096010E94F3E169837A838B839C83CA0195
:10CDB000B901A70196010E94F3E16B017C013320C8
:10CDC00061F1C301B20120E831E541E050E00E9489
:10CDD000F3E129013A015901DF92CF92C40168E1E0
:10CDE00070E00E9447E29F938F935F924F9289E693
:10CDF00091E29F938F93FE81FF938D818F930E9489
:10CE00005EDB0FB6F894DEBF0FBECDBF88E0FAE060
:10CE10004F165104D8F089E019C081149104D1F45F
:10CE20008A818F9399819F93DF92CF928DE591E2D2
:10CE30009F938F93EE81EF93FD81FF930E945EDBC2
:10CE40000FB6F894DEBF0FBECDBF85E02696E1E1B8
:10CE50000C94C8E20436110568F4DF926F939F9238
:10CE60008F9281E591E29F938F939E819F93ED81B5
:10CE7000EF93E4CFDF926F939F928F9287E491E2DA
:10CE80009F938F939E819F93ED81EF930E945EDB32
:10CE90000FB6F894DEBF0FBECDBF86E0D7CF80912E
:10CEA000D7059091D805009731F04AE050E070E046
:10CEB00060E00C94E6D960E070E0CB0108958091C9
:10CEC000D7059091D805009731F04AE050E070E026
:10CED00060E00C94B9D860E070E0CB010895EFDF1A
:10CEE00097FD0AC0ECDF6F3F71058105910509F0E0
:10CEF0002CF4E5DF862F089580E008958FEF0895E4
:10CF0000CF93C62F16DC882311F0E9DFC82F8C2FB2
:10CF1000CF9108958091D7059091D805892B39F04C
:10CF2000DEDF91E0811101C090E0892F089591E04A
:10CF3000FCCFCF93DF93C82FD62FFBDB882321F0C4
:10CF4000E9DFDF91CF9108958C2F7CDB8111F9CF40
:10CF50008D2FF7CFB4DFCB010895CF93DF93EB0193
:10CF6000E8DB882311F0F6DFEC01CE01DF91CF91F1
:10CF700008950F931F93CF938091D7059091D80573
:10CF80000097D9F0FC018F01C1912C2F2F7D81F0EA
:10CF9000C53411F0C536B9F7F801108270E060E0D1
:10CFA0000E9463D7F801C083CF911F910F9108951C
:10CFB00070E060E00E9463D7F7CF60E070E0CB01E3
:10CFC000F3CFCF92DF92EF92FF926A017B01B1DB48
:10CFD000882319F0CEDF6B017C01C701B601FF90F9
:10CFE000EF90DF90CF900895CF92DF92EF92FF9273
:10CFF000CF93C82F0E94DCC16B017C0124EA30E78B
:10D000004DE75FE3609108017091090180910A0189
:10D0100090910B010E94C5DB87FD18C08AEF90E05C
:10D02000A0E0B0E08C0D9D1DAE1DBF1D809351068C
:10D0300090935206A0935306B0935406C0935C019C
:10D04000CF91FF90EF90DF90CF90089580E090E037
:10D05000DC01E8CFCF9380911206811154C0109269
:10D06000671310926813109269131092351310927F
:10D07000341310923713109236131092391381E043
:10D080008093381382E280933A1310923F131092E8
:10D090003E13E3E5F3E121E633E18FEF81932E17B1
:10D0A0003F07E1F7C1E0C093501325E633EA309320
:10D0B000461320934513C0934713109248131092C0
:10D0C000491390E490934A1310924B1324E633EAE9
:10D0D000309362132093611324E531E030933313CE
:10D0E000209332139EE19093571391E1909358133C
:10D0F0009CE19093551380935413809353130E9493
:10D10000A6C3C093120681E08093110688E891E2DD
:10D11000909377128093761210927912109278126F
:10D1200053985B9A52985A9A3898409A0E941E587F
:10D1300010928C02CF910895FC0180E0309749F065
:10D140009491992331F0907C903809F08F5F31965B
:10D15000F7CF0895B0E0A0E0E0EBF8E60C94B3E27E
:10D16000EC015B018A01FB01099587FD10C0C82E07
:10D17000D12CF12CE12C2196F801C082D182E282DF
:10D18000F382CE01CDB7DEB7EAE00C94CFE2982F60
:10D19000907E903CA9F48F7190E0B0E0A0E06C012B
:10D1A0007D0156E0CC0CDD1CEE1CFF1C5A95D1F71E
:10D1B000CE010196F50109958F73C82A2296DCCF1E
:10D1C000982F907F903E11F58F7090E0B0E0A0E036
:10D1D0006C017D0136E0CC0CDD1CEE1CFF1C3A9589
:10D1E000D1F7CE010196F50109958F73C82A46E063
:10D1F000CC0CDD1CEE1CFF1C4A95D1F7CE0102962B
:10D20000F50109958F73C82A2396B6CF982F987F7A
:10D21000903F79F5877090E0B0E0A0E06C017D016F
:10D2200086E0CC0CDD1CEE1CFF1C8A95D1F7CE01EC
:10D230000196F50109958F73C82A96E0CC0CDD1C88
:10D24000EE1CFF1C9A95D1F7CE010296F5010995C7
:10D250008F73C82A26E0CC0CDD1CEE1CFF1C2A951F
:10D26000D1F7CE010396F50109958F73C82A24964C
:10D2700083CF982F907C903841F4807C803869F47B
:10D280002196CE01F5010995F8CF8E7F8D3F28F0CC
:10D290002196CE01F5010995F8CFC12CD12C76014C
:10D2A0006BCF9CE0899F802D112491E0980F909383
:10D2B00010062CE0280F2093460730E02E5F3F4FEA
:10D2C000409164134217130619F014F080E008959A
:10D2D000209166139217D0F7662341F08E5F0E946B
:10D2E0008BC4809146078E5F0E948BC48091460755
:10D2F00090916413891750F3209166139091100652
:10D30000291720F3109267138093681381E0089522
:10D3100020910F06022E000C330B8217130641F0EA
:10D3200080930F066DEA72E280E393E10C9454C59A
:10D330000895ACE0B0E0EFE9F9E60C94B5E26F3F98
:10D3400071058105910509F070F48CE293E1E4DC4C
:10D35000E0913413F09135133196849190E02C963E
:10D36000E8E00C94D1E2F0906713E090681320910C
:10D37000110621110FC047E251E26E2D8F2D0E9440
:10D3800005C690E080E0F80EF0926713E092681313
:10D390009927E5CFC0903413D090351320E333E1C3
:10D3A0003A8329832F2D30E03C832B832E2D30E0D0
:10D3B0003E832D8318861F822FEF3FEF3A87298700
:10D3C0001C861B8609E316E69E012F5F3F4FAB01CB
:10D3D000BC01C6010E9462A4B60180E393E10E94F1
:10D3E00054C58F819885CFCF4F925F926F927F9275
:10D3F0008F929F92BF92CF92DF92EF92FF920F9304
:10D400001F93CF93DF93CDB7DEB728970FB6F8946D
:10D41000DEBF0FBECDBF7C016A014901FB019081D7
:10D420008CE0989F800D1124982FF7012081822F86
:10D43000880F820F880F80936713909368134115AC
:10D44000510561F1FA82E9827C836B8301111FC06F
:10D45000AE014B5F5F4FB401C6017CDE6C016D8194
:10D460007E818F8198856115710581059105B1F0E7
:10D4700060DFF70180818F5F8083853148F3CE01C3
:10D4800001960E942262E4CFB12C860129C08A0154
:10D49000B12C26C0452846284728B1F728960FB654
:10D4A000F894DEBF0FBECDBFDF91CF911F910F91DA
:10D4B000FF90EF90DF90CF90BF909F908F907F90E4
:10D4C0006F905F904F900895B39407C0B1102DC036
:10D4D00001151105C9F20F5F1F4F01151105A9F2C2
:10D4E000AE014B5F5F4FB401C60134DE6C014D806D
:10D4F0005E806F8078844114510461047104A9F046
:10D50000F0E24F1651046104710401F3D301C2012A
:10D510008D97A109B1090297A105B10530F04BE241
:10D52000441651046104710479F6F7018081482F93
:10D530004B0D5527551F4631510534F0853020F0ED
:10D54000CE0101960E94226281E0411451046104DF
:10D55000710409F480E0B80EF70180818B0D80839F
:10D56000BB2009F497CFBA94AE014B5F5F4FB40173
:10D57000C801F0DD8C016D817E818F819885D9DEB7
:10D58000EFCFCF93DF93FC0125AD211104C021E043
:10D5900025AF0E94A6C3C0913213D0913313E091FE
:10D5A0006113F091621382E00995E0916113F091AB
:10D5B000621381E0099530E020E044E1BE0180E3A0
:10D5C00093E10E94A1C323E633E147E1BE0180E37A
:10D5D00093E10E94A1C3E0916113F091621380E096
:10D5E0000995DF91CF9108954F925F926F927F924C
:10D5F0008F929F92AF92BF92CF92DF92EF92FF9263
:10D600001F93CF93DF9300D000D0CDB7DEB70E9439
:10D61000DCC16B017C0180915C018F3FC1F10E94F4
:10D62000DCC18090510690905206A0905306B090B5
:10D630005406681979098A099B0997FD28C08091C9
:10D640000413909105138F5F8F70891701F1E0919A
:10D650005C01E53008F054C024E0E29FF0011124A1
:10D66000E55CFD4F80819181A281B38189839A839A
:10D67000AB83BC8320E030E0A901BE016F5F7F4F28
:10D6800082E791E00E94B6B78FEF80935C010E9421
:10D690001E5880918D0282FF3CC0809160068111EE
:10D6A0003AC091E09093600680915F07892780934C
:10D6B000220710925F0783E08093670110928D022A
:10D6C0000E94DCC16C507E4F8F4F9F4F60938E0243
:10D6D00070938F02809390029093910268E873E1B7
:10D6E00082E090E00E946C4016E01150A1F00E9490
:10D6F000104062E070E080E090E00E9450C1F5CF01
:10D700008091680190916901A0916A01B0916B01CB
:10D71000ADCF1092600680915C0690915D06A0915D
:10D720005E06B0915F06A7019601281B390B4A0BD4
:10D730005B0BDA01C901B7FF05C080919202882313
:10D7400009F4B9C1D701C6018C599F4FAF4FBF4FE4
:10D7500080935C0690935D06A0935E06B0935F068F
:10D7600060918C02062E000C770B77FF03C0719539
:10D770006195710990918C0280915B06981365C048
:10D78000633008F062C010928C0280918C0280930A
:10D790005B06643008F069C0809122078111E7C000
:10D7A00080912A1390912B13835A954741F48091CD
:10D7B0005D01882309F4EDC0815080935D010E94D2
:10D7C000F92B8090790790907A07A0907B07B09012
:10D7D0007C0781110E94062CD501C4013AE0B69560
:10D7E000A795979587953A95D1F7009741E0A407BB
:10D7F000B10520F08FEF9FEFA0E0B0E09695879500
:10D80000209167012111D7C030919202311180C15E
:10D8100080912A1390912B13835A954709F45FC185
:10D820008091930281115BC18091570690915806B7
:10D83000A0915906B0915A06C81AD90AEA0AFB0AF9
:10D84000F7FC5BC10E94E84158C1633009F09DCFED
:10D8500080918C0287FD07C081E0880F880F80933C
:10D860008C0264E092CF8FEFF8CF8091450721E0E2
:10D8700030E040E050E0882309F456C08090410732
:10D8800090904207A0904307B09044078114910400
:10D89000A104B104E9F170E090E080E00E94C9DBEE
:10D8A00020E030E040E85EE30E942ADC2B013C01EE
:10D8B000C701B601681979098A099B090E94C9DB69
:10D8C0009B01AC01C301B2010E945AE320E030E0A9
:10D8D0004AE754E40E942ADC4B015C0120E030E07E
:10D8E00040EA52E40E9446E424E630E040E050E0A2
:10D8F00087FF12C020E030E040EF51E4C501B401E1
:10D900000E9446E42AE030E040E050E087FF04C097
:10D9100021E030E040E050E0C0924107D092420761
:10D92000E0924307F0924407A0918C020A2E000C6B
:10D93000BB0B0E94A5E224E030E040E050E00E94F2
:10D940006EE280913D0790913E07A0913F07B09114
:10D950004007820F931FA41FB51F80933D0790932C
:10D960003E07A0933F07B093400710928C02D70167
:10D97000C6018856954CAF4FBF4F80935706909382
:10D980005806A0935906B0935A0681E08093670128
:10D9900007CF8CE080935D018091550690915606EB
:10D9A000009729F00197909356068093550681E0E1
:10D9B0008093670104CF009741F040915506509144
:10D9C00056064817590708F023CF8091920281111B
:10D9D00011C0223038F0243008F43FC0243011F454
:10D9E000109267018CE293E1CCDD81E080933C07EB
:10D9F0008093920283E08CDC81E080935013E0916D
:10DA00002A13F0912B13099510923C0780919202F2
:10DA1000811127C01092220780912A1390912B1315
:10DA2000835A954709F0FCCE0E94DCC1DC01CB0192
:10DA30008C199D09AE09BF09809055069090560635
:10DA4000B12CA12C88169906AA06BB0608F0E0CED8
:10DA50009093560680935506DBCE81E08093670154
:10DA6000C1CF80E393E10E9424C591E0811101C000
:10DA700090E090939202882369F280912A1390910A
:10DA80002B13835A9547B9F40E94DCC1DC01CB010A
:10DA90008C199D09AE09BF09C0905506D090560655
:10DAA000F12CE12CC816D906EA06FB0620F4909367
:10DAB0005606809355060F900F900F900F90DF91B0
:10DAC000CF911F91FF90EF90DF90CF90BF90AF90DC
:10DAD0009F908F907F906F905F904F90089548E94E
:10DAE000C40E4AE3D41EE11CF11CC0925706D0922A
:10DAF0005806E0925906F0925A06809192028111DE
:10DB0000DACF809167018130B1F610926701D3CFEF
:10DB1000009709F46FCF51CFACE0B0E0E2E9FDE649
:10DB20000C94B5E2F0906713E09068132091110611
:10DB3000211112C047E051E26E2D8F2D0E9405C6C3
:10DB400090E080E0F80EF0926713E0926813992756
:10DB50002C96E8E00C94D1E2C0903413D0903513A9
:10DB600020E333E13A8329832F2D30E03C832B835C
:10DB70002E2D30E03E832D8318861F827A87698799
:10DB80001C861B8609E316E69E012F5F3F4F48E384
:10DB900052E6BC01C6010E94F7A4B60180E393E1FE
:10DBA0000E9454C58F819885CDCFA4E0B0E0EBED05
:10DBB000FDE60C94B1E27C01062F5A01122F862F4C
:10DBC000660F990B9C01215D3D4F690186E0882E0F
:10DBD000912C11160CF03DC0AE014F5F5F4F68E312
:10DBE00072E6C701B7DA7C0169817A818B819C81F9
:10DBF000611571058105910561F16D33710581052F
:10DC0000910509F450C06E3771058105910509F43D
:10DC10004AC06A3271058105910501F507FF11C0FF
:10DC20008EE791E20E3F11F08AE791E236E01302AF
:10DC3000B001112471DF66E070E00E945BE2161B08
:10DC400060C065E470E080E090E073DB115069F53E
:10DC500010E0812F2496ECE00C94CDE26432710543
:10DC60008105910571F4A114B104D1F0E6E01E0222
:10DC7000B0011124C50150DFB4010E945BE2161B04
:10DC8000A8CF603471058105910551F41150F6015A
:10DC90006081062E000C770B880B990B4ADB99CF1D
:10DCA00048DB115096CF07FDBBCF61E089819A8197
:10DCB000AB81BC81CD97A105B10509F460E0600F8F
:10DCC0006A30A4F01150862F6AE00E943AE2092FD0
:10DCD000682F880F770B605D7F4F072E000C880B35
:10DCE000990B27DB112309F4B3CF602F062E000C0C
:10DCF000770B605D7F4F072E000C880B990B19DBAB
:10DD00001150112309F4A4CF86E01802B0011124A8
:10DD1000C70102DF66E070E00E945BE2161B99CF4C
:10DD2000ECE2F3E183AF64AF6FEF7FEFCA01F4CEB3
:10DD3000ACE0B0E0EEE9FEE60C94B5E2F0906713DB
:10DD4000E090681320911106211112C047EE50E2B5
:10DD50006E2D8F2D0E9405C690E080E0F80EF092A7
:10DD60006713E092681399272C96E8E00C94D1E2AF
:10DD7000C0903413D090351320E333E13A832983E4
:10DD80002F2D30E03C832B832E2D30E03E832D83DE
:10DD900018861F827A8769871C861B8609E316E628
:10DDA0009E012F5F3F4F4BE352E6BC01C6010E942C
:10DDB000F7A4B60180E393E10E9454C58F81988552
:10DDC000CDCF6FEF7FEFB4CFB0E0A0E0EAEEFEE69C
:10DDD0000C94B3E25C016B01AFD9E82EC6010E943E
:10DDE0003E62F12C03E110E0081B1109C5E20E159B
:10DDF0001F050CF4CFE18C2F90E09C012E5F3F4F6C
:10DE0000409164134217130609F08CF5099720918D
:10DE10006613281719065CF140914807509149078D
:10DE20006091470710926713C093681325E1C501FD
:10DE3000BCDED1E0C114D104A9F06AE370E080E057
:10DE400090E077DA0E151F05A4F4C45F8091641387
:10DE5000C81740F0209166134C2F4950550B2417DA
:10DE600015064CF4CDB7DEB7EAE00C94CFE2D0E073
:10DE7000E1CFDD23B9F3802F880F080F000F009347
:10DE80006713C093681360E270E080E090E051DABD
:10DE9000C60197DFE7CFACE0B0E0E1E5FFE60C9428
:10DEA000B1E2982F862F6A017901B02E692FF9D936
:10DEB000882309F487C010911106C701002371F16E
:10DEC0003BD9A82E8090341390903513111142C085
:10DED0002FEF3FEF122F23E12A194091480750916D
:10DEE000490760914707C60160DEAA2009F46AC0AD
:10DEF000B6E08B9F600111246AE370E080E090E05F
:10DF000018DA57E0C516D10408F442C060E270E0A8
:10DF100080E090E00EDAC81AD90AF3CF0E943E6280
:10DF2000A82E8090341390903513112389F2FE01AE
:10DF300033968AE0DF011D928A95E9F780E393E149
:10DF40009A83898302E116E69E012F5F3F4F4BE3E0
:10DF500052E612C0FE0133968AE0DF011D928A95D7
:10DF6000E9F780E393E19A83898302E116E69E0153
:10DF70002F5F3F4F48E352E6B701C4010E94F7A468
:10DF8000B40180E393E10E9454C52F813885A2CF6C
:10DF900040914607212F30E0A6E0AA9EC00111243F
:10DFA0002E5F3F4F281739070CF49C0180E8821B35
:10DFB0008093671340936813BB2041F06FEF7FEFAE
:10DFC000C701AADD2C96ECE00C94CDE2C701F9DE86
:10DFD000F9CF0C947DA54F925F926F927F928F92B2
:10DFE0009F92BF92CF92DF92EF92FF920F931F9377
:10DFF000CF93DF9310920706109206062FE320932B
:10E000000A06109209061092080610920206109253
:10E01000030610920406109205069C01F9019081F6
:10E020002F5F3F4F9032D1F39E34C9F4818190ED40
:10E03000980F9A3020F08D3211F08B3281F43296A5
:10E040009F012F5F3F4F808180538A3008F46DC05D
:10E050009F012F5F3F4F8081803209F468C0F093A9
:10E060005E07E0935D078F010F5F1F4FC0816AE27B
:10E0700070E0C8010E94FCE4009731F0FC01319788
:10E0800080818032E1F31182CD3421F0C43511F06A
:10E09000C734D9F5F80180810F5F1F4F8032D1F36B
:10E0A00080538A3090F5C0930A0690E080E06AE0E1
:10E0B000AF014F5F5F4F689F9001699F300D112442
:10E0C000C901C0972081820F911D27FD9A95FA0101
:10E0D000208120532A3060F390930906809308062C
:10E0E000DF0131962C912032D9F3CD3461F58E3198
:10E0F000910539F0F0F48731910519F08C319105D3
:10E1000011F5B0930706A0930606DF91CF911F91FA
:10E110000F91FF90EF90DF90CF90BF909F908F90E6
:10E120007F906F905F904F900895F90189CFF9012A
:10E130008FCF8537910538F08737910510F3803AF6
:10E1400013E09107F1F280905D0790905E0740E048
:10E1500050E0BA0130E020E0C12CD12C7601C3940C
:10E16000FD013196DC91DD2309F484C0D132F1F454
:10E17000CD34E1F480329105C9F440930206509306
:10E1800003066093040670930506F0930706E09378
:10E19000060663E270E0CF010E94FCE4009709F4F8
:10E1A000B4CFFC011082B1CFDF01DACFD154DA3124
:10E1B00008F05BC0DF011D91103291F0A0EDA10FBE
:10E1C000AA30E8F01E3271F4A181A053AA30B8F051
:10E1D0002115310519F49F0121503109B12C13C0CB
:10E1E000FD01E8CF1D3211F01B3291F7A181B0ED96
:10E1F000BA0FBA3020F0AE3259F7A281E6CFBE2E68
:10E20000B818309759F3AD2FB0E02601370104C09C
:10E21000440C551C661C771CDA95D2F74429552905
:10E2200066297729A851BA4FBC92A081A154AA317E
:10E2300008F4BACFDF01D191DD2309F491CF00EDCD
:10E24000B02EBD0E19E01B15A8F713EDB12EBD0EB3
:10E2500011E01B1578F7DB3269F3FD013196DC9193
:10E26000D03209F07DCFDF01F8CF21153105E9F675
:10E270009D01DBCF309307062093060640930206EC
:10E280005093030660930406709305063ECFFC018D
:10E29000659175918591949108958F929F92AF9217
:10E2A000BF92CF92DF92EF92FF92CF93DF93EC0178
:10E2B0008090B4029090B502A090B602B090B702E0
:10E2C00020E030E0A901C501B4010E94C5DB88232C
:10E2D00009F452C0C880D980EA80FB80A70196016A
:10E2E000C501B4010E94C5DB18160CF04AC020918C
:10E2F000D3053091D4054091D5055091D605C7017D
:10E30000B6010E94C5DB882321F1C092D305D092CB
:10E31000D405E092D505F092D6052091CF05309135
:10E32000D0054091D1055091D205C701B6010E9498
:10E330002ADC9B01AC0160E070E080E89FE30E9472
:10E34000E2E26093490170934A0180934B019093FC
:10E350004C016091490170914A0180914B0190916B
:10E360004C01DF91CF91FF90EF90DF90CF90BF9065
:10E37000AF909F908F90089560E070E080E89FE3F9
:10E38000F0CF60E070E0CB01ECCF682F70E090E060
:10E3900080E00C9420A5B0E0A0E0E1EDF1E70C9462
:10E3A000ADE2EC012091AC023091AD024091AE02A1
:10E3B0005091AF02688179818A819B810E94E2E25B
:10E3C0004B015C012091B0023091B1024091B20248
:10E3D0005091B3026C817D818E819F810E94E2E227
:10E3E0006B017C01A5019401609141017091420192
:10E3F00080914301909144010E94C5DB882309F478
:10E4000054C08092410190924201A0924301B09287
:10E4100044012091C7053091C8054091C90550912C
:10E42000CA05C501B4010E942ADC2B013C010E94EF
:10E43000F3E34B015C0120E030E040EA50E40E944D
:10E44000C5DB181634F4812C912CC0EAAC2EC0E444
:10E45000BC2E20E030E0A901C501B4010E9446E4D1
:10E4600087FF03C0812C912C5401A5019401C301A5
:10E47000B2010E94E2E26093BF057093C0058093F1
:10E48000C1059093C205C501B4010E94C2E3609327
:10E49000BD05062E000C770B6F5F7F4F6630710550
:10E4A00014F066E070E06093BB05D0913F011091DD
:10E4B000BD05A701960160914501709146018091CB
:10E4C0004701909148010E94C5DB811123C0D113FF
:10E4D00075C02091A3053091A4054091A5055091E8
:10E4E000A6056091BF057091C0058091C10590910E
:10E4F000C2050E942ADC2091A7053091A805409111
:10E50000A9055091AA050E94E3E2CDB7DEB7E0E18C
:10E510000C94C9E2C0924501D0924601E0924701B5
:10E52000F09248012091CB053091CC054091CD056A
:10E530005091CE05C701B6010E942ADC4B015C0157
:10E540000E94F3E36B017C0120E030E040EA50E4FC
:10E550000E94C5DB181634F4C12CD12CB0EAEB2E86
:10E56000B0E4FB2E20E030E0A901C701B6010E9413
:10E5700046E487FF03C0C12CD12C7601A701960188
:10E58000C501B4010E94E2E26093C3057093C40523
:10E590008093C5059093C605C701B6010E94C2E3EA
:10E5A0006093BE05062E000C770B6F5F7F4F6630C1
:10E5B000710514F066E070E06093BC05C091BE0583
:10E5C000D11305C0809140018C1709F470C080916F
:10E5D000BD059091BE059093400180933F010C2EA4
:10E5E000000CDD0B27E01203C0011124FC01EC0F2D
:10E5F000FD1FEE0FFF1FEE0FFF1FE753FD4F2081A2
:10E600003181428153812093B7053093B8054093FF
:10E61000B9055093BA050091BC05002E000C110BF2
:10E62000FC01E00FF11FEE0FFF1FEE0FFF1FE7537E
:10E63000FD4F60817181828193810E94E2E260934B
:10E64000B3057093B4058093B5059093B6052091FA
:10E65000BB0537E02303F0011124CE0FDF1FCC0FE1
:10E66000DD1FCC0FDD1FC753DD4F288139814A8163
:10E670005B812093AF053093B0054093B105509373
:10E68000B205E00FF11FEE0FFF1FEE0FFF1FE75364
:10E69000FD4F60817181828193810E94E2E26093EB
:10E6A000AB057093AC058093AD059093AE0580905B
:10E6B000C3059090C405A090C505B090C6052091F3
:10E6C000B3053091B4054091B5055091B605C5012B
:10E6D000B4010E942ADC2091B7053091B805409121
:10E6E000B9055091BA050E94E3E26B017C01C0922A
:10E6F000A705D092A805E092A905F092AA0520915D
:10E70000AB053091AC054091AD055091AE05C5010A
:10E71000B4010E942ADC2091AF053091B0054091F0
:10E72000B1055091B2050E94E3E2A70196010E9453
:10E73000E2E26093A3057093A4058093A5059093EE
:10E74000A605C7CEACE0B0E0E8EAF3E70C94BAE285
:10E75000182F882379F020E030E0A9016091B902F8
:10E760007091BA028091BB029091BC020E94C5DBFD
:10E770008823F1F08091B8028117D1F00E942529F9
:10E780008CE0E3E2F2E0DE01119601900D928A95B1
:10E79000E1F7CE010196FFDD8091B802882361F098
:10E7A00082E791E00E947B291092B8020E94203CEF
:10E7B0002C96E3E00C94D6E281E08093B80282E7E5
:10E7C00091E00E944729F2CFCF92DF92EF92FF9221
:10E7D00080E0B8DF1092B0021092B1021092B20243
:10E7E0001092B3021092AC021092AD021092AE02DF
:10E7F0001092AF021092BD021092BE021092BF02A0
:10E800001092C0021092B9021092BA021092BB028A
:10E810001092BC0249EC52E027E0C12CD12C60ECF4
:10E82000E62E6FE7F62E90E080E0FC01EE0FFF1F72
:10E83000EE0FFF1FE40FF51FC082D182E282F38248
:10E8400001968730910589F72150445E5F4F211171
:10E85000EACFFF90EF90DF90CF9008954F925F92B4
:10E860006F927F928F929F92AF92BF92CF92DF92E0
:10E87000EF92FF921F93CF93DF93EC01162F20911D
:10E88000B4023091B5024091B6025091B70268814E
:10E8900079818A819B810E94C5DB882309F497C016
:10E8A000B090B80280E04EDFC880D980EA80FB805B
:10E8B00020E030E0A901C701B6010E9446E487FFCD
:10E8C00003C0C12CD12C7601C092B402D092B50203
:10E8D000E092B602F092B7022DEB37E346E855EB33
:10E8E000C701B6010E94C5DB87FD0BC02DEB37E3E6
:10E8F00046E855E3C701B6010E9446E418160CF03D
:10E9000076C0A701960160E070E080E89FE30E9476
:10E910005AE36093CF057093D0058093D10590930F
:10E92000D20580EF9FEFA9E7B4EC8093D3059093D5
:10E93000D405A093D505B093D605BB2009F447C0F4
:10E940004090720150907301609074017090750155
:10E950008090760190907701A0907801B090790135
:10E96000C0907A01D0907B01E0907C01F0907D0115
:10E9700081E0E8DE112359F1A30192016091720157
:10E980007091730180917401909175010E94C5DBB3
:10E9900081111BC0A50194016091760170917701EE
:10E9A00080917801909179010E94C5DB81110DC0A1
:10E9B00020917A0130917B0140917C0150917D0141
:10E9C000C701B6010E94C5DB81110E94463CDF9160
:10E9D000CF911F91FF90EF90DF90CF90BF90AF90BD
:10E9E0009F908F907F906F905F904F90089560E020
:10E9F00070E0CB018ECF8F929F92AF92BF92CF9259
:10EA0000DF92EF92FF92C090B902D090BA02E090EC
:10EA1000BB02F090BC0220E030E0A901C701B601C2
:10EA20000E94C5DB8823E1F1A701960160E070E058
:10EA300080E89FE30E945AE36B017C018090BD0255
:10EA40009090BE02A090BF02B090C00220E030E0E3
:10EA5000A901C501B4010E94C5DB882329F1A501E4
:10EA6000940160E070E080E89FE30E945AE3C09266
:10EA7000C705D092C805E092C905F092CA05609317
:10EA8000CB057093CC058093CD059093CE05FF9078
:10EA9000EF90DF90CF90BF90AF909F908F900895B0
:10EAA000C12CD12C7601CACF60E070E0CB01DFCF62
:10EAB000CF92DF92EF92FF926B017C0183E3C81645
:10EAC000D104E104F10470F082E3C81AD108E1082E
:10EAD000F10862E370E080E090E00E9450C10E9483
:10EAE000FF25ECCFC701B6010E9450C10E94FF254F
:10EAF000FF90EF90DF90CF900895BC0190E080E010
:10EB00000C9420A580915B07813069F0909182146C
:10EB100092FB882780F992FF07C097FB882780F92E
:10EB200091E08927089581E008959091821494FBE3
:10EB3000882780F994FF06C081E090919C12911182
:10EB400001C080E00895ACE0B0E0E9EAF5E70C949C
:10EB5000ADE2109245078091220710922207882388
:10EB600061F020E040E070E060E080EC95E50E941C
:10EB7000AC402C96E0E10C94C9E220911001309158
:10EB8000110140913D0750913E07CA01820F931F2A
:10EB90002436310509F0E9C34730510544F00697A2
:10EBA0008A3091050CF0F0C38AE090E0F7C3069636
:10EBB0004A3F5F4FACF380913C07882309F4D0C1F2
:10EBC0006091881270918912072E000C880B990BA6
:10EBD0000E94CBDB11E0209184123091851240918C
:10EBE0008612509187120E9446E418160CF010E02D
:10EBF0001093500680907A0190907B01A0907C0148
:10EC0000B0907D0120E030E0A901C501B4010E946F
:10EC1000C5DBC12CD12CE0EAEE2EE0ECFE2E87FD08
:10EC200006C0C12CD12C70EAE72E70E4F72E20E04C
:10EC300030E04AE754E4C501B4010E942ADCA70190
:10EC400096010E94E3E22DEC3CEC4CEC5DE30E946B
:10EC50002ADC0E94C2E36B017C0180E2F7FE09C05E
:10EC6000F094E094D094C094C11CD11CE11CF11C20
:10EC70008DE2409072015090730160907401709029
:10EC80007501209176013091770140917801509182
:10EC9000790129873A874B875C878093940260E2E9
:10ECA00030E1C31637E2D306E104F1048CF0C7016A
:10ECB000B60120E137E240E050E00E946EE2CA0176
:10ECC000B9012AE030E040E050E00E946EE2605D71
:10ECD0006093950260E248EEC41643E0D406E10476
:10ECE000F1048CF0C701B60128EE33E040E050E0BB
:10ECF0000E946EE2CA01B9012AE030E040E050E033
:10ED00000E946EE2605D60939602C701B60124E640
:10ED100030E040E050E00E946EE26AE0862E912CE6
:10ED2000A12CB12CCA01B901A50194010E946EE287
:10ED3000605D60939702C701B601A50194010E942E
:10ED40006EE26B01CA01B901A50194010E946EE255
:10ED5000CC2009F433C32EE220939802605D6093C7
:10ED6000990250E3C50EC0929A0264E972E088E409
:10ED700096E00E9407E520E030E0A901C301B2015E
:10ED80000E94C5DB20E030E040E05FEB87FD04C07F
:10ED900020E030E040E05FE3C301B2010E94E3E223
:10EDA0000E94C2E3CB010E94F03EBC0183E496E0E6
:10EDB0000E9407E520E030E0A90169857A858B850E
:10EDC0009C850E94C5DB20E030E040E05FEB87FDE2
:10EDD00004C020E030E040E05FE369857A858B8500
:10EDE0009C850E94E3E20E94C2E3CB010E94F03EB8
:10EDF000BC018EE396E00E9407E58091821400E159
:10EE000017E283FD28C091DE882309F4E9C28091CE
:10EE10007A1490917B14A0917C14B0917D1400978A
:10EE2000A105B10509F4DCC2BC01CD01615F784DDB
:10EE30008F4F9F4F20E137E240E050E00E94F3E126
:10EE400060917E1470917F14809180149091811450
:10EE50000E94F3E189010E94463E4B015C018D82D4
:10EE60009E82AF82B886D62E80915B018017C1F159
:10EE700000935B01C80164E670E00E9447E27B01F9
:10EE800088E48E9DB0018F9D700D112490E080E08C
:10EE90000E94C9DB2AE037ED43E25CE30E942ADCF2
:10EEA0000E94C7E360933D060115110509F09BC25E
:10EEB0001092380610922E0680E880932D0688E383
:10EEC00096E0FC0101900020E9F7CF0188539640BD
:10EED000982F990F890F880F90E8981B90932C0614
:10EEE00080915A01D816E1F180925A0141E08D815A
:10EEF0009E81AF81B88580389145A140B10508F465
:10EF000040E06CE176E0CE0105960E94AF66982F56
:10EF1000990F990F891B880F805880931B06282D05
:10EF20002370822EE9F401151105A9F0A0E1B7E2E2
:10EF3000A01BB10B2D813E814F8158850E9415E2A7
:10EF4000980150E040E00E94F3E1211531054105B0
:10EF5000510509F06EC210922E0680E880932D06AE
:10EF60000E94DCC10091140610911506209116062E
:10EF7000309117066B017C01C01AD10AE20AF30A2C
:10EF80009701860137FD11C020911306209520932B
:10EF900013066A547C4F8F4F9F4F609314067093F3
:10EFA00015068093160690931706D090130611E06D
:10EFB000D11001C010E081E00E9488698091641343
:10EFC000873180F480916613843060F03BE3E32E58
:10EFD00032E2F32E03E126E044E069E080E393E1CE
:10EFE0000E942AC6809164138431B8F4809166131C
:10EFF000823098F0DD2009F435C280917D078823A6
:10F0000009F430C285E092E27C0102E123E042E0B3
:10F0100068E680E393E10E942AC6809164138C31F4
:10F0200008F06EC040908412509085126090861255
:10F0300070908712A0908812B0908912843198F451
:10F0400080916613883078F08091500680FF0DC261
:10F0500087EB91E27C010CE022E048E064E480E38D
:10F0600093E10E942AC680916413883040F4B7FE71
:10F07000FFC14BE951E267E082E40E94906E80910B
:10F0800064138C31B0F480916613843190F020E0E9
:10F0900030E040E05FE3C301B2010E94E3E20E947E
:10F0A000C2E377FF0EC24BE951E26CE182E40E94B9
:10F0B000906E809164138C3118F5809166138431C1
:10F0C000F8F080917D078823D9F024E6829FC00163
:10F0D000112481589F4F6FEF70E00E945BE2CB01DB
:10F0E0000E946F3F27E6209367132CE1209368135B
:10F0F0000E94E16E65E270E080E090E00E94996914
:10F1000014DD882379F180916413843358F580915C
:10F1100066138A3238F107E028E04AE26AE280E3C7
:10F1200093E10E94D1C405E022E04CE262E380E377
:10F1300093E10E94D1C424E04AE061E38AE20E94A4
:10F14000A1C4609132137091331382E380934C1306
:10F150008BE280934D132CE433E142E380E393E1AF
:10F160000E94A1C380916413853350F4809166138B
:10F17000813330F024E04AE461E386E30E94A1C4D5
:10F1800080916413843368F480916613823348F06D
:10F1900002E020913D0642E367E380E393E10E94B1
:10F1A000D1C480916413803358F5809166138832FE
:10F1B00038F180911A06811751F080911906109349
:10F1C0001A068F5F833008F0A5C1809319068091DD
:10F1D00019068111A2C180913806882389F0809197
:10F1E0002C068093671380E38093681388E396E08E
:10F1F0000E94E16E65E270E080E090E00E94996913
:10F2000080916413883208F05DC0809166138D315F
:10F2100008F458C02BE040E86DE180E00E94A1C4F2
:10F2200080916413873208F04DC0809166138F314E
:10F2300008F448C083E08093671306E200936813E4
:10F2400068E570E080E090E00E9499698BE080932F
:10F25000671300936813DD2009F491C183E496E0FD
:10F260000E94E16E88E28093671306E200936813C0
:10F2700069E570E080E090E00E94996980E3809306
:10F28000671300936813DD2009F49EC18EE396E0B6
:10F290000E94E16E8DE48093671306E20093681389
:10F2A0006AE570E080E090E00E94996985E58093CE
:10F2B000671300936813DD2009F4ABC188E496E07E
:10F2C0000E94E16E80916413833348F58091661348
:10F2D0008B3228F183E00E94886983E08093671372
:10F2E00003E30093681366E070E080E090E00E9422
:10F2F000996981E00E9488698091100190911101C3
:10F300000E946F3F2CE020936713009368130E94C4
:10F31000E16E65E270E080E090E00E949969809182
:10F320006413813408F025CC80916613863308F489
:10F3300020CC109267138EE38093681385E190E1EF
:10F340000E943E62082F863108F088C185E190E175
:10F350000E94E16E053109F40CCC60E270E080E0BF
:10F3600090E00E9499690F5FF5CF243631054CF487
:10F370008536910504F58A30910534F48AE090E0F1
:10F3800009C084369105BCF0883EE3E09E0714F086
:10F3900087EE93E02817390709F40DCC90931101FB
:10F3A0008093100110923D0710923E0710923F0784
:10F3B0001092400700CC84E690E0F0CF662351F035
:10F3C0002EE220939802605D6093990280E2809320
:10F3D0009A02CBCC80E28093990280939802F6CF78
:10F3E00010E000E038CD2E2D80E2243628F08E2D5E
:10F3F00064E60E942EE2805D8093980290E22A30BB
:10F4000040F03AE0822F632F0E942EE20E942EE20B
:10F41000905D90939902822F6AE00E942EE2905DA7
:10F4200090939A0268E972E088E396E00E9407E50B
:10F4300046CD29833A834B835C8381E02038314574
:10F440004140510508F480E0482F6EE276E0CE019D
:10F4500001960E94AF66982F990F990F891B880F0C
:10F4600080587CCD8FEC91E2CFCD8FE991E2F2CD47
:10F47000C5010E946F3FFC01808193E0803229F436
:10F48000818192E0803209F491E0892F880F880F02
:10F49000E92EE81A8E2D855B8093671387E08093B1
:10F4A000681323E030E0291B3109CF01820F931F3D
:10F4B0000E94E16E69E070E080E090E00E9499694E
:10F4C000DECDCB010E946F3FFC01808193E0803252
:10F4D00029F4818192E0803209F491E0892F880F2C
:10F4E000880FF92EF81A8F2D855B809367138CE1B6
:10F4F0008093681323E030E0291B3109CF01820F8C
:10F50000931F0E94E16E69E070E080E090E00E944D
:10F510009969CFCD109219065ACE8230B1F48091FC
:10F520002E06882391F048E951E260E386E30E94C9
:10F53000906E80912D068093671380E3809368130B
:10F540008EE296E00E94E16E5BCE80911C068823DD
:10F5500009F456CE86E38093671300E300936813A3
:10F560006FEF7FEF85E991E20E948C6D80911B0621
:10F5700080936713009368138CE196E0E3CF87E0F4
:10F580000E94493780FF15C023E4E22E26E0F22EC8
:10F59000F70161917F01662309F464CE6F320CF0AC
:10F5A0006FE3062E000C770B880B990B0E9499696C
:10F5B000EFCF80914B0780FD51CE6FEF7FEF80E959
:10F5C00091E20E948C6D4ECE87E00E94493781FF08
:10F5D00015C09EE3E92E96E0F92EF70161917F01B7
:10F5E000662309F457CE6F320CF06FE3062E000C41
:10F5F000770B880B990B0E949969EFCF80914B078D
:10F6000081FD44CE6FEF7FEF80E991E20E948C6D27
:10F6100041CE87E00E94493782FF15C088E4E82E7A
:10F6200086E0F82EF70161917F01662309F44ACE46
:10F630006F320CF06FE3062E000C770B880B990BE2
:10F640000E949969EFCF80914B0782FD37CE6FEF13
:10F650007FEF88E891E20E948C6D34CE809118068D
:10F660001817B1F0009114101093180685E190E17D
:10F670000E943E62081708F050C00F5FE02FF0E0D4
:10F68000EB5EFF4E8081807C8038B9F300931410CC
:10F69000E0901410F12C97012B5E3F4E7901C901C7
:10F6A0000E943E62182F60E870E0C7010E94986EC9
:10F6B000153108F05ECA60E270E080E090E00E94E0
:10F6C0009969143109F455CA60E270E080E090E075
:10F6D0000E949969133109F44CCA60E270E080E03D
:10F6E00090E00E949969123109F443CA212F30E059
:10F6F0002E5F3F4F4AEF4203B001439F700D11242C
:10F7000060587F4F85E190E10E94986E60E270E062
:10F7100080E090E00E9499692CCA10921410B8CF32
:10F7200080915B07823059F000DA882349F080919C
:10F73000821482FB882780F991E08927089581E06F
:10F74000089581E008959091C00095FFFCCF8093CB
:10F75000C6000895CF93DF93EC018991882311F0BF
:10F76000F2DFFBCFDF91CF910895CF93DF93EC01D0
:10F770008991882311F0E7DFFBCF8DE0E4DF8AE099
:10F78000E2DFDF91CF910895CF93DF93EC01FE018B
:10F7900084912196882311F0D6DFF9CFDF91CF91A4
:10F7A0000895CF93DF93EB01EFDFCE01D3DFDF913D
:10F7B000CF9108950F931F93CF938C01C62F84E0B0
:10F7C0009FE1E2DFC801E0DF8AE3BDDF80E38C0F69
:10F7D000BADF8AE0B8DFCF911F910F910895CF92E1
:10F7E000DF92EF92FF926A017B01CEDF42E0C70118
:10F7F000B6010E94C7A7FF90EF90DF90CF900895C9
:10F80000EEDF8AE0A0CFAEE4B0E0E9E0FCE70C94E4
:10F81000ABE270E060E085E40E94AD679AA789A73B
:10F8200081117CC26EEB70E083E50E94AD673C0104
:10F8300065E070E083E40E94AD678C0160E085E5DF
:10F840000E9499678DAF60E08AED90E20E94EC50D3
:10F850000E94DCC169877A878B879C8780916401CD
:10F86000909165010E976816790654F08BE890E246
:10F870008BDF0E9454B8C25BDF4FE2E10C94C7E219
:10F8800029853A854B855C85205E314B4F4F5F4F14
:10F890002BAB3CAB4DAB5EAB87E790E275DF0E94D4
:10F8A0005B258FE780938A1281E08093660160E098
:10F8B00083E690E20E94EC5089859A85AB85BC85F1
:10F8C000898B9A8BAB8BBC8B8BA79CA7ADA7BEA754
:10F8D000198E1A8E1B8E1C8E19A21AA21BA21CA294
:10F8E00019821A821B821C822FE730E040E050E030
:10F8F0002D873E874F87588B80E090E4ACE1B6E4DB
:10F900008D839E83AF83B8871D8A1E8A1F8A188EB7
:10F91000FFE7CF2ED12CE12CF12C2F961FAE2F9785
:10F920001FA618AA19AA1AAA1DA21EA21FA218A6CB
:10F9300091E09FAB312C212C812C912C540193010F
:10F94000072C000C440B550B22962CAF3DAF4EAF4D
:10F950005FAF2297402F002E000C550B5CAF4BAFD2
:10F96000C3014E969C01092E000C440B550B2696A4
:10F970002CAF3DAF4EAF5FAF2697CC979C01990F50
:10F98000440B550B2A962CAF3DAF4EAF5FAF2A9775
:10F9900036E0631A7108C301072C000CAA0BBB0BDD
:10F9A0002E968CAF9DAFAEAFBFAF2E978091660104
:10F9B000882309F48DC00E94DCC12B013C01109109
:10F9C0009803112309F473C00E94C625109298036E
:10F9D0008090841290908512A0908612B090871229
:10F9E000A50194016D897E898F89988D0E9446E4D6
:10F9F00087FF04C08D8A9E8AAF8AB88EA5019401C4
:10FA00006D817E818F8198850E94C5DB181624F454
:10FA10008D829E82AF82B88622966CAD7DAD8EAD12
:10FA20009FAD22970E94CBDB6D8F7E8F8F8F98A327
:10FA30009FA92D8D3E8D4F8D58A1992309F472C138
:10FA4000C501B4010E9446E418168CF5D301C20129
:10FA500029893A894B895C89821B930BA40BB50BCE
:10FA6000AC01BD01485853416109710977FD1FC0C0
:10FA70004D855E856F8578894C195D096E097F0912
:10FA8000759567955795479540938A128DA39EA3C8
:10FA9000AFA3B8A78D8D9E8DAF8DB8A18D8B9E8B9A
:10FAA000AF8BB88F49865A866B867C861FAA2696AE
:10FAB0006CAD7DAD8EAD9FAD26970E94CBDBA501D1
:10FAC00094010E94C5DB87FF21C08CED9FE15CDEC5
:10FAD000109266010E945B25CCCE4BEEC42ED12C39
:10FAE000E12CF12C76C124E130E040E050E02D879C
:10FAF0003E874F87588B34E1C32ED12CE12CF12C5B
:10FB000076C1CD86DE86EF86F88A71C1D301C20147
:10FB10002BA53CA54DA55EA5821B930BA40BB50B95
:10FB2000B7FD47C089A50E94D0248AE00CDED3012E
:10FB3000C2018053984FAF4FBF4F8BA79CA7ADA773
:10FB4000BEA72F969FAD2F9791116FC02FA538A9F3
:10FB500049A95AA9C501B4010E9446E418160CF03F
:10FB600050C020E030E040E050E4C501B4010E9404
:10FB7000E3E26FA778AB89AB9AABA3019201205E59
:10FB8000314B4F4F5F4F2BAB3CAB4DAB5EAB2E962B
:10FB90006CAD7DAD8EAD9FAD2E970E94CBDBA501E8
:10FBA00094010E94C5DB881F8827881F2F968FAF7E
:10FBB0002F9789859A85AB85BC858D8F9E8FAF8F5A
:10FBC000B8A329893A894B895C89281739074A07DC
:10FBD0005B0720F42D8F3E8F4F8F58A38D8D9E8D08
:10FBE000AF8DB8A1481A590A6A0A7B0A91E84916EA
:10FBF0009FE4590692E16906710460F18EEB9FE182
:10FC000066CFD301C2012BA93CA94DA95EA9821BD5
:10FC1000930BA40BB50B41E254E160E374E1B7FD33
:10FC2000C8CF80E00E946A25C4CF2A966CAD7DAD16
:10FC30008EAD9FAD2A970E94CBDB9B01AC01C50125
:10FC4000B4010E94C5DB87FFB4CF4CE35EE26CE4F5
:10FC50007EE2E7CFABADBCADA215B3050CF05BC047
:10FC6000B3E02B1631040CF456C081E69FE18CDD25
:10FC700084E49FE189DD49815A816B817C818DE536
:10FC80009FE1BEDD84E49FE17FDD49A15AA16BA124
:10FC90007CA189E59FE1B4DD84E49FE175DD498DB8
:10FCA0005A8D6B8D7C8D85E59FE1AADD2DAD2223DC
:10FCB00009F4DFCD89819A81AB81BC8180938B125D
:10FCC00090938C12A0938D12B0938E122CEA35EC87
:10FCD00047E25EE369A17AA18BA19CA10E942ADC84
:10FCE00060938F127093901280939112909392125E
:10FCF00020E030E543EC50E4698D7A8D8B8D9C8D4E
:10FD00000E942ADC60939312709394128093951250
:10FD100090939612AECD0E94F46A48CE86EB90E2A4
:10FD200033DDA9CDC501B4010E94C5DB87FFBFCE7D
:10FD3000D301C20129853A854B855C85821B930BD3
:10FD4000A40BB50BAC01BD014858534161097109C1
:10FD500077FDADCE2114310409F4FCC02DA13EA1E4
:10FD60004FA158A5280F391F4A1F5B1F298B3A8BBB
:10FD70004B8B5C8B2DA13EA14FA158A5281B390BA5
:10FD80004A0B5B0BC701B6010E94E4E129893A895D
:10FD90004B895C890E946EE2CD84DE84EF84F88812
:10FDA000C20ED31EE41EF51E34E1C316D104E104D5
:10FDB000F1040CF498CE4CEEC416D104E104F10425
:10FDC0000CF08BCE50E8C516D104E104F1040CF41C
:10FDD00098CECD86DE86EF86F88A8EEF90E0A0E0A2
:10FDE000B0E08C199D09AE09BF096C017D018BE55E
:10FDF00090E2CADC6D857E858F8598890E94E96FC7
:10FE000086E590E2C1DCC701B6010E94E96F4D8131
:10FE10005E816F8178858FE490E2E1DC4D895E89B7
:10FE20006F89788D88E490E2DADC33E023163104C0
:10FE30000CF490C0C701B6010E94CBDB20E030E09B
:10FE400040E850E40E942ADC69837A838B839C8398
:10FE50002D813E814F8158856D897E898F89988D4E
:10FE60000E94E2E22BED3FE049EC5FE30E942ADCD6
:10FE70009B01AC0169817A818B819C810E945AE34C
:10FE80006FAB78AF89AF9AAF69897A898B899C8982
:10FE90000E94CBDB2FE632E143E85AE30E942ADCE2
:10FEA0006D837E838F8398872AE939E949E15FE38F
:10FEB0006FA978AD89AD9AAD0E942ADC69837A83F7
:10FEC0008B839C839B01AC010E94E3E22D813E81E8
:10FED0004F8158850E945AE369A37AA38BA39CA300
:10FEE00020E030E040E05EE36D817E818F81988587
:10FEF0000E942ADC29813A814B815C810E942ADCA4
:10FF0000698F7A8F8B8F9C8F4FA958AD69AD7AAD71
:10FF100082E490E264DC4D815E816F8178858CE3C0
:10FF200090E26EDC8DE290E22FDC49815A816B8198
:10FF30007C8187E290E253DC49A15AA16BA17CA1AC
:10FF400081E290E24CDC498D5A8D6B8D7C8D8BE18A
:10FF500090E256DC8D859E85AF85B8898C0D9D1D00
:10FF6000AE1DBF1DB595A7959795879580938A126D
:10FF70004CAD4F930F933F922F9287E090E29F9367
:10FF80008F9322E130E23F932F931F920E94CF5034
:10FF90005FEF251A350A0FB6F894DEBF0FBECDBF4E
:10FFA0002D8D3E8D4F8D58A12D833E834F835887D5
:10FFB000498A5A8A6B8A7C8A1FAB79CD67E778E1D8
:10FFC0000E940BB860914F0D7091500D8091510DB2
:10FFD0009091520D0E94C9DBAB01BC018EE698E105
:10FFE000FEDB40917F0D5091800D6091810D7091ED
:10FFF000820D8BE698E1F3DB4091830D5091840DE7
:020000021000EC
:100000006091850D7091860D88E698E1E8DB40915E
:10001000610750916207609163077091640785E6FC
:1000200098E1EECBCF93DF936BE178E10E940BB8C0
:10003000CFE3DDE04CA95DA96EA97FA982E198E13B
:10004000CEDB48AD59AD6AAD7BAD8FE098E1C7DB43
:100050004CAD5DAD6EAD7FAD88E698E1D1DBDF9153
:10006000CF910895CF93DF9367EF77E10E940BB8AC
:10007000CFE3DDE04CA15DA16EA17FA18EEE97E103
:10008000AEDB48A559A56AA57BA58BED9CE2A7DB55
:100090004CA55DA56EA57FA588ED9CE2A0DB48A9D7
:1000A00059A96AA97BA985ED9CE2AADBDF91CF91D2
:1000B0000895CF93DF9362ED77E10E940BB8CFE311
:1000C000DDE0688179818A819B810E94C9DBAB0177
:1000D000BC0189EC97E183DB6C817D818E819F81FE
:1000E0000E94C9DBAB01BC018BED9CE278DB68852B
:1000F00079858A859B850E94C9DBAB01BC0188EDAF
:100100009CE26DDB6C857D858E859F850E94C9DBB9
:10011000AB01BC0185ED9CE273DBDF91CF910895CB
:100120008F929F92AF92BF92EF92FF920F931F9385
:10013000CF93DF938AEF96E127DBC0E0D7E0D15081
:1001400019F080E200DBFBCF8C2F0E94C571CF5FDE
:10015000C730A1F78AE0F7DA09EC12E0C0E080E2EC
:10016000F2DA8C2F0E94C5717801D7E080E2EBDAD9
:10017000F70180809180A280B38020E030E0A90167
:10018000C501B4010E9446E487FD02C08BE2DBDAC0
:1001900043E0C501B4010E94C7A7D150FCE1EF0EB6
:1001A000F11CD111E3CF8AE0CEDACF5F0C5F1F4F95
:1001B000C730A9F68AE0C7DADF91CF911F910F917E
:1001C000FF90EF90BF90AF909F908F900895811116
:1001D00005C083EF96E1D8DA8AE0B5CA87EF96E1E9
:1001E000FACF8CEE96E1D0CA86EE96E1CDCACF93D7
:1001F00084E50E949963C0E08823D9F00E946F676C
:10020000C82F1816B4F4F0DF8DE49DDA809108064B
:10021000909109060E947D7584E099E1B5DA6C2F12
:10022000CC0F770B880B990B0E947DA58AE08BDAA7
:10023000CFEF8C2FCF910895CF93C82F6BED78E13E
:100240000E94F4B7C11101C0CFDF40918B125091D1
:100250008C1260918D1270918E1282ED98E1BFDA4E
:1002600020E030E543EC50E460918F1270919012E1
:1002700080919112909192120E942ADCAB01BC01F4
:100280008FEC98E1ACDA2CEA35EC47E25EE3609162
:1002900093127091941280919512909196120E94EF
:1002A0002ADCAB01BC018CEC98E199DA8AE04BDAEC
:1002B000CF910895CF93DF93EB0166DABE01DD0F96
:1002C000880B990B0E947DA5DF91CF9108955CDA90
:1002D0008AE039CACF93DF9365E17FE10E940BB8D2
:1002E000C091FF12D0910013488159816A817B81AE
:1002F0008CE09FE174DA4C815D816E817F818BEDB2
:100300009CE26DDA4091FB125091FC126091FD125B
:100310007091FE1288ED9CE262DA89E09FE134DAA6
:100320008BE29BE0D4DFDF91CF910895EC018B014C
:10033000F42E0E945B25209709F477C055DFCE018B
:10034000C6DF0115110511F406E11CE20E942A68BE
:100350001F930F93DF93CF9386EB96E19F938F9339
:1003600081E08F930E94CF500E94E841C0913113E9
:10037000C695C6958CE293E10E94C16ADC2FDD0F21
:100380001D2F1C0F8DB79EB707960FB6F8949EBF12
:100390000FBE8DBF83E00E94886910926713C093DF
:1003A000681385E190E10E94E16E10926713D0938B
:1003B00068136FEF7FEF87EA96E10E948C6D1092D1
:1003C0006713109368136FEF7FEF8AE996E10E943D
:1003D0008C6D80E393E10E9424C58111DBCF01DFA6
:1003E00086EC96E1D1D989EE93E0019739F000C00F
:1003F0000000EEE5F9E03197F0F7F7CFF89489EED9
:1004000093E0019739F000C00000E6EEF3E0319789
:10041000F0F7F7CF0E945B25FF2021F00E94C22752
:10042000A895FECF0E947D27FBCF0115110511F481
:1004300006E11CE2CDEBD6E189CF8091890D909148
:100440008A0D2FEF3FEF981751F0E92FF0E0E757B3
:10045000F24F228130E09F5F9F7790938A0DC90110
:1004600008951F920F920FB60F9211240F900FBE96
:100470000F901F9018951F920F920FB60F92112494
:100480000BB60F922F938F939F93EF93FF939091BF
:10049000C60020918A0DE091890D81E08E0F8F7743
:1004A000281729F0F0E0E757F24F9283E82FE09306
:1004B000890DFF91EF919F918F912F910F900BBE1E
:1004C0000F900FBE0F901F9018958EBD0DB407FEB4
:1004D000FDCF08958FEF8EBD0DB407FEFDCF8EB515
:1004E0000895909164009B7F90936400982F906A88
:1004F00096959CBD80FD03C091E0863009F490E0A4
:100500009DBD0895A8E0B0E0E8E8F2E80C94ABE205
:10051000B82E8091720E843008F0F4C131E6D32EEB
:100520008091720E843008F01FC18091890D9091E6
:100530008A0D891B8F7709F417C17FDF97FF09C0E8
:1005400050DE86EE95E120D98091890D80938A0D49
:10055000E7CF8A3019F08D3009F0FDC01092710E8E
:1005600080910F0E9091100EFC01E55FF14F168205
:10057000892B19F40E94FF25D3CF1092100E1092F0
:100580000F0E01E11EE0F8018191803209F446C0AE
:100590008E3409F09CC061EE75E1C8010E9444DB15
:1005A0007C01892B41F06EE470E0C80104960E9442
:1005B000FCE4009709F4C8014AE050E070E060E014
:1005C00001960E94B9D82B013C0180910B0E9091AD
:1005D0000C0EA0910D0EB0910E0E0196A11DB11D35
:1005E000481659066A067B0629F060E08EEA95E116
:1005F000EF2851F16AE270E0C8010E942BE59C01EE
:10060000009729F1982F901BF12C992349F09150D4
:10061000F801E90FF11D8081F826F7CF8F01B3CFE4
:100620004AE050E070E060E0C90101960E94B9D84C
:100630002F2D30E050E040E06217730784079507E4
:1006400051F060E08FE895E10E9487B769CF60E0E4
:1006500085E695E1F9CF40920B0E50920C0E609218
:100660000D0E70920E0E80911D078130D9F467E453
:1006700070E0C8010E94FCE40097A1F04AE050E05D
:1006800070E060E001960E94B9D862307105810582
:10069000910540F484EC94E177D860E08AEB94E132
:1006A0000E94EC50F80180818D3481F58381823382
:1006B00009F445C0883301F1803341F581818433E9
:1006C00029F58281813311F50E94223C1FC080915F
:1006D000821480FFC8CF6FEB7BE2C8010E9444DB2D
:1006E000009731F0FC01838180538A3008F0BBCF42
:1006F00060E08BE395E1A8CF8281803339F481817A
:10070000813321F41092660110925F078091110EDF
:100710008B3309F405CF8091720E843008F000CF3E
:100720008091740E8D9DC001112461E17EE08B5893
:10073000914F0E9407E580E00E9447B7F1CE828189
:10074000813321F78181813309F741E070E060E076
:1007500089E89AE1EBDD2FE03EE041E15EE061E710
:100760007EE00E94A462DCCE8091821483FDCAC028
:1007700082FFC8C087FDC6C01A82198281E6F82EA2
:1007800094E0E92E29E6D22E8091720E843008F092
:10079000B9C00E94DC628111B5C041E050E0BE01E9
:1007A0006D5F7F4F89E992E10E9429CB0B8110E0B8
:1007B000019711F00FEF1FEF8091A1129091A212FB
:1007C000A091A312B091A41280937E1490937F14F1
:1007D000A0938014B09381140E94DC620F3F100735
:1007E00041F4811106C0FDDC8EEF95E10E94C47BCF
:1007F000CBCF4091740E242F30E00A3061F00D30E1
:1008000051F0882309F470C089819A81009719F00A
:1008100001969A8389831092950589819A81F29E27
:10082000F001F39EF00D1124EE58F14FDF01A80FF7
:10083000B91F13961C92892BA9F50E94FF250E94CF
:10084000DC62882309F4A0CF89E992E10E94122199
:10085000809179148823F1F18150809379148D9DD2
:10086000C001112462E08B59994F0E94E0CEE091C3
:10087000791424E0E29FF0011124EF59F94F4081EF
:1008800051816281738140937E1450937F146093F1
:1008900080147093811489E992E10E942ECA0E940B
:1008A00071C672CF1A82198283818D3479F4848162
:1008B000823361F48581853349F4868180538A309F
:1008C00028F0809182148B7F8093821481E00E94B3
:1008D00047B7B5CF0E9463C6809182148860809329
:1008E0008214E0921D0750CF4F9DA00111244B5858
:1008F000514F9E012F5F3F4F65E975E0802F0E94A9
:10090000A46242CF0E94DCC16B017C01BB2041F09C
:10091000C0920B06D0920C06E0920D06F0920E06E5
:100920008091E3059091E405A091E505B091E6057D
:100930000097A105B10529F140910B0650910C06D5
:1009400060910D0670910E06840F951FA61FB71FAC
:10095000A7019601281B390B4A0B5B0BDA01C90171
:10096000B7FD0FC03EDC60915D0770915E078DE0C2
:1009700096E10E9490CE40E070E060E090E080E080
:10098000E9CE80914E0190914F01A0915001B0911C
:100990005101892B8A2B8B2B79F090910413809134
:1009A0000513981709F4C4C0C0920B06D0920C0628
:1009B000E0920D06F0920E0680919A0590919B05AB
:1009C000A0919C05B0919D0546015701881A990A8E
:1009D000AA0ABB0AD501C401B7FDC0C19091041396
:1009E0008091051320913D01981709F4D5C0E0913D
:1009F00005133BE5E39FF0011124EC51F84F808192
:100A0000281799F080933D010E94DCC1B0903D0110
:100A10000B2D10E084E00E94A8A70115110509F034
:100A2000BEC060E084E00E94F4C0809197038823F8
:100A300009F487C10091060110910701C8010297CE
:100A40002091881230918912281739070CF479C146
:100A5000809005138C82812C912C54018091041379
:100A60002C81821709F4FDC0822F90E03BE5389F6E
:100A7000F001399FF00D1124E257F84F458956894E
:100A80006789708D452B462B472B81F4418D528D04
:100A9000638D748D452B462B472B41F4458D568D28
:100AA000678D70A1452B462B472BE9F14BE5489FFD
:100AB0009001499F300D1124C9018257984F1C01A4
:100AC000FC0161817281838194810E947FE46D8346
:100AD0007E838F839887F10161A172A183A194A184
:100AE0000E94C9DB2B013C01F10165A176A187A120
:100AF00090A50E94C9DB9B01AC01C301B2010E9419
:100B00005AE32D813E814F8158850E942ADC2B01BA
:100B10003C01AC019B01C501B4010E9446E487FF82
:100B200002C0530142018C818F5F8F708C8396CFFE
:100B3000BB2019F010929E053FCF0E94DCC10091AE
:100B40000B0610910C0620910D0630910E06809038
:100B50004E0190904F01A0905001B0905101080DAE
:100B6000191D2A1D3B1D601B710B820B930B97FDFA
:100B7000E1CF80919E0581111FCF81E080939E057A
:100B800080E00E94922781E00E94922782E00E94EA
:100B900092270E947D2710CF80917D0731CF0F3F94
:100BA000110511F461E03ECFEAEFFBE2E491E15080
:100BB000EA3008F051C0F0E0E052FA470C948AE2C3
:100BC000EA85EF85F485FE852C862C8608861086BE
:100BD0001886228684B5806884BDB7BC26CF84B5CC
:100BE000806284BDB8BC21CF8091800080688093F2
:100BF0008000109389000093880017CF80918000B7
:100C000080628093800010938B0000938A000DCF48
:100C10008091B00080688093B000B092B30005CF9F
:100C20008091B00080628093B000B092B400FDCE9D
:100C300080919000806880939000109399000093B9
:100C40009800F3CE80919000806280939000109382
:100C50009B0000939A00E9CE003811050CF0A2CF5A
:100C6000E0CEB801110F880B990B0E94CBDB2B0152
:100C70003C0120910001309101014091020150910D
:100C80000301C501B4010E942ADCA30192010E9464
:100C9000E3E24B015C010091040110910501AC01FC
:100CA0009B01C301B2010E9446E418168CF0B80102
:100CB000012E000C880B990B0E94CBDB2B013C0111
:100CC000A50194010E94C5DB181614F42401350116
:100CD0008090960590909705A0909805B090990502
:100CE000A3019201C501B4010E9446E41816D4F490
:100CF00020E037ED43EA5CE3C301B2010E942ADC45
:100D00002B013C0128E431EE4AE75FE3C501B40161
:100D10000E942ADC9B01AC01C301B2010E94E3E204
:100D20002B013C01409296055092970560929805E0
:100D300070929905C301B2010E94C2E3CB010E94E7
:100D40001DC2F4E6CF0ED11CE11CF11CC0929A0525
:100D5000D0929B05E0929C05F0929D050E94FF2594
:100D600080911D07882309F4D2C010913E011130F3
:100D700061F18091821480648093821481E0809379
:100D80003E0164EF71E080E090E00E9458750E949F
:100D900033CD8091821484FFCFC0123028F460E0FC
:100DA0008AE496E10E94EC5083E0809367010E9400
:100DB000DCC16C597F4F8F4F9F4F60935C067093DF
:100DC0005D0680935E0690935F060E94DCC16B0116
:100DD0007C0110914D011123F1F08091600788236F
:100DE000D1F040919F055091A0056091A1057091AF
:100DF000A20546015701841A950AA60AB70AB50149
:100E0000A40177FD1AC0833009F492C00CF083C0AE
:100E100081300CF087C0212F30E0A8EEB3E00E94B3
:100E20001FE2C60ED71EE81EF91EC0929F05D09283
:100E3000A005E092A105F092A2050E9410400E9438
:100E4000F46A8091E205882379F10E94DCC16B018C
:100E50007C018091DE059091DF05A091E005B091C5
:100E6000E105A7019601281B390B4A0B5B0BDA0140
:100E7000C901B7FD19C02091E20530E0A8EEB3E04A
:100E80000E941FE2C60ED71EE81EF91EC092DE05A4
:100E9000D092DF05E092E005F092E10580E00E944B
:100EA000D0248AE00E94A37B8091DD05882379F11C
:100EB0000E94DCC16B017C018091D9059091DA051B
:100EC000A091DB05B091DC0546015701881A990A0B
:100ED000AA0ABB0AD501C401B7FD19C02091DD05DE
:100EE00030E0A8EEB3E00E941FE2C60ED71EE81E57
:100EF000F91EC092D905D092DA05E092DB05F09296
:100F0000DC050E9434A886E093E10E94C42628965E
:100F1000E2E10C94C7E2843009F07DCF65D989E520
:100F200096E103C061D988E896E10E94C47B73CF43
:100F30005BD981E796E1F9CF112309F446CF34CF8D
:100F4000A2E1B0E0E6EAF7E80C94ACE290913E0D45
:100F500093FD7EC0082F4BD9182F87FD79C089E4F7
:100F60000E949963882309F48BC00E946F67282F21
:100F700030E01216130614F421E030E0220F331F84
:100F8000220F331FF901EF53FD4F80819181198AA0
:100F90000E941DC280918812909189128635910518
:100FA00074F0002381F00E94933E0DC082E50E9400
:100FB0009963882309F46CC00E94AA67E9CF0E9454
:100FC000DB3E0E9454B86091881270918912072EFE
:100FD000000C880B990B0E94CBDB2091841230917E
:100FE000851240918612509187120E9446E418168D
:100FF00044F0298984E29FE1222329F049894A8B20
:1010000048C08FE29FE19F938F938AE39FE19F9374
:101010008F931F920E94CF500F900F900F900F90C0
:101020000F9031E03A8B35C060E070E0CB014FC0EB
:10103000C701B6010E94C5DB87FF0EC08091660123
:10104000882321F0109266010E9454B830929703D1
:101050006296E1E10C94C8E24601570100E098C0B5
:101060008FE30E94A37BCFC020E030E040E450E457
:101070000E9446E418160CF004C12601370101C194
:1010800083E50E949963898B811196CF01118ECFE0
:101090001A8A83E50E949963882331F00E94AA6727
:1010A000909307018093060182E40E94996388234C
:1010B00031F00E94AA67909305018093040186E4B1
:1010C0000E942263882309F4AFCF0E94B96760931E
:1010D0000001709301018093020190930301332476
:1010E000339420E030E0A9010E94C5DB811101C0EA
:1010F000312C30929703002309F4AACF5A89552343
:1011000009F4A6CF1092970381E0809366011D82B7
:101110001E821F82188619861A861B861C8680E00E
:101120009CE3ACE1B6E48D879E87AF87B88B812CBA
:10113000912C90E8A92E9FEBB92E00E0412C512C68
:1011400032016091881270918912072E000C880B71
:10115000990B0E94CBDB6B017C01A50194010E94DD
:10116000C5DB8823A9F0209184123091851240912B
:10117000861250918712998991115ACFC701B601F1
:101180000E94C5DB082F001F0027001F46015701E2
:101190000E94DCC16B017C01DC01CB0129853A8511
:1011A0004B855C85821B930BA40BB50BB7FD2EC042
:1011B000D701C60188519C4FAF4FBF4F89879A878F
:1011C000AB87BC87812F0E94D02480E49FE10E94DE
:1011D000C47B411451046104710409F441CFC3017B
:1011E000B201605F784D8F4F9F4F6C197D098E095A
:1011F0009F0928EE33E040E050E00E94F3E1CA018D
:10120000B9010E94E96F8AE00E94A37B80E07AD94D
:101210000E94DCC160930B0670930C0680930D0650
:1012200090930E062091841230918512409186127F
:101230005091871229833A834B835C83C501B401A3
:101240000E94E2E29F77411451046104710409F0A5
:101250000BCF20E030E040E85FE30E94C5DB87FF72
:1012600010C03A89412C512C3201332331F085E0F2
:10127000482E8DE0582E612C712C4C0C5D1C6E1C80
:101280007F1C0023C1F18D819E81AF81B885892BA0
:101290008A2B8B2B61F0D701C6012D813E814F81B6
:1012A0005885821B930BA40BB50BB7FD24C0298175
:1012B0003A814B815C816D857E858F8598890E94FE
:1012C000E2E220E030E040EC5FE30E94C5DB87FD16
:1012D000B5CED701C601805A9541AF4FBF4F8D8320
:1012E0009E83AF83B88729813A814B815C812D87AA
:1012F0003E874F87588B80916601882309F49ECEE4
:10130000411451046104710461F030E1C31A37E201
:10131000D30AE108F108C418D508E608F708F7FE73
:101320008DCE1A8A0ECFA1E4B0E0E9E9F9E80C9479
:10133000ABE222968FAF2297209160072CA781E025
:101340008093600780910A068D3409F4F1C48435D6
:1013500011F40C94F49D873491F4809108069091D7
:1013600009068D31910509F462C308F0E5C18430A6
:10137000910509F406C330F4029708F45FC20E9495
:1013800082CED7C28531910509F4D3C24C97B9F703
:1013900087E00E944937811111C080910206909127
:1013A0000306A0910406B0910506FEE0B695A79548
:1013B00097958795FA95D1F780FDBBC20E942529A4
:1013C000109213016091B8028CE40E949967382E44
:1013D00080E00E94A2730E94DCC160930B067093B0
:1013E0000C0680930D0690930E060E94CF3A81E082
:1013F0008093D8060E940C3DC0900206D090030650
:10140000E0900406F0900506E9E1F694E794D7949D
:10141000C794EA95D1F7C0FE0DC081E00E9449371C
:10142000182F82E00E94493711110C94319E11E06F
:10143000811101C010E08091020690910306A091F5
:101440000406B091050677E1B695A795979587951F
:101450007A95D1F780FF02C00C94179E1111CBC270
:101460008091020690910306A0910406B0910506B2
:101470003B2F3170A32E3113C0C28C2D8170A12E51
:101480008113BBC211E0AA24A394BB24B39482E5C8
:101490000E949963882309F4B4C20E94B9676C8FD3
:1014A0007D8F8E8F9F8F20E030E0A9010E94C5DBE9
:1014B000882359F0111105C0A11003C0BB2009F405
:1014C00028C1CE014C960E9477B8112309F489C037
:1014D000AA2009F483C01092720110927301109235
:1014E000740110927501109276011092770110929A
:1014F0007801109279010E94203C85EE96E00E94CE
:1015000047716B017C0189EE96E00E9447712B01C7
:101510003C01AC019B01C701B6010E9446E41816CC
:101520000CF074C2A7019601C301B2010E945AE3F4
:101530009B01AC010E942ADC20E030E040E85FE340
:101540000E94E3E20E947FE421E030E048E452E4BC
:101550000E942ADC69837A838B839C8380917A0141
:1015600090917B01A0917C01B0917D0188A399A30A
:10157000AAA3BBA320E030E040EC5FE3C301B201CB
:101580000E942ADC2B013C0177FA709477F8709462
:1015900020E030E040EC5FE3C701B6010E942ADCA6
:1015A0009058DE0111966D01E8A0F9A00AA11BA1D7
:1015B000A30192010E94EE3A0E94103E1092720125
:1015C00010927301109274011092750110927601BD
:1015D00010927701109278011092790180E00E94B8
:1015E0006854AA2019F081E00E946854BB2009F4D5
:1015F00090C083E00E94643781118BC00E94203C20
:1016000020917A0130917B0140917C0150917D01C4
:1016100028A339A34AA35BA32093A8023093A9026D
:101620004093AA025093AB02A090FF12B090001317
:10163000D501CD90DD90ED90FC90A701960160E082
:1016400070E080EE92E40E94E2E22B013C014092C5
:101650009C0250929D0260929E0270929F02F50140
:1016600084809580A680B780A501940160E070E039
:1016700080EE92E40E94E2E26CA37DA38EA39FA37E
:101680006093A0027093A1028093A2029093A302A0
:101690002DE030E044EE52E4C501B4010E9446E47E
:1016A00018160CF4B8C12EE030E042EE52ECC50141
:1016B000B4010E94C5DB87FDAEC12DE030E04EEEE7
:1016C00052E4C701B6010E94C5DB18160CF4A3C191
:1016D0002EE030E042EE52ECC701B6010E9446E433
:1016E00087FD99C119821A821B821C829E012F5F7D
:1016F0003F4F6901E8A0F9A00AA11BA12CA13DA1BF
:101700004EA15FA1C301B2010E94EE3A82E00E94A5
:1017100068540E94203C8091D7068093D8063320DD
:1017200019F081E00E94A2730E94B63A83E0809390
:1017300067010E94463CFDC08A35910509F4E9C263
:1017400050F58E31910509F475C18A9709F017CECD
:1017500080911D07833008F4ECC089E40E949963EE
:10176000082FF12C882319F00E94AA67F82E8AE42A
:101770000E949963E82E882309F4C9C10E94AA67D0
:10178000182F0111C7C1173008F4CAC185E599E1C6
:101790000E94C47BCEC08B35910509F4BDC28C3547
:1017A000910509F0ECCD5FE2252E52E0352E62E77F
:1017B000E62E61E0F62EC12CD12C10E0D1018D91E6
:1017C0001D010E949963082F882351F10E94B96777
:1017D0002B013C01F70120813181428153810E941C
:1017E000E2E24B015C012DEB37E346E855EB0E944A
:1017F000C5DB87FD0AC02DEB37E346E855E3C5019D
:10180000B4010E9446E418165CF4133011F0C02EA7
:101810000D2DD7014D925D926D927C921397D02E33
:101820001F5FB4E0EB0EF11C143041F6CC2009F43C
:1018300077C20E94203C0E94463C7BC080911D07DD
:10184000833008F476C0ACE9CA2EA2E0DA2EB2E703
:10185000EB2EB1E0FB2E10E088E5810F0E9499632A
:10186000882309F472C00E94B9674B015C01812F83
:101870000E94FB62882359F0D7012D913D914D9133
:101880005C91C501B4010E94E3E24B015C01F601E9
:1018900080829182A282B3821F5FF4E0CF0ED11CBE
:1018A00024E0E20EF11C1330B9F685E40E9499633E
:1018B000882309F455C00E94B9676B017C0183E05D
:1018C0000E94FB62882371F020917E0130917F019C
:1018D0004091800150918101C701B6010E94E3E26D
:1018E0006B017C01C092A802D092A902E092AA02E8
:1018F000F092AB0240E050E0BA0186E40E94E1675A
:1019000020E030E0A9010E9446E4181684F40E9409
:10191000B96729E838E848E85CE30E942ADC60936C
:101920000C0170930D0180930E0190930F010E94A2
:10193000A73722969FAD2297911102C00E9441B80D
:10194000ACA5A09360070C943095F701808191813C
:10195000A281B381F60180839183A283B3839CCF5C
:1019600080917E0190917F01A0918001B0918101D1
:101970008093A8029093A902A093AA02B093AB020D
:10198000B9CF80E50E949963C12CD12C76018823C0
:1019900021F00E944F676B017C0183E50E949963EF
:1019A000882361F00E94B96720E030E04AE754E400
:1019B0000E942ADC0E94C7E36B017C010E9425295A
:1019C00080911510811105C060E087E199E10E94C6
:1019D000EC500E94DCC1C60ED71EE81EF91E0E9404
:1019E000DCC16C197D098E099F0997FFA2CF80E0A9
:1019F0000E948282F4CFA12E10E04C2D4170B42EB3
:101A000046CD60E070E080EA90E449CDA301920108
:101A1000C701B6018BCD60E082E399E10E94EC50F2
:101A20000E94F48080E299E10E94C47B72CE0E9401
:101A30008D9E7FCF0091FF1210910013D8012D9140
:101A40003D914D915C916091720170917301809113
:101A50007401909175010E94E3E2AB01BC0188E53D
:101A60000E94E16769837A838B839C83F8012481D8
:101A7000358146815781609176017091770180911F
:101A80007801909179010E94E3E2AB01BC0189E504
:101A90000E94E1676D837E838F839887BE016B5FB1
:101AA0007F4FCE0101960E94E4B8882309F441CF0C
:101AB00080E00E94A2730E94CF3A61E085E40E9418
:101AC000996721E0482FBE016B5F7F4FCE010196E1
:101AD0000E941ABA6B017C0149815A816B817C8119
:101AE0008DE499E10E94EF7B4D815E816F81788565
:101AF00088E499E10E94EF7BB701A60183E499E1B4
:101B00000E94007C0E94B63A0E94463C12CF10E030
:101B1000002331F0F6E0FF1508F438CEE11033CEA3
:101B200080E1E2E7F1E0ACE9B2E001900D928A9544
:101B3000E1F7002319F16F2DFF0C770B880B990B40
:101B40000E94CBDB2091B9023091BA024091BB02D6
:101B50005091BC020E942ADC2091AC023091AD026F
:101B60004091AE025091AF020E94E3E260939C026A
:101B700070939D0280939E0290939F02EE2019F134
:101B8000612F110F770B880B990B0E94CBDB2091F3
:101B9000BD023091BE024091BF025091C0020E942E
:101BA0002ADC2091B0023091B1024091B2025091F2
:101BB000B3020E94E3E26093A0027093A1028093BB
:101BC000A2029093A30260E080E50E9499678823B7
:101BD000C1F10023D1F0E091FF12F09100132081B8
:101BE00031814281538160919C0270919D0280916C
:101BF0009E0290919F020E94E2E260939C02709389
:101C00009D0280939E0290939F02EE20D1F0E0917E
